:020000040000fa
:08000000c07d040001000000b6
:020000040000fa
:100200005406040000000000820604000000000004
:10021000af202200807f2200000188000000000043
:10022000050007000c000700464502000000000022
:100230000040da000000fe004440a90000c92b0085
:100240000000e0000300320020002000a001880030
:100250004440a8000000060040c82600110020000d
:100260001600370062004000e080480091018800dd
:100270009001ba0062004000e080480091018800cf
:100280009002ba0062004000e08048000002eb00eb
:100290006028e10005003a008301e900070033000f
:1002a000038009000059eb00040037006128e100d9
:1002b000010032000082eb00050007009101880078
:1002c0001001ba000200e000e6ff3a00000005005d
:1002d000910188008002780062004000e0804800c0
:1002e0003559ba008301e900080032002559ba00e7
:1002f0008301e900050032000400e000f4ff320051
:1003000015d9ba008301e900f1ff3a0000000600a8
:100310001004b100070035009001b1000400340062
:100320007000b100030035009001b10001003c00f5
:100330001000050000000500ea874700889fbe0006
:100340008a9fbe008c9fbe008e1f780080067800ba
:10035000010678008204780000047800010037006c
:100360000804e8001800fb00a10207000000e000fc
:10037000fbff3a0098407800d0c2b30080cf500015
:100380000400320000c0e900d0ef9f0080cf500091
:1003900002003a00d1ef9f000804e8000900e000e5
:1003a00046003500e18f5400440032004002200036
:1003b000808f540041003c000900e0000d00340033
:1003c000f08f54001a003a0000c3b300984f100099
:1003d00017003a009840900080c7b30080cf5000cb
:1003e0001200320080c5b30080cf500010003a00e8
:1003f0000e00370000c3b300984f10000200320017
:10040000a90020000a0037009840900080c7b30080
:1004100080cf5000040032008900200080c5b30066
:1004200080cf500002003a00090120000884e80053
:10043000d8b79f0000c3b300984f100002003a00e5
:10044000d84f1000feff32006055b8000807780052
:100450000e003700fab79f008bbf9f00405e21005f
:1004600000425200c4ef9f006149b9000a00be007b
:10047000e81107004fea97000401fb00cf91de006e
:1004800000054100818549000804e8001800fb00d0
:10049000400107008000780009017800405e2100db
:1004a0005b020700000278000000e000e9ff3a006c
:1004b0005fb09700880f500005003a000c00e00084
:1004c000010032000d0e78006000b80027003700f0
:1004d0008e00540090602100694078000000fb000d
:1004e00000805000170033004240a9000f003c007c
:1004f0004fe997000200fb00cf80de0000005500ae
:1005000081805d00800f5500818f5d0007003900fc
:100510006149b900ef1207007fb197008fb99700ca
:10052000820f5000838f5800060032002002200006
:1005300060be88000085eb008085eb00b3c2b3008d
:10054000d3ef9f00d0c2b3005fea9700804f520004
:1005500002003a0060051500e0851d000c00e00077
:1005600001003200080e78000a00be004f07780034
:100570004f06be004f05be004f04be00af00b100e5
:1005800000000600f8874700889fbe008a9fbe00d3
:100590008c9fbe008e1f7800c0b79f0001047800ba
:1005a0000206be000005780078805700210207008f
:1005b000680760000030a100e10f500043003a00de
:1005c000cfb0970024002000c3fd2f008f81410091
:1005d000080178000a00780098020700800578007a
:1005e0000000e00007003a006000b8006011b800a9
:1005f000d0b79f00e1b79f00f2b79f0083bf9f0075
:100600002d0037006400b800c2fd2f000f0141002b
:10061000000041001000be003b0e0700d0b79f0055
:10062000e1b79f00f2b79f0083bf9f000b05e90071
:100630004240a900200034006450b800c2fd2f00e1
:100640000f014100000041001000be00e00f50000b
:10065000e08f5800150032000a8455006844b80045
:100660004273210002044400270e07000002be006e
:100670000203be003800be002801be00580f07006c
:100680000002be000203be005fb09700efb097000b
:100690007fb197008fb997009e0e0700d0b79f00db
:1006a000e1b79f00f2b79f0083bf9f000a05e900f2
:1006b0004240a900e0ff3c006fa89700ffa8970008
:1006c0000c0240008d82480045003700e20f5000c8
:1006d00049003a00cfb0970000027800c3fd2f0018
:1006e0008f814100080178000a0078003903070073
:1006f000800578000000e00007003a006000b800c4
:100700006011b800d0b79f00e1b79f00f2b79f001b
:1007100083bf9f002d0037006400b800c2fd2f008a
:100720000f014100000041001000be00f60d07005f
:10073000d0b79f00e1b79f00f2b79f0083bf9f0033
:100740000b05e9004240a900200034006450b800c5
:10075000c2fd2f000f014100000041001000be004b
:10076000e00f5000e08f5800150032000a84550059
:100770006844b8004274210002044400e20d0700fe
:100780000002be000203be003800be002801be0009
:10079000130f07000002be000203be005fb0970007
:1007a000efb097007fb197008fb99700590e0700ff
:1007b000d0b79f00e1b79f00f2b79f0083bf9f00b3
:1007c0000a05e9004240a900e0ff3c006fa997003c
:1007d000ffa9970076805700f60307000c02be00c1
:1007e0005fb09700efb097007fb197008fb9970087
:1007f0008004070013003700e30f500004003a00a4
:100800006000b8000200200003ff27000600370048
:10081000e40f500009003a00f0ff2f00f1ff2f0015
:10082000f2ff2f00f3ff2700d0b79f00e1b79f0032
:10083000f2b79f0083bf9f00060037006000b8003a
:100840006011b800d0b79f00e1b79f00f2b79f00da
:1008500083bf9f005fb09700efb097007fb1970014
:100860008fb997000e00e0000100320003f0a200f3
:100870004f0778004f06be004f05be004f04be0074
:100880008f01b10000000600800178000200e00046
:10089000070032001104e00005003200b159780071
:1008a0000201e900020032001104e000fbff3a00ff
:1008b0000200e000030032008059eb000201e90071
:1008c000fdff3a00000006001004e0000a003200bc
:1008d000010178001104e000050032009041780029
:1008e00092cf5100050032005204e000fbff3a00b5
:1008f0005004e000f6ff3a000000eb0000000600a4
:10090000800178000200e000030032008159780085
:100910000201e900fdff3a000000060080007800b7
:100920001004e000020032005104e000feff3a0033
:1009300000805000000006000400fa00889fbe00fe
:100940008a9fbe008c9fbe0080bf9f0091bf9f000a
:100950000206be00b51007000001be000004be0084
:100960000c00be00ab1007000fb997009fb99700ad
:1009700000055100818559000800be000a01be0033
:100980004f06be004f05be004f04be000080fa00b7
:1009900000000600800078001104b100030035005b
:1009a0009101b10001003c000050a00000000600d1
:1009b00080027800800178001004e0000b00320013
:1009c0000101780012427800058051000404e00023
:1009d00007003200934f1200020032000201e800cb
:1009e000f8ff37005304e000f5ff3a00058051009e
:1009f00000000600800178001004e0000a003200c8
:100a0000010178001104e000050032001042780076
:100a1000924f5200040032005204e000fbff3a0003
:100a20005004e000f6ff3a0003005000000006000a
:100a3000800178000200e00003003200b159780024
:100a40000201e900fdff3a00000006000200fa0082
:100a5000889fbe008a9fbe008c1f7800000578002a
:100a600081047800020678000100e00001003a00ed
:100a7000ec8457000a047800010037000804e800fd
:100a80001800fb00da0007000000e000fbff3a005e
:100a900098407800d0c2b30080cf500003003200ed
:100aa000bbc2b3008bcf500002003a0081457800f2
:100ab0000804e8000c0178000800be001efe0700d4
:100ac0000001be00990f540001003a008a0c780022
:100ad000990f550003003a00e00f5100e08f5900d4
:100ae0000e003a00b0c2b30080cf550003003a00b8
:100af000e00f5100e08f590008003500d0c2b3006c
:100b000080cf55000f003a000000200001002800af
:100b1000800f5100818f59000a003600200220000a
:100b200060be880002002000030028006b404000e7
:100b300080cf550008003200f2ff2f00f3ff27009e
:100b400005003700d0c2b30080cf550002003a0044
:100b500060011100e08119000200be004f0678001c
:100b60004f05be004f04be000080fa0000000600e2
:100b700000017800314978003204e000fdff3a00be
:100b800000000600800078001106b1000300350067
:100b90009101b10001003c000050a10000000600de
:100ba0000003b100030035009000b10001003c00db
:100bb000100005000000050010417800914f510021
:100bc00006003a008001eb000204e0000a00320057
:100bd00050417800d14f5100faff320010407800a8
:100be000914f5000020031000080eb0001003700ff
:100bf000100020008001780003007800000006004b
:100c0000800278000200e0000e003200954178007a
:100c10001142780084cf5100030032000080eb00c5
:100c200009003900100005000000eb000304e0009b
:100c3000050032008502e8008100e8000201e900b9
:100c4000f2ff3a000000eb00000006000200e000a6
:100c50000b0032001042780091417800834f52001f
:100c6000030032000080eb00060039001000050090
:100c70000000e8008100e8000201e900f5ff3a0009
:100c80000000eb000000060090cf100005003200cd
:100c90001004e00001003a0000000500d0cf100071
:100ca000fbff3a0000000600881f7800020478006d
:100cb0005fff0700080040004f04780000000600b6
:100cc0000000fa00881f7800000478003fb9970000
:100cd000ea8157008000780040652000f403070097
:100ce000800078000000e000020035000040eb00ca
:100cf00000f47800010078004f0478000080fa00ca
:100d000000000600889fbe0000047800820478007e
:100d100010019000890f5100010031008204780019
:100d2000180078000901780041ff0700188c440082
:100d30001800900009005000100498000800780086
:100d40004f04be00000006000400fa000100e000ad
:100d500004003a000f80e900e0bf9f000008eb00ac
:100d600003003700e0bf9f008100e900f1bf9f0052
:100d7000e480570020682000cd030700efb89700fb
:100d80008048eb000080fa000000060001017800b6
:100d900000027800110009000200d8000002fd00e6
:100da0000491b900820250000400be000000060059
:100db00080017800000178001004e0000200320099
:100dc0005204e000feff3a0011407800004978002c
:100dd0000004e0000400320051407800006978000f
:100de0000004e000fcff3a00030078000000060069
:100df0006900e100040035006d00e10003003400eb
:100e00000002b100010032000000050010000500e2
:100e10000200e0000500320090cf10000400320014
:100e20000000e8000201e900fbff3a000000eb00cf
:100e300000000600889fbe008a9fbe008c1f7800bd
:100e40000006780081057800100478000005eb00aa
:100e5000010037000804e8001800fb00e4ff070069
:100e60000000e000fbff3a0098407800d0c2b300d9
:100e700080cf500002003a008a00200003003700b3
:100e8000b0c2b30080cf500001003a000804e8006f
:100e900098407800e2c6b30082cf500003003200d1
:100ea000e3c4b30083cf50001f003a00d84078005d
:100eb00010c6b30080cf50000300320010c4b3004e
:100ec00080cf50002a003a00d840780082cf5000ee
:100ed00003003200e0c4b30080cf500024003a0089
:100ee0000804e800880478004a00200080c2b300ab
:100ef000984f100007003a005900fb00210407003a
:100f00000000e000fcff3a00f0c5b300994f10006c
:100f1000f9ff320090c2b300994f10003c003a0034
:100f20000904e8003a00370090c6b30080cf5000b3
:100f30000300320090c4b30080cf500038003a0064
:100f400058407800824f500002003200834f50001a
:100f500007003a00d840780060c6b30080cf500048
:100f60000600320060c4b30080cf5000030032009e
:100f70001c0478000005eb00250037003a00b300a0
:100f8000d840780093c6b30083cf500003003200ee
:100f900090c4b30080cf50001d003a008800e800e4
:100fa00011417800e0c6b300804f510003003200c9
:100fb000e0c4b300804f510015003a005141780061
:100fc000834f51000300320090c4b300804f5100a2
:100fd0000f003a005141780040c7b300804f5100e4
:100fe0000300320040c5b300804f510008003a00b2
:100ff0005141780090c7b300804f51000300320088
:1010000090c5b300804f510001003a000104e80090
:101010000b00e00003003200880d7800010037006b
:101020000a00a000080e78000a0078004f06780039
:101030004f05be004f04be0000000600e6874700d3
:10104000889fbe008a9fbe008c9fbe008e1f7800c6
:10105000f0b79f000105780082bf9f00030678006b
:10106000830478006920b900000478008006eb0052
:1010700000c3b3009a4f100003003a001d00200087
:10108000da4f1000fdff32008005eb00000eeb0090
:101090003c16780028003700888f550016003d0068
:1010a00092002000110009008205d800010078009c
:1010b0000000e00003003a00e4844400800ceb00f0
:1010c000b91478001900be00a2002000030020001f
:1010d000d00e07001a4178000201fb00cf91de001c
:1010e00000004100818049000003b1000180b1008f
:1010f000808cbe000d003700100020000100200091
:101100001c0e40005c964800888f550008003a008d
:1011100040c3b3009a4f10000500340012002000b5
:1011200003002000990c4100d99449008b05e80088
:101130000a05e8001d0020001a00fb0098fe0700c9
:101140000000e000d4ff3a008b0f540001003d0086
:1011500088057800e0c2b3009a4f100001003a0001
:101160000a05e8000b00e00029003a0000c3b300c4
:101170009a4f100026003a000081eb008081eb00be
:101180001c0e41005c9649001d002000da4f100043
:10119000f9ff32001e003700888f55001a003d000d
:1011a00092002000110009008205d800010078009b
:1011b0000000e00003003a00e4844400800ceb00ef
:1011c000b91478001900be00a2002000030020001e
:1011d000900e07001a4178000201fb00cf91de005b
:1011e00000004100818049000003b1000180b1008e
:1011f000808cbe008b05e8000080eb008080eb0057
:101200001c0e40005c9648000a05e8001d00200006
:101210001a00fb0062fe07000000e000deff3a005b
:1012200092002000110009008205d8000104780016
:101230000800e00010003200690414001902be002a
:10124000e00f5200e08f5a00070032006440b800ff
:1012500082752100020040001001be000400be00a3
:101260006c0e0700808cbe00888545006140b90087
:101270001c1e10001c961800e88f5500100034004a
:101280001900be00e00f5000e08f58000c003a003b
:10129000e985550090002000010020001c0e400050
:1012a0005c964800e4845400e88f55000400340044
:1012b0001900be00e00f5000e08f5800f4ff32002c
:1012c0000d00e000310032009a40780050c6b300b3
:1012d00080cf50000300320050c4b30080cf5000d4
:1012e0002a003a00da407800b0c2b30080cf500044
:1012f000040032000047780000c0e80080cf5000b2
:1013000002003a00014778000a05e8006044b8008e
:101310008006eb0012003700f00f2e00515f200016
:10132000800f5400818f5c000b003c00a200200065
:10133000030020000800be00360e07001a417800a6
:101340000201fb00cf91de000004410081844900ce
:101350000803b1000980b1000a05e8001d00200063
:101360001a00fb000efe07000000e000eaff3a0052
:10137000d0c2b300804f570002003a00600414004e
:10138000e0841c001c0e44005c964c008fb8970053
:101390000100e00006003200ffb097000d00e00001
:1013a000010032008a0078000fb997000109780027
:1013b00092002000110009008205d8004f07780034
:1013c0004f06be004f05be004f04be006f00b100c7
:1013d00000000600e6874700889fbe008a9fbe0087
:1013e0008c9fbe008e1f7800f0b79f00010578002b
:1013f00082bf9f0083057800030478006720b9004e
:10140000800478008006eb0000c3b3009a4f100000
:1014100003003a001d002000da4f1000fdff3200eb
:101420000006eb00800deb00bb1578002e003700a6
:10143000890f560019003d0072002000811f7800be
:10144000110009000206d80001007800cf007800e2
:101450000000e00003003a0064044400000ceb00cc
:10146000381478001801be004418dd00cc11de00ed
:10147000830170004411dd00006c210000805000e9
:10148000716d210060c078000000fb00cf80de009d
:10149000001c410001944900100037001200200098
:1014a000030020009b0d4100db954900890f560089
:1014b0000b003a00006c210000805000716d21008b
:1014c00060c07800e74f5000050034001000200095
:1014d00001002000180c4000589448000c06e80059
:1014e0000a05e8001d0020009a00fb0062012000b0
:1014f000006c210046fe0700800078000000e0003c
:10150000cbff3a008c8f540001003d0009067800a3
:10151000e0c2b3009a4f100001003a000a05e8004b
:101520000c00e0002c003a0000c3b3009a4f1000fa
:1015300029003a000081eb008081eb009b0d410007
:10154000db9549001d002000da4f1000f9ff320042
:1015500021003700890f56001d003d007200200059
:10156000811f7800110009000206d80001007800f0
:10157000cf0078000000e00003003a00640444005b
:10158000000ceb00381478001801be004418dd0090
:10159000cc11de00830170004411dd00006c2100dd
:1015a00000805000716d210060c078000000fb00d9
:1015b000cf80de00001c4100019449000c06e800c9
:1015c0000081eb008081eb009b0d4100db95490021
:1015d0000a05e8001d0020009a00fb0062012000bf
:1015e000006c21000afe0700800078000000e00087
:1015f000d8ff3a0072002000110009000206d8004e
:10160000010078000000e0000d00320067001000cb
:101610006402b9001801be000402e90003003300af
:101620000201410083814900fbff3700028cbe00ac
:1016300000064600cf80de009b1d10009b95180021
:10164000e60f5600100034001800be00e00f5000f6
:10165000e08f58000c003a0067065600700020002a
:10166000010020009b0d4000db95480064045400fd
:10167000e60f5600040034001800be00e00f5000d2
:10168000e08f5800f4ff32001b00be004209dd006d
:10169000ce00de00810071004200dd00808dbe00c2
:1016a0000d00e000310032009a40780000c7b3001e
:1016b00080cf50000300320000c5b30080cf50003f
:1016c0002a003a00da407800b0c2b30080cf500060
:1016d000040032000047780000c0e80080cf5000ce
:1016e00002003a00014778000a05e8006044b800ab
:1016f0008006eb0012003700f00f2e00515f200033
:10170000800f5400818f5c000b003c00a200200081
:10171000030020000800be003e0d07001a417800bb
:101720000201fb00cf91de000004410081844900ea
:101730000803b1000980b1000a05e8001d0020007f
:101740001a00fb0016fd07000000e000eaff3a0067
:10175000d0c2b300804f570002003a00600414006a
:10176000e0841c009b0d4400db954c008fb9970072
:101770000300e00006003200ffb097000d00e0001b
:10178000010032008a0078000fb897000108780045
:1017900072002000110009000206d8004f077800ef
:1017a0004f06be004f05be004f04be006f00b100e3
:1017b00000000600881f78008a9fbe0000047800a1
:1017c0000205be00300190000200d000c500de001e
:1017d000f07f2000808f50000c003a006f00610005
:1017e00008003a00280090000000e00005003a00e0
:1017f000180090000000e00002003a001800e0002d
:101800001c003200200020005d0037000100e000d5
:1018100006003a0008007800e80107008000780020
:101820000000eb000100e00055003c006108b90039
:101830000a0540008b854800e07f2000800f55009e
:10184000e08f5d000d003400380090006022b80089
:101850000600200007ff2f000000e0000300350015
:101860006022b8000600200007ff2700049cbe008d
:101870000694be001000200041003700b800900020
:10188000e00f5500e08f5d0005003400f0002800f7
:1018900000806000c450dd00010070003600370099
:1018a00000002800808260006f8060000040a0007f
:1018b0003004980061055500e0855d00c0fc2f00f4
:1018c000f1ff2f00800f5500818f5d0006003d0065
:1018d000350498000000eb002004980010049800e4
:1018e000000ceb00260037000a027800f00f4500dc
:1018f0000b003c0018009000000c780028009000bd
:101900001004980038009000200498000000eb00bc
:101910003004980070024200f00f4200f5ff3400de
:101920000402ea0012003200180178000411de00ff
:10193000f0011200180090008300dd00010c71001e
:101940000400de00280190008310dd00010070001b
:10195000100498000411de00380090008301dd00bf
:1019600003017100220498000400de003004980096
:101970003800900005007000300498000080eb00f3
:101980004f05be004f047800000006000200fa0078
:10199000889fbe008a9fbe008c1f780000067800da
:1019a0000404be000605be00800078006c8057006d
:1019b000d50107003c00be002c01be000802be009d
:1019c0000a03be00860a0700009ebe000296be0003
:1019d0002fb99700cf91de000c00780075ff07004b
:1019e0004f0678004f05be004f04be000080fa008d
:1019f000000006001800fa00889fbe008a1f7800c9
:101a000090b79f00a1b79f00b2b79f00c3b79f00d8
:101a10000404be00e00f5200e08f5a009c00320028
:101a20006022b8006033b800370a07000000e00009
:101a3000970032006000b8000200200003ff23007e
:101a4000d0b79f00e1b79f00f2b79f0083bf9f0010
:101a5000e00f5400e08f5c0048003d00600414007b
:101a6000e0841c000005eb001a0032000808a30007
:101a7000100032006850b800e2622100020040000d
:101a80003002be002003be005fb09700efb09700a9
:101a90007fb197008fb99700510a07000002be007e
:101aa0000203be00d4b79f00e5b79f00f6b79f00c2
:101ab00087bf9f008904d1000884d3000a05e8008d
:101ac000e00f5400e08f5c0002003200e70f550089
:101ad000e6ff36005fb29700efb297007fb3970042
:101ae0008fbb97006000b8000200200003ff2300b6
:101af000080907000002be000203be007e805700f6
:101b0000a2ff0700000578000000e00059003d003a
:101b1000e00f5400e08f5c0056003200e3662100c5
:101b20003302be002303be006000b80002002000a4
:101b300003ff2300f708070090bf9f00a1bf9f008d
:101b4000b2bf9f00c3bf9f001fba9700afba9700f4
:101b50003fbb9700cfbb97007e8057008bff0700ed
:101b6000000578000000e00042003d0061045400e0
:101b7000e0845c00f4ff3a003e003700e00f5400c0
:101b8000e08f5c003b0034000005eb000808a30078
:101b9000100032006850b800e262210002004000ec
:101ba0003002be002003be005fb09700efb0970088
:101bb0007fb197008fb99700090a07000002be00a5
:101bc0000203be00d4b79f00e5b79f00f6b79f00a1
:101bd00087bf9f008984d1000884d3000a05e800ec
:101be000e00f5400e08f5c0002003400e70f550066
:101bf000e6ff36005fb29700efb297007fb3970021
:101c00008fbb97007e80570060ff070000057800bb
:101c10000000e00017003d00e00f5400e08f5c0082
:101c200014003400e16621005101be004100be00f5
:101c3000d0b79f00e1b79f00f2b79f0083bf9f001e
:101c40005fb29700efb297007fb397008fbb97000a
:101c50007e8057004dff0700000578000000e0007f
:101c600004003d0061045400e0845c004240a9008f
:101c7000f3ff3c00000120000a00e00003003200f6
:101c8000e10f550002003a00800020004c010700df
:101c90001fb09700afb097003fb19700cfb197004a
:101ca0004f0578004f04be000080fa0000000600d7
:101cb0006200fa00889fbe008a9fbe000004be003a
:101cc00002057800830078006a805700470107000a
:101cd000f88f9f0089979f000000eb00909f9f0066
:101ce0001a80fb008005fb000000ea00cf04de0044
:101cf0000904780050022000808f550001003a004e
:101d00000904e9000800e0000c0034000f9097007f
:101d1000080178008a007800ff899700030001001d
:101d200080979f008080eb000000e0009000320070
:101d30001f98970008004000909f9f0009054500ec
:101d400050022000808f5500040032000b00e0009c
:101d5000e3ff3a009f989700850037000000eb00f2
:101d6000f0979f00e0979f00d0979f00c0979f003b
:101d7000b0979f00a0979f00b09f9f000900370079
:101d800020792100008050000000d00081792100de
:101d900001004000bf98970090807000b19f9f00a5
:101da0000a05e8009a00fb0020792100b6fb070035
:101db000800078000000e000f1ff3a00a0c2b3000c
:101dc0009a4f10000e003a003fb897000080e900db
:101dd000b0bf9f0010007800a09f9f000000e000af
:101de00005003d000000ea00a09f9f003f9897007b
:101df0000020a000b09f9f000a05e80011003700f6
:101e0000a19f9f000b003700af989700f0ff2700bd
:101e1000808f5000060032006a09b9001a00fb00ea
:101e20000200400001fd2f0001004000a09f9f0024
:101e30000a05e8001a00fb0059fb07000000e0005b
:101e4000f1ff3a00e0c2b3009a4f100003003200e5
:101e50000080eb00809f9f001c003700a0c2b300f1
:101e6000da4f100007003a003fb897000080e90001
:101e7000b0bf9f0010007800809f9f000a05e80017
:101e8000120037000000eb00809f9f000b0037001e
:101e90008f989700f0ff2700808f500006003200d7
:101ea0006a09b9001a00fb000200400001fd2f0082
:101eb00001004000809f9f000a05e8001a00fb0017
:101ec00037fb07000000e000f1ff3a009a00fb003a
:101ed000002022006cfb07008040eb000000e000c7
:101ee00001003200ba407800817f9f0080c6b300b5
:101ef00080cf500004003a009acf100002003a0050
:101f000066405000070037008f789700c0c6b300c6
:101f100080cf500005003a009acf100003003a002d
:101f200065404000807f9f000a05e800a0fb2f006d
:101f3000008447003a01fb0088017800ea805700de
:101f400060f92f000f004000780107000000e0005a
:101f500006003a008800780060f92f000f0040006a
:101f6000a40007000000e0005dff3d008080eb0062
:101f7000010078004f05be004f04be000080fa004b
:101f8000000006000003b1000b0035009000b10016
:101f9000080034008000b100070035009001b10056
:101fa000040034007000b100030035009001b1005e
:101fb00001003c0010000500000005000002780050
:101fc000300090000100280001036000150020008f
:101fd0006f0060003002980008003a002400900072
:101fe0000000e00005003a00140090000000e0004e
:101ff00002003a001400e0003e003200340090007d
:102000000000e0000b003a0024009000300298002d
:10201000140090002002980014007800100298002c
:10202000000aeb00f0825200340090000000e00053
:10203000f5ff320034009000ef0f500014003e0016
:102040008001d000a40090004f08de008081710064
:10205000330298008100d000140190004f10de0080
:1020600080807000210298000201d0009400780066
:102070004f08de000001710012029800010ad00032
:102080008502e90003007800ef8f5100ecff360075
:10209000b4019000ff8f5100130036001401d100ed
:1020a00014009000cf00dd00010a71000000d10093
:1020b000a40090004f09dd0002007000100298009b
:1020c0008100d1004f18dd0080807000210298004f
:1020d0000300d100300298008502e80080017800fa
:1020e000ff0f5000edff3e00340090006f006000d5
:1020f0003002980034009000060070003002980012
:102100000500780000000600889fbe00800478006b
:1021100001047800310090000000d0004501de008d
:10212000f07f2000800f510010003a00800ceb007f
:10213000310090006f00600008003a00210090001c
:102140000000e00005003a00110090000000e000ef
:1021500002003a001100e0000200320020002000de
:102160001500370010002000130037000200e000c7
:1021700005003c000100780090ff07000001780096
:102180000000e0000a003c0038009000f100280048
:102190000100600001fe230001007000300498007f
:1021a00020c02f00800c41000080eb0002003700af
:1021b000800ceb000000eb004f04be0000000600a6
:1021c00080007800650060000300320010022000eb
:1021d00060be8800000006007880600002003200c7
:1021e0002002200060be8800000006000108780080
:1021f000000006000400fa00889fbe008a9fbe000f
:102200008c1f7800000478000106780070089000a8
:10221000f800900001005000880890000100500074
:102220009808900001005000a8089000010050009c
:10223000b808900001005000c808900081055000c7
:102240000002220090bf9f0000032300a0bf9f0058
:10225000081090000028a30018003a000b00e000ce
:10226000160034000b0578008a047800e20f550050
:1022700001003600290020000900e0000c003400b5
:1022800058009000c801900009017800ee805700c6
:1022900003000100500498008080eb000000e00083
:1022a0009c0032006808900009004000600c980013
:1022b000090555004240a900ebff3c007801900061
:1022c0000200e0000c00340058009000c8019000ab
:1022d0008c00780003000100500498008080eb001f
:1022e0000000e0008b00320068089000f8009000c9
:1022f00001004000600c9800080890000000e00019
:1023000016003400000578008a047800e20f5500ba
:1023100001003600290020000900e0000c00340014
:1023200058009000c801900009017800ec80570027
:1023300003000100500498008080eb000000e000e2
:10234000740032006808900009004000600c98009a
:10235000090555004240a900ebff3c001809900018
:102360000200e0000c003400e800900058009000eb
:10237000c801900003000100500498008080eb0029
:102380000000e000630032006808900098089000a8
:1023900001004000600c9800280890000000e00058
:1023a00016003400000578008a047800e20f55001a
:1023b00001003600290020000900e0000c00340074
:1023c00058009000c801900009017800ec80570087
:1023d00003000100500498008080eb000000e00042
:1023e0004c0032006808900009004000600c980022
:1023f000090555004240a900ebff3c003809900058
:102400000200e0000e003400e80090001808900080
:102410008080400058009000c80190000300010037
:10242000500498008080eb000000e000390032008a
:1024300068089000b808900001004000600c980007
:10244000480890000000e000160034000005780005
:102450008a047800e20f55000100360029002000b0
:102460000900e0000c00340058009000c801900002
:1024700009017800ec805700030001005004980027
:102480008080eb000000e00022003200680890002d
:1024900009004000600c9800090555004240a90061
:1024a000ebff3c00081090000028a3001800320049
:1024b0000b00e000160034000b0578008a04780059
:1024c000e20f550001003600290020000900e0005d
:1024d0000c00340058009000c801900009017800f9
:1024e000ee80570003000100500498008080eb004c
:1024f0000000e0000700320068089000090040007a
:10250000600c9800090555004240a900ebff3c0013
:102510008000eb00010078004f0678004f05be00f8
:102520004f04be000080fa0000000600889fbe0035
:102530008a1f7800000478000102780002457800c4
:10254000830478000200fb00cf80de005002b1005f
:102550000180b10032052000820f5000e08f58004a
:102560008c013e00006001008401370089013700c2
:102570008801370087013700860137008501370061
:102580008401370083013700820137008101370061
:10259000800137007f0137007e0137007d01370061
:1025a0007c0137007b0137007a0137007901370061
:1025b0007801370077013700760137007501370061
:1025c0007401370073013700720137007101370061
:1025d000700137006f013700ed0037006d013700e3
:1025e0006c0137006b013700e9003700e800370065
:1025f000e7003700670137006601370065013700e3
:102600006401370063013700620137006101370060
:10261000600137005f0137005e0137005d01370060
:10262000420137005b0137005a013700590137007a
:102630005801370080003700560137005501370038
:102640005401370053013700520137005101370060
:10265000500137004f013700cd0037004d013700e2
:10266000150037001c003700c9003700c8003700cc
:10267000c700370047013700170037004501370012
:10268000440137004301370042013700e3003700bf
:1026900069003700160137003e0137003d01370061
:1026a000220137003b013700630037003901370052
:1026b00038013700600037006e01440012007800d6
:1026c000808141009480e900010a78000009e80057
:1026d0009149780038013700a8609000c0c6b30067
:1026e00080cf50000a003a009400780064805000c7
:1026f000000a78001000be004f89de00cf91de0096
:102700000002be0002037800820378001500370043
:1027100010c7b30080cf500002003a0014017800c7
:102720000400370014017800a0c6b30080cf500029
:1027300005003a0068005100000a78003002be002f
:102740002003be00070037000280e900000a78007d
:102750001000780000027800cfa2de0005037800a8
:1027600086037800049cbe000694be00a86090001a
:1027700080c6b30080cf50000f00320020c6b300e7
:1027800080cf500006003a00184078000000fb009f
:10279000cf80de0001017800820178000a00370056
:1027a00040c7b30080cf50000300320066404000b5
:1027b00080cf500006003a0018007800cf80de007d
:1027c0000101780082017800009cbe000294be00e6
:1027d0003800be002801be00e00f5000e08f580016
:1027e000e00f5900e08f590004003d006e014400e5
:1027f00092007800d0c2b3000c003700081090009f
:102800000018a300040032006e014400920078001a
:10281000b0c2b300050037000008a3005700320023
:102820006e0144009200780000c2b30080f478008a
:102830000109e80051003700a8609000c0c6b3004d
:1028400080cf500006003a00940078006480500069
:10285000000a78001002be006033b800150037008f
:1028600010c7b30080cf500002003a001401780076
:102870000400370014017800a0c6b30080cf5000d8
:1028800005003a0068005100000a78003002be00de
:102890002003be00070037000280e900000a78002c
:1028a00010007800000278000500200006002000db
:1028b00007002000049cbe000694be00a8609000a3
:1028c00080c6b30080cf50000f00320020c6b30096
:1028d00080cf500006003a00184078000080fb00ce
:1028e0000100200002002000030020000a00370041
:1028f00040c7b30080cf5000030032006640400064
:1029000080cf500006003a00180078000100200037
:102910000200200003002000009cbe000294be00c4
:10292000081090000038a300140032003800be00e8
:102930002801be00e00f5000e08f5800e00f590062
:10294000e08f59000d00320080c7b300804f550062
:102950000300320080c5b300804f550007003a00e5
:102960006e0044009000780002c3b30082f4780047
:102970008100e8008af478000108e80078009000ff
:1029800000804400600498008a40780064003700aa
:102990001401780068005100000a78005001be0060
:1029a0004000be00009cbe000294be0038009000b3
:1029b0000000e00004003d006e0144009200780039
:1029c000d0c2b3000c003700081090000018a3001c
:1029d000040032006e01440092007800b0c2b300df
:1029e000050037000008a300050032006e01440016
:1029f0009200780000c2b30080f478000109e8007a
:102a00007800900000804400600498008a407800bc
:102a1000080078001e01070067003700286090005a
:102a20008000fb00c0062000808f50002300320091
:102a30000a003c0064005000808f500026003200e5
:102a400004003c0066005000808f50000b003200f4
:102a500021003700a00620000500370040072000b5
:102a6000808f50001c0032001b003c0063005000af
:102a7000808f500007003200170037001480e900f3
:102a8000000a780010007800485c90000848780040
:102a9000490037001480e900000a7800100278002d
:102aa00068089000cf80de00010178008201780084
:102ab000009abe000292be003f0037001480e90079
:102ac000000a78001001780068089000cf80de00ce
:102ad0000089be00380037001480e900000a780041
:102ae00010007800680c9000080878003200370069
:102af0001480e900000a780010007800cf80de0022
:102b00000101780082017800009cbe000294be00a2
:102b100078009000008044006004980081c7b300f2
:102b20000800780028000700230037001480e9001f
:102b3000000a78001000780060049800580990009e
:102b40000200e00002003d0074f7070009003700b2
:102b50008000eb00aef80700800078000000e00085
:102b60000300320068009000008050000100370030
:102b700058089000100c98000f0037006e014400b8
:102b80009200780050c2b30080f178000109e8009b
:102b900009003700ee0044001100780080814400f5
:102ba0000a4278008008e8000a04e00001003a00c8
:102bb00054c2b300844978000000eb004f05780050
:102bc0004f04be00000006006f02b000889fbe00e8
:102bd0008a9fbe008c9fbe008e1f78008006780002
:102be000b0722100b0b79f0080c5b30080cf500005
:102bf00002003200a2712100b2b79f0083002000c2
:102c0000c3b79f00f0c6b30080cf50000a00320067
:102c10006940400080cf500005003200a400200031
:102c2000c4b79f0080c5b30080cf500002003a00b7
:102c300000012000c0b79f008e0120003d04be00af
:102c40002d05be0040c6b30080cf50000300320007
:102c50006540400080cf50000a003a00e00f540069
:102c6000e08f5c00e00f5d00e08f5d0005003d003f
:102c70000800be000a01be00fb0707000205be00f7
:102c80000004be00e00f5400e08f5c00e00f5d0028
:102c9000e08f5d0003003a005d0890000000e00056
:102ca0000c0032007e012000cfb0970001027800b6
:102cb000cfa2de0005037800860378000800be007e
:102cc0000a01be007e0807003fb29700644078000a
:102cd000d0e79f004fb09700cf80de000101780061
:102ce00082017800d0b79f00e1b79f00f2b79f0044
:102cf00083bf9f000203be000002be000800be00aa
:102d00000a01be0067080700809ebe008296be00d2
:102d1000e00f5000e08f5800e00f5900e08f59009d
:102d2000220034000e00e000200034003d00be0010
:102d30002d01be005fb29700efb297007fb39700fe
:102d40008fbb9700620807000205be000004be00aa
:102d50000e07e900e1fc2f008f80400001064700cc
:102d60005fb29700efb297007fb397008fbb9700d9
:102d70000800be000a01be00100b07001d00100075
:102d80003fb19700624e7800889ebe008a96be00d2
:102d9000e00f5400e08f5c00e00f5d00e08f5d000d
:102da000020034000e00e000e0ff3c00cfb19700cd
:102db000e88f510010003a000d1090000038a30079
:102dc0000d003200f70f570006003e00e4fc2f0014
:102dd0000e024200e4c07f0000c3b30080cf500069
:102de000050032000e07e90000c3b300e1fc2f002c
:102df0008e80400080f07f0078011700920e9800ce
:102e00006d009000e3fc2f008f8141008e80410017
:102e100007f707001d0e90005d089000800f560018
:102e200006003d000c005000800e98000d10900030
:102e30000040a100801698000f0037000000e0005d
:102e40000d003d000d10900074006000f00f500068
:102e500009003a007d089000fd009000010050003c
:102e60008d089000010050000c0750004240a9005e
:102e7000010034008e0e98004f0778004f06be0008
:102e80004f05be004f04be006f02b10000000600f7
:102e9000ef04b000889fbe008a9fbe008c9fbe00da
:102ea0008e1f7800c0af9f00a1df9f0060fa2f0047
:102eb0000f004000e0af9f00cfaa97005503be006f
:102ec0004502be0084af9f0095af9f00a6af9f0054
:102ed000b7af9f0010c6b30080cf5000160032007d
:102ee00010c4b30080cf5000130032004fab9700e6
:102ef000560890000000e00003003d006000200044
:102f0000500b98000c0037000000e0000a003a0067
:102f100070c6b300afdb970080cf530003003200d0
:102f200070c4b30080cf530003003a0010002000ab
:102f3000cfa89700d0089800cfa89700e2fc2f00f8
:102f40000280470070fc070080017800e20f50000b
:102f500014003a00cfa99700e30090003000200051
:102f60009009980010c6b3002fda9700804f5200e6
:102f70000a00320064404000804f520007003200d7
:102f80000040e800804f520004003200e21c2200a2
:102f90000040e800804f520017003a00221d220036
:102fa000150037000000e00018003400cfaa970099
:102fb000e500900030002000900a980010c6b30091
:102fc0002fdb9700804f53000a003200644040001e
:102fd000804f5300070032000040e800804f53004c
:102fe00004003200621d22000040e800804f5300c0
:102ff00001003a00a21d2200b258780002007800b9
:10300000b058780090487800f201370014c6b30039
:10301000afdb970084cf53000300320010c4b3002d
:1030200080cf530010003a004fa89700ec004000fa
:103030001101780000c3b300005978008208e8004d
:1030400080c7b300afd8970084cf50000100320092
:1030500080c5b300004978004fa997007200900026
:103060000080e800700198000300e00003003a00cf
:103070008006eb00fda79f00d001370011c6b3000a
:10308000afd9970081cf51000300320010c4b300c4
:1030900080cf5100ad003a00ee1d22002fda9700dc
:1030a000814f520001003200fe1e2200cfaa97007d
:1030b000550890008006e8000000e00001003d0097
:1030c0001d0220000d06e8004fab97003604be003d
:1030d0002605be006022b8006033b8000fa8970034
:1030e0009fa897002fa99700bfa997008604070003
:1030f0000000e00001003d000bf0a20088af9f003f
:1031000099af9f00aaaf9f00bbaf9f007fa0970021
:1031100064005000f0a79f00efab9700805beb00ce
:10312000e7af9f003f003700c201200003002000ee
:1031300001fd2f00018047009ef907000faa9700ac
:103140009faa97002fab9700bfab9700f4af9f00eb
:1031500085b79f0096b79f00a7b79f000400be00e9
:103160000601be00700407000004be000005be009a
:10317000670656004240a9000c00340062030700b5
:103180000002be000203be007fa897008fb0970028
:103190001fb19700afb197008f04070080af9f0069
:1031a00091af9f00a2af9f00b3af9f00efaa97001f
:1031b000e7824200e5af9f0070002000e00f54005e
:1031c000e08f5c000d003400600020006fab9700c2
:1031d0006f636500e6af9f00cc5bdd004455de0009
:1031e0000a857300c4ddde00e00f5500e08f5d004e
:1031f000020034000000e900f4ff3b000000e90099
:1032000005003300efa897008060eb00e1af9f005e
:103210000000e900fbff3b006fa997006701410038
:10322000e2af9f000c00e000090034006022b8000b
:103230006033b8000fa897009fa897002fa99700a8
:10324000bfa997009e0707000000e000b6ff3c0002
:10325000efa9970064fa2f000f024200048051008a
:103260000006e90075fa2f0085824700e5af9f0050
:103270008d0f560001003d008c0678000d00e00027
:103280002b0035008c8f560005003d006fab97007a
:1032900066c07e00f2c0b300e74f500001003c0062
:1032a0000041eb008d00e900efab970067c07800ac
:1032b000824f500006003a008d06e9008100e900c7
:1032c000efa9970063c07800824f5000faff3200e8
:1032d000ef4f510004003a006faa970064c07800d5
:1032e0000040e80000f278000100e00007003d0027
:1032f000efaa97008502e900e5af9f008d06e80080
:103300007fa0970064004000f0a79f008d00e900b7
:10331000070033006fab970066c078000000fb0029
:103320006e40780000f378008100e900f9ff3b006f
:10333000cfab9700570890000000e0001f013d0050
:103340000d00e900d00b98001c0137000fac97006e
:103350009fac97002fad9700bfad97006022b800db
:103360006033b8000800be000a01be00e603070093
:103370000000e00005003d000bf0a20088af9f00b8
:1033800099af9f00aaaf9f00bbaf9f007fa097009f
:10339000725927000280b900026a28001300200039
:1033a00022060700e4005000f1a79f001d003b002b
:1033b00063801000c1ff2f00010460000800ea00d4
:1033c000f0a79f008004eb000800e00047003400f5
:1033d0000808a3000e0032006848b8008267210088
:1033e000020040003002be002003be000fa897007c
:1033f0009fa897002fa99700bfa99700f80307007f
:1034000080af9f0091af9f00a2af9f00b3af9f001e
:103410000884d1008904e8000800e000ecff3c00cb
:10342000320037000100e000300034006022b800b4
:103430000600200007ff2300b4b79f00c5b79f0018
:10344000d6b79f00e7b79f00c0ff2f000080600045
:10345000f0a79f00000478008004eb001600340001
:103460000808a300100032006848b80085672100f2
:10347000050040003002be002003be003fb09700b0
:10348000cfb097005fb19700efb19700d40307006a
:103490000002be000203be00b4b79f00c5b79f0084
:1034a000d6b79f00e7b79f000884d1008904e800e1
:1034b0000800e000eaff3c003fb29700cfb297005f
:1034c0005fb39700efb397000fa897009fa89700ee
:1034d0002fa99700bfa997008e02070080af9f0019
:1034e00091af9f00a2af9f00b3af9f004fab97007b
:1034f000d608900060c6b300afdb970080cf5300c2
:10350000040032006687400060c4b30080cf5300df
:1035100003003a007fa09700008040006a07400047
:10352000f30f5700010034003e01200000c3b30038
:10353000efa8970080587800e1af9f003a0037006d
:103540000800be000a01be00770307000006be00a7
:10355000f0b79f0081bf9f00680757004240a90055
:103560000e003400680207000002be000203be0025
:103570000800be000a01be00970307006022b800e1
:1035800046782d00771924009503070080af9f002f
:1035900091af9f00a2af9f00b3af9f00efa997002c
:1035a000e8814100e3af9f0088002000e00f560053
:1035b000e08f5e001100340078002000a20020009f
:1035c000030020007fb097008fb89700daf407005f
:1035d0006faa970005c3b30005624100e4af9f00e6
:1035e000f0b79f0081bf9f00e00f5000e08f5800b0
:1035f000020034000804e900f0ff3b000804e90081
:103600000600330000c3b300efab9700806378007f
:10361000e7af9f000804e900faff3b006fa897009e
:1036200068004000e0af9f000e00e0000b00340097
:103630000fac97009fac97002fad9700bfad9700e0
:103640006022b8006033b8000800be000a01be0066
:103650009b0607000000e000b9ff3c00efa89700c0
:1036600062fa2f000f014100028050000007e900bc
:1036700073fa2f0083814700e3af9f007fa097007c
:1036800067004000f0a79f0001c3b30093cf100074
:103690000a003a000e07e9007fa097000000e90049
:1036a000f0a79f006faa97000402e800e4af9f0014
:1036b00014427800814f5200f6ff3200cfaa9700e3
:1036c000d508900060c6b3002fdb9700804f5300f1
:1036d0000300320060c4b300804f530004003a007e
:1036e0007fa09700008040008006e8000a003700b5
:1036f0008001eb0050c6b300afdb970080cf5300d2
:103700000300320050c4b30080cf530001003a00e0
:1037100013002000838640008d0f570001003d00fc
:103720008e0678000d00e000240035008e8f5600d4
:1037300006003d006fa89700e0c07e0092c3b30072
:1037400040c3b30080cf500001003c0002c3b3006f
:103750008d00e900efa9970063c07800824f500008
:1037600006003a008d06e9008100e9006faa970083
:1037700064c07800824f5000faff320090c3b3005b
:10378000804f510004003a00efaa970065c078000e
:103790000040e80080f278000100e00007003d00f2
:1037a0006fab97000603e900e6af9f008d06e800c7
:1037b0007fa097000000e800f0a79f007fa297007d
:1037c0008d0178006fa99700afd897004fa8970098
:1037d000060007004f0778004f06be004f05be00e9
:1037e0004f04be00ef04b100000006000a00fa001a
:1037f000889fbe008a9fbe008c9fbe000004780098
:10380000014578008205780083047800040678007a
:103810000300e00002003c00190020008b20220081
:1038200060c6b300804f55000e00320060c4b30084
:10383000804f55000b00320070c6b300804f55001a
:103840000300320070c4b300804f550083003a007b
:10385000e40f46008100350058089000800f5600a4
:103860007e003d000c06e80060c6b300804f5500a6
:103870001000320060c4b300804f55000d003200cc
:10388000081090000038a30004003a005808900087
:10389000808f540001003d00590c9800580890009a
:1038a0000c005000500c980002003b000000eb00a0
:1038b000500c98000c00e00027003c00f20144008e
:1038c000130178006800900001c3b3000170790013
:1038d0000201e80082097800580890000000e0002a
:1038e00003003c00081090000038a30004003200e0
:1038f000e8009000e0c2b300807079008209e8001f
:103900000c00ea00d8089000808f500001003d00b4
:103910000106ea000c00ea00200c98000c80400030
:10392000500c9800890f500001003d008004780081
:10393000680090009808900001004000390c980041
:10394000090178008b00780039f4070058089000ce
:10395000090050001a003700e80090001808900095
:103960008c8f540018003d00008040000901780051
:103970008b0078002ef40700180890000901400021
:10398000120c980009005600200c9800580890006e
:103990000000e00003003c00081090000038a30085
:1039a00006003200e8009000e0c2b30080707900a9
:1039b000380890000000e800300c9800580890008b
:1039c000400c9800a3003700008040000c017800f4
:1039d0008b00780016f40700180890000c004000d7
:1039e000100c98008c845400580890000000e000ef
:1039f00003003c00081090000038a30006003200cd
:103a0000f20144009300780068019000e0c2b30026
:103a100000f178008109e80058089000890f5000f3
:103a200001003d0080047800680090009808900034
:103a3000010040008c80450009017800fcf307007c
:103a40001808900009004000100c980058089000d9
:103a500009005000200c98007e00370070c6b300ab
:103a6000804f55000300320070c4b300804f5500f2
:103a700014003a0058089000808f540004003d0064
:103a8000081090000038a30001003a00590c98007b
:103a9000580890000000e900500c980002003b001c
:103aa0000000eb00500c980051c6b30070c6b30084
:103ab000804f55000100320051c4b3000145780029
:103ac0000900370010c6b300804f550002003a00cd
:103ad0000ac7b3000400370010c4b300804f55007c
:103ae00001003a000ac5b300f20144001301780056
:103af000680090003b7079000201e80082097800bc
:103b0000580890000000e00003003c0008109000fe
:103b10000038a30004003200e8009000e0c2b300c7
:103b2000807079008209e800580890000000e000e9
:103b3000100034008904e900890f500001003d00a5
:103b40008004780068009000980890000100400010
:103b5000090178008b007800b5f307001808900081
:103b600009004000100c980058089000090050000f
:103b7000200c9800e8009000180890008085400014
:103b80008a5d78008b06e8000c00e0000400350038
:103b9000b0c2b300804d78008d0578000400370076
:103ba000d0c2b300804d78008d0578000c06ea0085
:103bb0008004eb000c00e00009003400a1002000ac
:103bc0000c00780071f407007681540001f17f0049
:103bd000000678008904e8000000e000f7ff3c00e0
:103be000e18f540009003c0050c6b300804f5500df
:103bf0000300320050c4b300804f550003003a0068
:103c000000c3b300805e78008d0578000900e000f5
:103c100002003a0000c3b300805d78000900e000b4
:103c2000070034008904e900f680540061c07f0079
:103c300002c3b300825d40000900e000f9ff3c00d0
:103c40006800900098089000010040000080550036
:103c5000300c98000810900074006000f00f5000c5
:103c60000e003a0078009000980890000100400093
:103c7000a808900001004000b80890000100400032
:103c8000c80890008100400078089000808f5000a4
:103c900002003d0001005000000c98004f06be00dd
:103ca0004f05be004f04be000080fa000000060071
:103cb000f4ff2f007d023700810378009602070091
:103cc0000001be006000b8000478a30013003a00b1
:103cd0006220e10015003e000d0039008301d10093
:103ce0000281d3008180d3008301d1000281d300ff
:103cf0008180d3008301d1000281d3008180d30071
:103d00000538b000c42add00f300b20083817200e0
:103d100007f0a70003f0a00000000600f3ff270053
:103d2000f2ff2f006110b900fbff370003ff2700ef
:103d3000f7ff3700889fbe008a9fbe00010578000c
:103d40000100e0000400350008003c000000e00035
:103d5000200032000500370060001000e0801800ed
:103d600002003b0001f02c001a0037000004be00e6
:103d70006011b8006b0920000982cf0002003900f1
:103d80000882cf000441b000694252000e003200a8
:103d900008003b0082817100610164008904d10048
:103da0000884d3008b05e8000442e800f9ff3a00dc
:103db000050037000804440089844c008b05e900a5
:103dc0000442e900fbff3a00680207000af0a7007e
:103dd00001f0a0004f05be004f04be000000060029
:103de0001400fa00889fbe008a9fbe008c9fbe0010
:103df0000005be000206be00680047000c90be0031
:103e00000a90be007f0207006400e1001a00320041
:103e100016003e006100e1001a0032006e049000be
:103e2000fe0490000e0b90009e0b90006011b800f5
:103e30009e0590000b38b100d501200082817100f1
:103e4000610164008703d1000683d3008984d30015
:103e50000884d3008502e900f8ff3a004302070016
:103e60000df0a70001f0a000a1023700f1ff27002c
:103e7000f0ff2f009e02370001f82700000020000d
:103e8000f7ff37006000b800f5ff3700889fbe00dd
:103e90008a9fbe008c1f78009a0207001002200043
:103ea00002003b0060be88009e0237008a0062006c
:103eb0006408e10002003a0060be8800a6023700f4
:103ec0006108e100fcff32000800be000304780036
:103ed000db05070001f0a100ba09070008f0a60001
:103ee000040037000001be0091042400b0fd200052
:103ef000e504070009f0a70001f0a20092023700d4
:103f000014002000e90137004f89de0082017800ab
:103f1000940237002800fa00889fbe008a9fbe00e6
:103f20008c9fbe0003866b005d0207006400e10009
:103f3000440032006408e1004a0032006100e10000
:103f4000460032006108e10049003200ec064700fb
:103f50006000b8003d02be003d03be00f48657007d
:103f60006011b8003d04be003d05be007d03200089
:103f70000b0037000000a0008d06e900130032009e
:103f80000402420085824a0006034b0087834b00ef
:103f900000004000818048000201490083814900ff
:103fa0000802520089825a000a035b008b835b007f
:103fb000f0ff3b000802420089824a000a034b00de
:103fc0008b834b008d06e900edff3a00848272007e
:103fd00086827200f707b200878272000100320009
:103fe000150020001e0490003e0b900006035400b4
:103ff000e63fb0000368a300070032000000a700fe
:104000000500a0008301d1000281d3008180d3008c
:104010000080d3000603e8008301d1000281d300b1
:104020008180d3000080d3000002eb000482d20024
:104030008302070003f0a1000cf0a70003f0a0002a
:104040002b023700640247006408e10025023200b9
:104050003400be003401be00f6ff37006108e10005
:10406000200232006011b8006000b800f1ff370094
:1040700003ff270002002000fbff37001400fa00b6
:10408000889fbe008a9fbe008c9fbe000004be00b9
:104090000205be00680047000a90be000890be00fe
:1040a000d80107000070a7000bf0a1000bf8a300d7
:1040b00016003a009e029000304320008082520099
:1040c000b0fe2f000028e1000d003c00b0fc2f00e6
:1040d0000028e1000d0034001e0990008e089000b9
:1040e0007e0090000501b0000201d1008180d30064
:1040f0000080d3008502e800fbff3a00fc01370096
:104100000100280000002000f90137006000b8001d
:10411000f70137002800fa00889fbe008a9fbe0082
:104120008c9fbe0007067800878669000c003b0064
:10413000030478008704780008f0a10009f0a100ca
:10414000840f5000858f5800860f5900890f5c003e
:10415000030033000cf0a20001003a000cf0a100b3
:10416000cf0107006400e1005f00320078014700e2
:104170006408e100610032006c014700748557005b
:104180003200be001201be003a04be001a05be0095
:104190001e039000be0a90008503530006003d00f8
:1041a0000004fd008104fd000205fd008305fd0003
:1041b0008703ea00050378000df8a300040032002d
:1041c00060041400e0841c0060051d00e0851d00f3
:1041d0006022b8007d0320000d38e1008006eb006e
:1041e0000b0039004433dd00f300b200830173009b
:1041f00039003700848272000d027800e106640005
:104200008b85d1000a85d3008984d3000884d3002c
:104210008703e900f7ff3b00080040008980480061
:104220000a0149008b81490004003b006000100036
:10423000e080180060011900e08119000358a30014
:10424000090032008d827200848272006102600077
:104250008301d1000281d3008180d3000080d3008c
:104260000603e8001b0037000348a30017003a00cc
:104270000600e000170034000603e9000d00a3006b
:104280000000480081804800020149008381490004
:104290000348a3000f003a000600e00009003400c4
:1042a0000603e90000004000818048000201490047
:1042b0008381490001003a000003eb000348a3009a
:1042c000f5ff32006022b8000200370084827200dd
:1042d00061826600da01070003f0a1000cf0a7007c
:1042e00003f0a00082013700640147006408e10088
:1042f00002003a000df8a3007a013a003200be0035
:104300001201be007a0137008f1fd100f8010700ab
:104310008f87e9000000e000000006006d03070041
:104320000400be00000006001400fa00889fbe00d2
:104330008a9fbe008c9fbe000004be000205be0026
:10434000680047000a90be000890be002d010700db
:104350000070a7000bf0a100304320009e029000e7
:1043600080825200b0fe2f000028e10011003d00c5
:10437000b0fc2f000028e100150034001e09900059
:104380008e0890007e0090000501b0000201d1006f
:104390008180d3000080d3008502e800fbff3a0053
:1043a0000b00e00052013b0060001000e0801800ac
:1043b0004f013700f0ff2f00f1ff27000b00e00056
:1043c0004b013b000100280000002000480137009d
:1043d0006000b8004601370007f0a2004dff37002b
:1043e0002800fa00889fbe008a9fbe008c9fbe00f6
:1043f00003866b002a0107000028a30064003a002e
:104400000128a30067003a000008a30062003a00f8
:104410000108a30065003a001e009000be0890004d
:1044200081064000ed3fb100f4805700ee0190009e
:10443000111ab8008e099000311bb8009e09900037
:10444000311cb800511db800f48557004600070024
:10445000fe0190003a0007008b85e8003e0007004f
:104460008e09900040000700ee0190003400070024
:104470008b85e800380007008e0990004000070097
:104480009e0990001b18b800890440000a85480066
:10449000fe019000340007008b85e800380007001b
:1044a000ee019000300007008e0990001b18b80044
:1044b000890440000a8548000a98a30008003a00d1
:1044c0000402420085824a0006034b0087834b00aa
:1044d00008044c0089844c000a054d008d06e90053
:1044e00084827200850273004c3add0085027200fe
:1044f0000100320015002000443ade001400b20032
:104500004538de00cb45dd000b007000c540de0005
:10451000cb4ddd008b8070004549de00cb55dd00c2
:104520000b017100c551de000d0378004401070046
:1045300003f0a1000cf0a70003f0a000ec0037008e
:104540001b18b8008502400006834800e0834b003a
:1045500060044c00070037001b18b8000603400039
:1045600087834800faff37001b18b8008703400014
:1045700008844800e0844c0060054d0000000600ff
:104580001b18b8000804400089844800faff37006f
:104590000108a300d3003a005800be005801be0035
:1045a000e3ff37000008a300ce003a0009047800ba
:1045b000f9ff37000001be00570007000470a70094
:1045c00003f0a1006509b100160032000d003500ae
:1045d0006828e10006003500f0ff2f00f1ff2700fa
:1045e0000300e00013003b0001002800000005006c
:1045f00000004000818048008502e900fcff3a008d
:1046000008003700f88f420002003c008000eb00f9
:10461000000005008100d1000080d3008502e80081
:10462000fcff3a000300e00002003b0060001000c5
:10463000e0801800000006000001be003600070000
:104640000470a70003f0a10003f8a30013003a00d0
:104650006509b10010003200090035006928e10049
:1046600002003500010028000000050000004000a5
:10467000818048008502e900fcff3a000000060046
:10468000f88f4200050035008100d1000080d30082
:104690008502e800fcff3a00000006008000eb0005
:1046a000000005000400200000003700889fbe00c5
:1046b0008a9fbe00841f7800920007004f00780098
:1046c00011003300f0ff2f00838f6c0006003b00c9
:1046d000040565000a00a7000800370009f0a600dd
:1046e0001000200008003700820f5400838f5c0008
:1046f000030039001000200001003e0000002000ef
:1047000009f0a7000000ea004f05be004f04be00fc
:104710000000e00000000600c70ade00f107b2005a
:10472000f50fb20008003200e1cf42000200320073
:104730000170a00024000500810f7000010032000c
:104740000408050044000500810f700002003a00d3
:10475000140005008502e9000000400081c0480007
:10476000fcff3b000170a000240005008100200038
:10477000618055000b003d000b00200061fe2f0002
:104780000100e1001d0034008281710061016400bc
:104790008904d1000884d3000000e800faff3a0041
:1047a00071002000610064000300700002006000de
:1047b0000900320061044400e0844c000988a5002f
:1047c000050032008b05e8006808e10002003a00ad
:1047d0008904d1000884d300f20f20000258e100c0
:1047e00005003d00c75ddd00f907b2008980750056
:1047f00008007800000006000bf827008b00780006
:1048000000000500800078005002be005003be008a
:104810004439de00f700b200f37f2000030161009d
:10482000090032000218e10016003a00850172000a
:1048300083017300838173000008200015003a0093
:1048400040002000130037008501720083017300cf
:104850008381730005003a0004a8be0006a8be00cc
:10486000100020000b0037000201e90004024200a2
:1048700085824a0006034b0087834b000748a3004c
:10488000f9ff32000740a00004a8be0006a8be0041
:104890002000200080009800920098000000060090
:1048a000680447000294be000094be00fc04470068
:1048b0008694be008494be0009007800d1ff0700f2
:1048c00008007800cfff070099007800814f700042
:1048d0000b003b000800be00ae0007004f00b10017
:1048e00003003700f3ff2700f2ff2f006110b9002b
:1048f0004f06be004f05be004f04be000080fa0008
:10490000000006000004be0083ff07000003be0095
:104910000405be000200be007fff0700844f750043
:10492000000006000200be006450e10005003600f1
:104930006420e100020036000968a30001003a008b
:104940000800be000160a0004f0678004f05be00c1
:104950004f04be0000000600f0ff2f00f1ff27000b
:10496000f9ff3700889fbe00830478000300e00051
:104970002c00350003003c0000827000040271002e
:104980002600320036432000c50020008383cf007c
:104990000a0039000541b1008283cf0007003900c9
:1049a0000541b1008183cf00040039000541b10009
:1049b0008083cf00010039000541b10085c3530059
:1049c0006022b800120032000a003b0084827200ac
:1049d000610260008301d1000281d3008180d30095
:1049e0000080d3000603e8008743e800f7ff3a00a1
:1049f00007003700000040008180480002014900a4
:104a0000838149000603e9008743e900f9ff3a0082
:104a10000b00070009f0a70003f0a0004f04be0040
:104a20000000060060001000e0801800600119001e
:104a3000e0811900d3ff3b00033e2c00f7ff370055
:104a40001800200057002000080453000d003d000e
:104a50000600200097fc2f000740e1001e003400f4
:104a600084827200610260008301d1000281d30060
:104a70008180d3000080d3000804e800f8ff3a00ea
:104a80004700200061046000050474000404640011
:104a90000d00320061004000e080480060014900e4
:104aa000e081490003b8a500070032000603e800d2
:104ab0006538e10004003a008301d1000281d3008f
:104ac0008180d3000080d300f87f20000830e1000f
:104ad00003003500080378006000b8006011b800da
:104ae0004433dd00f300b2008301730000000600d0
:104af000889fbe008a9fbe008c9fbe000404be003b
:104b00000605be00809fbe00829fbe002f000700ea
:104b1000040678000800be000a01be002b00070052
:104b2000840678004f03be004f02be008d4f760012
:104b30007fb0970013003300f0ff2f008b8f6b00c6
:104b400006003b000d0666000c00a7000a003700b7
:104b500007f0a600100020000a003700880f52005e
:104b6000898f5a008a0f5b008b8f5b00030039002e
:104b70001000200001003e000000200007f0a70008
:104b80000000ea004f06be004f05be004f04be0005
:104b900000000600e48240001078a3000700320005
:104ba000640240001178a3003400be001401be006e
:104bb000040032000330a700000006003500be00ec
:104bc0001501be000330a0000000060005ff27000d
:104bd00005826100070032000428e1000100320074
:104be000240005000600070001003a00440005000b
:104bf0000408050002000700f9ff3a001400050050
:104c00006f8261008102700085027100850272006e
:104c100000000600020ab900001bb9000200b8003b
:104c2000810042008100430000000600839f68006d
:104c30000100e00002003d0060001000e08018006c
:104c40000300e00002003d0060011100e081190056
:104c5000200107004f00e00002003b006000100050
:104c6000e08018000000060060001000e0801800de
:104c700060011900e081190000000600881f78001b
:104c8000000478005001be004000be000000420059
:104c900081804a0002014b0083814b00009cbe00d2
:104ca0000294be00dc0007000300310048009000c1
:104cb0000000e800400498004f047800000006005f
:104cc000889fbe00000478008004eb005001be0005
:104cd0004000be00d0000700010031001900200094
:104ce0000400500085805800060159008781590052
:104cf000009cbe000294be004800900009005000d5
:104d0000400498004f04be00000006001200fa00a4
:104d1000889fbe008a9fbe008c1f78000205be00df
:104d20000004be00f4b79f0085bf9f0096bf9f00a0
:104d3000a7bf9f000000eb00e0b79f00d0b79f0027
:104d4000c0b79f00b0b79f00a0b79f000006eb0060
:104d50005fb197006fb097008000d0000000e000c6
:104d600015003d00e1b79f00010078000200e0005f
:104d700001003d000000a000ac00070001003d0064
:104d80000000a000af00070001003d000000a000ef
:104d9000b200070001003d000000a00081000700f4
:104da00001003d000000a000b20007007c80570019
:104db000b2ff070014003700e1b79f000100780040
:104dc0000200e00001003d000000a0009700070085
:104dd00001003d000000a0009a00070001003d0016
:104de0000000a0009d00070001003d000000a000a1
:104df0006c00070001003d000000a0009d000700be
:104e00007c805700aeff07006fb097000000e00005
:104e10000700350010002000010020006011b800dc
:104e200008047000898470000a0571008b85710088
:104e30000c06e800f0032000800f5600c4ff340089
:104e40006fb097000000e00006003d007fb29700c1
:104e50008fba97001fbb9700afbb97007c805700ad
:104e600086ff07000802be000a03be006fa8970075
:104e70000000e00004003a002fb29700bfb2970094
:104e80004fb39700dfb397000400be000601be00d9
:104e90004f0678004f05be004f04be000080fa00a8
:104ea00000000600881f780018002000881f780086
:104eb00096ff07008f87e9004f0478000000060086
:104ec000801feb0091ff07008f87e90000000600bc
:104ed0000800fa00889fbe008a9fbe008c1f7800e1
:104ee0006e00070005003d0043000700300007008a
:104ef0000c003d00330007000b003700e00f5200ac
:104f0000e08f5a00e00f5b00e08f5b0006003d0081
:104f10000400be000601be0053ff07000205be00ec
:104f20000004be001c0020002c000700ddff07006d
:104f30000c00e000010032004bff07004f06780034
:104f40004f05be004f04be000080fa0000000600be
:104f50000800fa00889fbe008a9fbe008c1f780060
:104f60004e00070002003d001c0020002200070048
:104f70000f00070001003d001200070017000700a6
:104f8000cfff07000c00e0000100320036ff0700f1
:104f90004f0678004f05be004f04be000080fa00a7
:104fa0000000060090b79f000100d00080b79f006e
:104fb000e00f5400e08f5c00e00f5d00e08f5d00cb
:104fc000000006000800be000a01be0026ff070020
:104fd0000205be000004be00000006000802be007c
:104fe0000a03be005fb09700efb097007fb1970053
:104ff0008fb99700000006001bff070001000700a3
:1050000000000600b0b79f00c1b79f00d2b79f0055
:10501000e3b79f00000006000400e1000588e100fe
:105020000690e1000798e10000000600c0b79f006d
:105030000200d000b0b79f00afb097000100e000c1
:1050400000000600b0b79f000100d000a0b79f008d
:105050009fb097000100e00000000600a0b79f008d
:105060000100d00090b79f008fb097000100e000d2
:105070000000060080b79f000804d0008984d20099
:105080000a85d2008b85d2005fb29700efb29700fd
:105090007fb397008fbb970000000600d9ff070081
:1050a0000605be000404be000006eb00e00f500041
:1050b000e08f5800e00f5900e08f59000000060013
:1050c000809feb008afe07008f87e9000000e00068
:1050d000000006000202500083825800610039007f
:1050e00003037100620032000503720059003200b0
:1050f0000300e0005500330017003a000100e00013
:105100004b0032000208e1000600310011000900e6
:105110004288d800010178008001eb008000eb009c
:10512000000006006110e100550032000002be00e0
:10513000110009008280d800800278000400780005
:10514000110009004288d800010178008001eb00bd
:105150008500780000000600889fbe008a9fbe0080
:105160008c9fbe000386cf000c06e9008c1f7800e0
:105170008c19dd00f00216000512de00848171003a
:105180000c11dd000003be008004eb00053cde00d6
:105190008c3bdd000532de00848373000c33dd00c0
:1051a0000700780088007800110009004388d800c3
:1051b0000202b8000306b8008c82420060854e00ef
:1051c0008005eb000402530085825b000a055c0049
:1051d0008b855c000b0033008000eb004f067800ed
:1051e0000c21de00700516000a2ddd000a01710099
:1051f0008c29de004f06be004f05be004f04be00e6
:10520000000006000202420083824a0060054d0051
:10521000e0854d000000e9000b00e000eeff3d00de
:105220000202420083824a000000e900eaff3700e0
:105230000000e00012003200110009000280d800d6
:10524000010178008000eb00000006000401be00b0
:10525000010037006011b800100020008000eb0052
:10526000000006000001be006000b800000006005b
:105270000001be00f0ff2f00f1ff2f00000006002c
:105280006011b8000000060007f8270007836100de
:105290000638e10004003a00f70720008783610028
:1052a0008703710001003a0003f0a200889fbe004e
:1052b0008a9fbe008c9fbe00470ade000480a100ca
:1052c000c71ade000580a1000700280007856000de
:1052d00087856100f70f20000720e1009e00320063
:1052e0000728e1009c003200010678000400e0007d
:1052f000b4003200f7072000878060000170a00032
:105300000500e000c0003200f7072000878161003f
:105310000370a000050652000f003a000b50e10098
:105320000b0032000308e10002003a000200e10035
:105330007e003200020450008384580004003100d3
:105340000001fd008101fd008402fd008a05fd00d1
:105350006044b800210037000520e10005003d0051
:105360000001fd008101fd008402fd008a05fd00b1
:10537000050652007a60e100050035000170a100c9
:105380004722dd00848070008a807000630037004f
:105390006044b800ef02660007ff2f0007066600b2
:1053a0000500e00006003400f08312008714dd00e1
:1053b0000511de00071bdd00060171008519de0006
:1053c0007060e1000500350009047800820478006f
:1053d000030178008001eb00700656000b50e100dd
:1053e00003003a00020040008380480004003700b8
:1053f00060041400e0841c00020058008380580000
:105400000188a300060032008100d1000080d30093
:105410008984d3000884d3000402e8002700370001
:105420000178a30025003a000100e00003003200eb
:105430008186cf00698656000a0037008c00200064
:105440000000e00004003a000900780088047800b9
:105450000004eb00700252008086cf000d0646006b
:105460000c06e9007060e10006003500800078005d
:1054700009007800880478000004eb0070065600ec
:10548000700252000c00e0000c0034008c08dd00bb
:10549000f00316000703de00868070000c00dd00bc
:1054a000074bde00060070008c4cdd000743de0079
:1054b000868474000c44dd000c0252006120e1007f
:1054c000200035006101600007002800878164002a
:1054d000f7ff270087836400070374000300e000e0
:1054e0000600320082037300040032000000e8006e
:1054f000e08048000188a3000e003a00f70f20006a
:105500000720e1004a003d000170a1004722dd00b4
:10551000810072008a8070000000be004f06be004d
:105520004f05be004f04be00000006006000b8003a
:10553000faff37008100d1000080d3000402e800a8
:10554000eeff370004017800890174001c02070097
:105550008a807000f1ff3700ff0107000702780022
:105560000001fd008101fd00fb01070087027800ba
:10557000850372000778a300040032000001fd00db
:105580008101fd0038020700e4ff37008503620057
:105590000768a300080032000b50e100030032004e
:1055a000f0ff2f00f1ff2700dcff37000001fd00b6
:1055b0008101fd00d9ff37000468a300d7ff320046
:1055c000faff3700f8ff2700888360000b003a00dd
:1055d0000000e00009003a00830364008283730046
:1055e000020032000200be00ccff37000b50e10089
:1055f000ceff3a000200be00c8ff370014002000b2
:10560000810064003eff3700f8ff270088836100b7
:1056100004003a000200e00002003a008c0078002a
:10562000beff3700150020008301640039ff3700fa
:1056300001f827000000200081007500b7ff370047
:10564000889fbe008a9fbe008c9fbe001b0020006a
:105650000202be00058668000600280006066600f5
:105660004709de00f20fb200820032000243e80078
:1056700080003200c729de00f30fb2007d00320047
:105680000343e8007b003200f107b2000170a00084
:10569000f507b2000570a000c708dd004903de0071
:1056a000868070004700dd00c72add004923de0048
:1056b000868272004722dd0003055100040350007a
:1056c00085835800030031000000400081804800bd
:1056d0000a05e9008c1f78008a9fbe000400500074
:1056e000858058000402420085824a000000400084
:1056f000818048000005eb000004be006033b80064
:105700000406be000d48e1005600310011000900fa
:105710004dccd8000c01b8000d02b80084814100c6
:1057200060824a008283530003045c0084845c002e
:1057300060055d000a00e00025003a008005780061
:105740000d40e10049003100880078000700780032
:10575000110009004d88d8000c01b8000d02b800f6
:105760008481410060824a006003110083835b00f2
:1057700004045c00e0845c000900e00021003a00c1
:105780004f01be000300e0002b003200e301600087
:10579000070673008c817100010032006400700004
:1057a0004200de004e5edd000c007000c258de00dc
:1057b00001e0a00082020700cf0178008180710023
:1057c0004f06be004f05be004f04be00000006009d
:1057d0008c8343000d044c00e0844c0060054d00b8
:1057e0000000e9000a00e000d4ff32008c8343008f
:1057f0000d044c00e0844c0060054d000000e90001
:10580000ceff37000c0343008d834b0060044c0037
:10581000e0844c000000e9000900e000d8ff3200fd
:105820000c0343008d834b0060044c00e0844c006b
:105830000000e900d2ff37004200de004e5edd00ce
:105840000c007000c258de0001e0a000cf0178001b
:105850000300e000daff320060001000e080180072
:10586000d7ff3700f0ff2f00aaff3700f0ff2f000f
:10587000b9ff37000404be0037010700870678002f
:105880000004fd008104fd0033010700078366006a
:105890000678a300030032000960a7000800be00dc
:1058a0002c0037000d78a300020032000800be0073
:1058b000280037000778a30026003a0001f0a10075
:1058c00009f0a1000668a30003003200f1ff2700e1
:1058d000f0ff2f00baff37000d68a300030032006d
:1058e0000800be008c807000b5ff37000768a30079
:1058f00007003a000648a30003003200f1ff27002a
:10590000f0ff2f00aeff37000d48a3000300320068
:105910006000b8008c807000a9ff37000748a30022
:105920000400320001f82700000020008c80700085
:10593000a3ff3700ef0107000004fd008104fd0014
:1059400002057800eb0107000802be008a0178001a
:1059500059ff37000160a0001202200062be8800db
:1059600097ff37000100e000120032000500e00060
:1059700010003200889fbe008a9fbe008c9fbe0030
:105980000006eb0001f8a3000300320060001000e5
:10599000e08018000cf0a00005f8a300030032001e
:1059a00060021200e0821a000cf0a2008005eb00f9
:1059b00041ff37006000b80002000500889fbe006c
:1059c0008a9fbe008c9fbe000004be000205be0080
:1059d0000400b8000546b8008c80400060814e008d
:1059e0008001eb00044eb8008c8040000d0149009e
:1059f000e08149000646b8000c0141008d81490054
:105a0000054eb8000c0141008d8149000456b800d4
:105a10000c0141008d8149000746b8008c8141008e
:105a2000064eb8008c8141000556b8008c814100bb
:105a3000045eb8008c8141004f06be004f05be00d9
:105a40004f04be0000000600038368000700280022
:105a500007036300470ade000480a100c71ade00c6
:105a60000580a100f70f20000720e100420032006e
:105a70000728e10040003200889fbe008a9fbe00d8
:105a80008c1f7800f107b200f307b2000400e000b9
:105a9000640032000170a0000500e00068003200e0
:105aa0000370a00085054200eb07b1000204b800b6
:105ab0000302b8008484440060854a00020ab800ea
:105ac000848444000a854a00030ab800040545009e
:105ad000040033000804d0008984d2000a85d20073
:105ae0008b05e9006158e1003d00350002102000ff
:105af000090161000308200089816100f707200087
:105b00008783640008867300c84cde00c853dd003c
:105b1000878474004855de000300e0000600320070
:105b200082037600040032008904e80060054d001d
:105b30000a88a3000c003a00f70f20000758e10084
:105b400044003d000a70a100c75ddd000a857500b4
:105b50008a007300090078004f0678004f05be00e8
:105b60004f04be00000006000a05d1008984d3005e
:105b70008b05e800f0ff3700881f780006047800e6
:105b800075000700070278000001fd008101fd009b
:105b90007100070087027800850372000778a30070
:105ba000050032000001fd008101fd00ae0007008c
:105bb0004f04780000000600850372000748a30028
:105bc00003003200f0ff2f00f1ff2700f8ff37003d
:105bd0000000200001f8270088807000f4ff3700e3
:105be000880178004848dd00808171004848de0067
:105bf000c850dd0001007000c850de0006047800c7
:105c00000b0178006e00070088807000d2ff37001b
:105c10000500e00005003200170020000601070023
:105c20009dff370081037000f9ff3a00860078007d
:105c30004f0678004f05be004f04be00000005006f
:105c400083037100f9ff320027002000fa000700eb
:105c500094ff370001f8270086807000f4ff3700ba
:105c600001f8a3001d003a004709de00f40f2000f0
:105c70000410e100260032000200e0002c00320097
:105c8000f107b200c708dd004902de008480700021
:105c90004700dd0001e0a000f207b1007b00070033
:105ca000f207b00004042000840160004700de0019
:105cb000490add0004007000c708de000300e000b0
:105cc0000200320061004000e0804800f107b200ad
:105cd0004711dd008280700000000600f4ff2700fd
:105ce000048260008002720001003a000000060099
:105cf00006f827000620e10012003500810263004b
:105d000006826a00040270000e00320006003700ae
:105d100004f827000482680003003a000400200011
:105d200000026a000b0032000160a00000000600c3
:105d30000082700001003a0000000600ed0007003c
:105d4000d6ff37001202200062be8800f0ff2f004d
:105d5000f1ff2700000006002700200001f0a70047
:105d600017002000470bde00f60fb20004003200df
:105d70000643e8000a0032004702b30000000600b4
:105d800001037800f607b2000603700002003a0033
:105d90000703b300000006008702b30000000600fe
:105da00001037800f607b20006037000020032001b
:105db0000770a000000006000760a00000000600b9
:105dc0000100e00026003200610111007810e100be
:105dd00023003c006022b8007010e1000400350090
:105de00080027800010078008000eb007001510013
:105df0000200e0000900340070031100062add00f3
:105e0000822ade008603dd00878272000200de0047
:105e1000860bdd00070070008208de0084817100bf
:105e2000f4ff2700048262008481710004002800ce
:105e3000848262006102600005f0a6000000060096
:105e400004827100070032000000e800e080480092
:105e5000000006000002be006000b800efff37003f
:105e60006000b800000006000478a30004003200bf
:105e70000578a300030032000168a30001003a0086
:105e80000200be000160a000000006008103700057
:105e900068003200889fbe008a9fbe008c9fbe00b3
:105ea0003400f80028002000a80188000208a300a0
:105eb000030032000000d0008180d2000201e9001e
:105ec00081017800800278000002eb00821f7800d8
:105ed0004a1cde000801b10049de280069417c004f
:105ee0000281fb000214b8004644dd000340e100db
:105ef000010036000201e9004111dd001200b3008b
:105f00000214b8004444dd000340e1000100360003
:105f10000201e9004111dd001200b3000214b800d3
:105f20004244dd000340e100010036000201e900c7
:105f30004111dd001200b3000214b8000340e1007b
:105f4000010036000201e9000214b8000886510081
:105f50004763dd00492cde000803730082047800eb
:105f60004834de000940e1002e0031001100090034
:105f70000983d8004811dd00000171000214b80047
:105f80000006eb00840678000885520089855900d8
:105f9000040031000201e9000214b8000885520033
:105fa00089855900820478000b04d1008a83d300cc
:105fb0000d83d3000938e1001c00310011000900f5
:105fc00049bbd8008002eb000003b8000204b8000f
:105fd0000804440089844c00e0824a00870344009e
:105fe00060824c00e0814a000603560087835e0011
:105ff00004025d0083815d00010031000000e900c2
:106000008200d1000080d3004f0178004191de0072
:106010003400f9004f06be004f05be004f04be001d
:1060200000000600f00f2000d2ff3700f0ff2f0025
:10603000e4ff370002000500889fbe000004eb006b
:106040006138e10016003a000100e00008003a0063
:10605000c800de004800dd00880020000100e000ec
:1060600003003a00c800de004800dd006804440078
:106070008184cf00e9845400060034008908dd00e3
:10608000f08314008703de00878070000900dd00c4
:1060900009044400610214004f04be000000060021
:1060a0000300e00008003a00c811de004811dd00de
:1060b000880020000300e00003003a00c811de0061
:1060c0004811dd00680444008384cf00e984540053
:1060d000060034008919dd00f08314008713de0008
:1060e000878171000911dd0009044400e1021400f8
:1060f000e9ff37004f0ade004709de00f107b20072
:10610000f20fb2000b003200f207b1000170a000e4
:10611000c708dd00c901de00838070004700dd0094
:106120000400a6000000060060001000e0801800d7
:1061300000000600810f700001003a000000060018
:106140008182cf000500e00010003e008082cf0079
:10615000ee8242007028e1000400390007003e0092
:10616000800078000000eb000e0037007083120002
:106170008600de000500dd000a0037007083520053
:106180008600dd000000eb0006003700e2825200ce
:106190008508dd00708312000603de008680700033
:1061a0000500dd007507b0000501ea000400a60047
:1061b0000000060060001000e080180000000600eb
:1061c00081017000270032008002eb0001f8a3007b
:1061d0000300320060001000e0801800150020006d
:1061e000f40720000202420020003400f7032000e0
:1061f00087036000060420000003630002082000fb
:10620000000161004700de00c909dd000080710067
:10621000c708de000600e0000800320087037100b6
:10622000060032001000b0000180b0000188a30019
:1062300002003200c108de000402e800f107b200eb
:10624000f30f20000320e10003003d004722dd00a2
:10625000810072002900370001f827000000eb00e0
:10626000260037006000b800000006006802120037
:106270007f20e100020034006000b8001f003700fa
:106280006011b8007020e100040035008001780042
:10629000010078008000eb00700252000400e00072
:1062a00009003400f00312000719dd008419de0034
:1062b0000703dd00868171000400de00070bdd00ae
:1062c000060070008408de00f7ff27008383630068
:1062d00087037100060028000303630007003200f3
:1062e0000700e00003003a006101600002817300d2
:1062f000020032001000b0000180b0000500a600ce
:106300000000060001f0a00000000600889fbe000b
:106310003400f80023002000a301880003002800b7
:106320008384600001f0a100b2fd200093f42300fb
:1063300002015000838158000c003100020020004f
:1063400003982300020150008381580003003900a4
:1063500068ff07003900070099ff0700898068007f
:106360003400f9004f04be00000006008a9fbe0002
:106370008c9fbe0002002000039824000001510001
:10638000818159001e0039005aff070030020700c2
:106390000005eb000100e00003003d00600010007c
:1063a000e08018000a002800630362006333b8002d
:1063b000066001002100070000000000080037000f
:1063c0006d0007000005eb00050037001b0007000b
:1063d0000af0a20002003700670007000a00280048
:1063e00077ff0700898068008a8068004f06be003a
:1063f0004f05be003400f9004f04be000000060047
:1064000055fe07000778a300050032000160a000d8
:10641000898070001202200062be8800f3ff3700fe
:106420000768a30003003200f0ff2f00f1ff2700f0
:10643000f8ff37006000b800f6ff37000100e00009
:10644000120032006f03410010003500809fbe0033
:10645000821f78000002be008201780080010700e0
:106460006403410003003d004300200084e1280054
:10647000020037005300200044e12800e601070035
:10648000cf0178004f02be00750107000000060032
:10649000889fbe003400f80023002000a30188007c
:1064a000030028008384600001f0a100b2fd2000f9
:1064b00093f4230002015000838158001000310042
:1064c000020020000398230002015000838158003d
:1064d0000600390007ff07002700070038ff070004
:1064e0003400f9004f04be000000060001f823004c
:1064f000000020003400f9004f04be000000060038
:106500008a9fbe008c9fbe000200200003982400da
:106510000001510081815900b9ff3900f5fe0700e3
:10652000cb0107000005eb000100e00003003d0087
:1065300060001000e08018000a0028006303620079
:106540006333b8008004eb00066001000a00070016
:106550000005eb00a2ff3700b8ff07000af0a20019
:106560009fff3700040007000a0028009cff370047
:10657000b2ff07009aff37000100e0000e00320072
:106580006f0341000c0035000002be00820178005c
:10659000330107006403410003003d004300200075
:1065a000c4e22800020037005300200084e22800e3
:1065b00099010700000006000000200001002400ef
:1065c00002000500889fbe008a9fbe008c9fbe000f
:1065d0003400f80026002000a601880006002800ec
:1065e0008686600001f0a1000600200007e023007d
:1065f0000603500087835800120031000600200077
:106600000798230006035000878358005c00390078
:10661000b8fe07000005be00820478000002be003c
:10662000820178000e0107004300200084d3280077
:10663000360107000a02be00890178000801070040
:106640004e0037000600200007102400060350000b
:1066500087835800380031000600200007fd230022
:1066600006035000878358000b003100a1fe07008d
:106670000005be008204780062014100e4010700c9
:1066800000067800b801070062015100809fbe003b
:10669000821f78000800370096fe07000005be0044
:1066a00082047800da01070065064000ae010700a9
:1066b000809fbe00821f78000a02be008901780018
:1066c00007002400060020000800200051000700f9
:1066d0000005fd008105fd008204fd00cf0178006a
:1066e0004f02be00230207000a02be0089017800a3
:1066f0009cfc07000104780008f8a30002003200a7
:1067000060001000e08018002d00070008f8a300ca
:106710000200320060001000e080180086d42800db
:106720006665b800060345003602be009601780093
:1067300012020700110037000600200007c82400dd
:1067400006035000878358001300310069fe0700dc
:106750000002be0082017800010024000000200039
:10676000020020007ffc0700150007007548260086
:1067700014d52e0003002000fb01070090fe070047
:106780008d8070003400f9004f06be004f05be003a
:106790004f04be00000006006ffd07000778a3004d
:1067a00003003a00b0fd200091fc2300f4ff370005
:1067b0000160a0001602200066be8800f0ff3700ce
:1067c0000100e0000d003200ef0341000b00350036
:1067d000809fbe00821f78000002be008201780008
:1067e0009f0007004300200084d32800c700070053
:1067f000cf0178004f02be0099000700000006009c
:1068000060001000e08018000200370060031300f1
:10681000e0831b00889fbe008a9fbe008c9fbe0045
:10682000830441000405b800050eb8000501b80056
:106830008285450003064e00e0864e000409b8003c
:106840008285450003064e00e0864e000100e00010
:1068500002003d000406560085865e000500e0004b
:1068600002003d000006560081865e000d00e0003b
:10687000740032000700e000750032006022b800aa
:106880008783d1000683d3008582d300090054009a
:106890000000e9001b003c003b0035000804e80054
:1068a0000a0042008b804a000c014b008d814b0096
:1068b0003d020700040454000300e0000e00320013
:1068c000090028000918e100060032000200be009d
:1068d000080178004f06be004f05be004f04be0001
:1068e000000006000200e000f8ff3a0003002c0060
:1068f0000804e800f5ff37006000b8000001eb0075
:10690000f4ff37000804e8007e00e10001003400d5
:10691000e0012000cfecde00ef0060000100e000ad
:106920000c003200f08110000155de000359dd003b
:1069300002057500815dde000361dd008285750062
:106940000166de000369dd000206760081eede00ee
:10695000010050004400de006501b8000260010043
:106960000a0042008b804a000c014b008d814b00d5
:10697000cfff37000b0042008c804a000d014b0016
:1069800089814b00caff3700628444000000ea009e
:10699000030420000300e100010034000004200093
:1069a000cfbcde00ef0060000a003200f081100072
:1069b000032add00812ade000331dd0082827200bd
:1069c0000133de000339dd000203730081bbde000a
:1069d000010050004400de006501b80002600100c3
:1069e0000a0042008b804a000c014b008d814b0055
:1069f000afff37000a8042008b004b000c814b0038
:106a00008d814c00aaff37000a0043008b804b00a9
:106a10000c814c008d814c00a5ff37000a8043009b
:106a20008b804c000c814c008d814c00a0ff370006
:106a30000a8044008b804c000c814c008d814c00fe
:106a40009bff37000600be0008017800a1ff370059
:106a50000c01be000a00be006284440094ff3700af
:106a6000889fbe008a9fbe000004be000405be00d1
:106a7000030141000201e8008000eb000a42b80077
:106a80000b43b8008682420060804b000a4bb8007e
:106a90008682420007004800e08048000b4bb800a7
:106aa00006004000878048000103700002003a00a1
:106ab0000001eb00120037000900e00002003d0079
:106ac0000a0050008b8058000b00e00002003d00df
:106ad000080050008980580085824200000048006c
:106ae000818048008101df000300e00004003200e3
:106af0008582420000004800818048000201e900d0
:106b00004f05be004f04be00000006006218e10001
:106b10003b003500889fbe008a9fbe008c9fbe0050
:106b20008301e9000004be000205be0004067800ef
:106b3000620545000a05ea003c00be007050e10015
:106b4000170035000d0032007f50e10001003400d5
:106b5000fa012000f00655000801be0052010700ae
:106b60000d99de00cf99de003c004100bc80490059
:106b70008b05e900f8ff3c00140037000801be0057
:106b80004901070003017800cf99de003c00410075
:106b9000bc8049008b05e900f8ff3c000b00370082
:106ba000f00615000801be003f0107000a11de00d3
:106bb0008d1add00050171008a99de003c0041005c
:106bc000bc8049008b05e900f6ff3c000103df00b3
:106bd0000605ea00050034008a08dd007002150091
:106be0008402de00858070000a00dd000601780066
:106bf0004f06be004f05be004f04be000000060059
:106c00000300e00002003a006000b8000200050046
:106c10003400be0002000500e10241000200350020
:106c20009b01070000000600e2024100020035005f
:106c30003a01070000000600e302410002003500af
:106c4000a400070000000600b0ff070000000600d7
:106c5000889fbe008a9fbe008c9fbe000006be00bb
:106c600082057800741b2c00c5172500f3ff2f0048
:106c70007bff070066000700809fbe008101700057
:106c800036003200e7015000608258000d003100ec
:106c90000000e900c9d928006c00b8008904400050
:106ca0000c00be000b0178003902be00b90178006b
:106cb000b00007003902be00b9017800ad0007003e
:106cc000210037002800070014d52e007548260043
:106cd000030020000c03be000b0478000006be0079
:106ce00082057800c6fe0700d3ff2f008381450090
:106cf0000218e100140034000003be000204780012
:106d00000c00be000b01780094462800152d2400cd
:106d1000e3fd2f00bafe0700e3fd2f00838145004d
:106d20000218e100080034000003be0002047800ed
:106d30000c00be000b017800b4282600654c24002e
:106d4000f3fb2f00aefe07004f02be004f06be0051
:106d50004f05be004f04be00000006000c00be0040
:106d60000b017800f8ff37000003eb008101df0022
:106d70008301ea006f18e1000f0032000300e00019
:106d8000060032008308dd00708211008402de00fc
:106d9000858070000300dd00030343000100e00074
:106da00014003200040028000408e100130032003f
:106db0007e011300000006008100d1008080d30016
:106dc0004f00dd00f60020008101df008301ea00b2
:106dd0006f18e100e9ff3a008100d1008080d30004
:106de0000000eb00e60120008101df008301ea00e2
:106df000e2ff37006000b800020005000000e0007c
:106e0000ebff3a0001002c000603e900e8ff370021
:106e10000100e000210032008201e8002b00350073
:106e20007e0211001e0034006011b8007020e100e5
:106e3000040035008001780001007800cf88de0072
:106e4000700252000400e0000700320003017800e5
:106e5000700312008601dd000400de00860bdd00f9
:106e6000070070008488de00e10260000600280050
:106e700003036300f7ff27008383630082837300ab
:106e80000600e00005003200078172000200e00009
:106e90000200320061004000e0804800000006006f
:106ea0007e10e10001003a00000006000100e00051
:106eb00003003500f1ff2700f0ff2f00000006005f
:106ec0000100280000002000000006006000b8005b
:106ed000000006006218e1001d003500889fbe001a
:106ee0008a9fbe008c9fbe008301e9000004be00a3
:106ef0000205be00040678003c00be000801be008a
:106f0000690007008381d1000281d3003c00410069
:106f1000bc8049008b05e900f8ff3c000103df005d
:106f20008606ea00050034008d08dd007082160038
:106f30008402de00858070000d00dd00060178000f
:106f40004f06be004f05be004f04be000000060005
:106f50000300e00002003a006000b80002000500f3
:106f60003400be000200050060001000e080180040
:106f70000200370060021200e0821a000100e00007
:106f80003f0032000500e00039003200889fbe005b
:106f90008a9fbe00820378008304510004003d00f4
:106fa0000002fd008102fd008904ea0083037800ed
:106fb00001017800800078000000eb0005037800f4
:106fc000840278000002eb00060569000700350026
:106fd0000281d1008180d3000080d3000683d100dc
:106fe0008582d3000482d3008703e8007048e10063
:106ff000060035007f48e10029003c0005027800ca
:10700000860278004fb3de00f08454000900e000ef
:10701000080032000922de00708514008a2ddd0090
:107020000b027200892ade008a35dd008b82720035
:1070300009b3de00040040008580480006014900d5
:10704000b9000700838353000200e000090032000a
:107050000b0028000b10e1000c003200010078004a
:1070600082007800070178004f05be004f04be0083
:10707000000006006000b8000001eb00faff3700d6
:107080000400be0003017800000006000100e000db
:10709000f2ff3a0002002c008703e800efff370000
:1070a000f9012000d5ff3700889fbe008a9fbe00ef
:1070b0008c1f78000002be000203be000620b8004c
:1070c000062db8008a80400060814d000724b8007a
:1070d000072db8008a84440060864d00810044007a
:1070e00002814c00e0014e000700e000080035007e
:1070f0000500e00002003d000601510087815900b3
:107100004f0678004f05be004f04be000000060089
:107110000401510085815900f5ff37006218e10034
:107120001b003500889fbe008a9fbe008c9fbe005a
:107130008301e9000004be000205be0004067800d9
:107140003c00be000801be00d7ff07003c00410024
:10715000bc8049008b05e900faff3c000103df0019
:107160008606ea00050034008d08dd0070821600f6
:107170008402de00858070000d00dd0006017800cd
:107180004f06be004f05be004f04be0000000600c3
:107190000300e00002003a006000b80002000500b1
:1071a0003400be00020005000002eb008302df0095
:1071b0008502ea006f28e10023003a008301d10034
:1071c0008281d3000181d3008080d3004f00dd0095
:1071d000f40020008302df008502ea006f28e1004e
:1071e00019003a008301d1008281d3000181d300cc
:1071f0008080d3000000eb00e40120008302df0068
:107200008502ea006f28e1000f003a008301d100f7
:107210008281d3000181d3008000eb00d4022000e2
:107220008302df008502ea006f28e10006003a00d1
:107230008301d1008281d3000001eb00c403200050
:107240008302df008502ea000500e0000c00320046
:10725000708312008519dd008613de0087817100be
:107260000511dd00860bde00070171008508dd00d9
:107270008603de00878070000500dd000502420005
:107280000300e000010032000000060004000500d9
:107290006218e1001e003500889fbe008a9fbe0074
:1072a0008c9fbe008301e9000004be000205be0001
:1072b000040678003c00be000801be007aff07000b
:1072c0008100d0000281d2008381d2003c004100c5
:1072d000bc8049008b05e900f7ff3c000103df009b
:1072e0008606ea00050034008d08dd007082160075
:1072f0008402de00858070000d00dd00060178004c
:107300004f06be004f05be004f04be000000060041
:107310000300e00002003a006000b800020005002f
:107320003400be00020005008001eb000202df0015
:107330000402ea006f20e10010003a000201d100cf
:107340000181d3008080d3004f00dd00f3002000d6
:107350000202df000402ea006f20e10007003a00a9
:107360000201d1000181d3008080d3000000eb0036
:10737000e30120000202df000402ea000400e00052
:1073800009003200f00212000411dd00050bde00de
:10739000060171008408dd000503de0086807000b0
:1073a0000400dd00848141000200e00001003200a1
:1073b00000000600030005008f02b000889fbe0099
:1073c0008a9fbe008c9fbe008e1f7800000478004c
:1073d0000000e00003003200104078000004e000ec
:1073e00011003a00881f7800c0e32800801f780051
:1073f00010072000a6890200000000000003eb0037
:10740000e50420001407200053052000f2e62800c0
:10741000d102200080e7280040890200000000001f
:10742000e4875700184078008000eb0081b79f0088
:107430000005eb00fab79f000007eb008ebf9f002e
:10744000eeb79f00880478000004e00013003200cb
:1074500098407800d0c2b30080cf50005202320072
:10746000a0c3b30080cf50004d023200e0c2b30091
:1074700080cf5000460232000180fb0088010200ec
:10748000000000000000e000010032000a05e800f2
:10749000d94078000104e000eeff3a008fb8970071
:1074a000e18f500035023c000e00e000e90132009f
:1074b000e20f5700e3013a00ffb09700e18f500060
:1074c000dc013c000a00e000d6013a006000b80090
:1074d00090b79f00a1b79f000006be000005be0048
:1074e0008000eb00d1b79f00c1b79f00b1b79f00ec
:1074f0000802780088047800184078000004e00052
:107500000e003200ea4f50000c0032000e00e00086
:10751000ad003200a0c3b300994f100070003200dc
:107520008900e80081047800114078000004e00040
:1075300002003200ea4f5000f4ff3a00890f520077
:107540005c003a0002002000032724001fb09700cf
:10755000afb09700581e0200000000000000e000dd
:107560004a003d0002002000032724000c00be005a
:10757000581e0200000000000000e0003a003d003c
:107580009288280083c823000c00be00242d02002e
:10759000000000000004be00422b2a0013992300c3
:1075a0001fb09700afb09700242d0200000000002c
:1075b0000001be000800be005629020000000000c5
:1075c0000001be000a00be005629020000000000b3
:1075d0000005be000fb097000000e0001e00320062
:1075e0000bf0a2000a00be0001f0a1000200200082
:1075f000433b2400581e0200000000000000e00091
:1076000007003c000a00be004f0778004f06be008e
:107610004f05be004f04be008f02b10000000600ff
:107620000a00be005c1e020000000000809fbe0039
:10763000829fbe0003e82800831f780050082000c6
:10764000a689020000000000f0ff2f00f1f72700dc
:10765000ea875700ecff37008fb897000100e00081
:10766000e0ff3200deff37000c00be005c1e0200af
:1076700000000000809fbe00829fbe00e3ea280059
:10768000831f780040082000edff37001fb09700ef
:10769000afb097005c1e020000000000809fbe009b
:1076a000829fbe0001ef2800811f78003008200073
:1076b000e3ff3700891f7800841f780020f328003b
:1076c000801f780020082000a6890200000000002a
:1076d000f0ff2f00f1f72700e6875700caff3700b9
:1076e000e20f570012003a00a20020008000eb00d9
:1076f000040078009c0102000000000000017800f6
:107700000000e000080035006110b9009a1e020078
:10771000000000000005be000902e80084007800b7
:107720001e0020007fff37000001ea00f6ff37004f
:10773000e10f57001b003a00a20020008000eb0080
:10774000040078009c0102000000000000017800a5
:107750000000e000110035006110b9009a1e02001f
:10776000000000000006be000902e8006011b80039
:107770008000eb0004007800c2020200000000005c
:10778000f01e02000000000001f0a10090b79f0071
:10779000a1b79f000902780068ff37000001ea00e6
:1077a000edff3700e3f62800831f7800b0072000c4
:1077b000a689020000000000f0ff2f00f1f727006b
:1077c0008f87e90090ff37006fb097000000e0005e
:1077d000e4003200194178000280fb000100200023
:1077e00069005000e0805800e3062000830f50003d
:1077f000e08f5800cf003e000060010048ff3700d6
:10780000cc003700cb003700ca003700c900370072
:10781000c8003700c7003700c6003700c500370072
:10782000c4003700c3003700c2003700c100370072
:10783000c0003700bf003700be003700bd00370072
:10784000bc003700bb003700ba003700b900370072
:10785000b8003700b700370031ff3700b5003700f8
:10786000b4003700b3003700b2003700b100370072
:10787000b0003700af003700ae003700ad00370072
:10788000ac00370026ff3700aa00370024ff37007e
:1078900023ff3700a7003700a6003700a5003700f8
:1078a000a4003700a3003700a2003700a100370072
:1078b000a00037009f0037009e0037009d00370072
:1078c0009c0037009b0037009a0037009900370072
:1078d0009800370097003700960037009500370072
:1078e000940037003700370052003700320037006d
:1078f000900037008f0037008e0037008d00370072
:107900008c0037008b0037008a0037006f0037008b
:1079100029003700870037008600370085003700d0
:1079200084003700240037008200370081003700d0
:1079300080003700200037007e0037007d003700d0
:107940007c0037007b0037007a0037007900370071
:107950007800370077003700760037007500370071
:10796000740037001700370032003700120037006c
:10797000700037006f0037006e0037006d00370071
:107980006c0037006b0037006a0037004f0037008b
:1079900009003700670037006600370065003700d0
:1079a00064003700040037006200370061003700d0
:1079b00060003700000037000902e800840078000a
:1079c000d8fe37005fb097000000e0000f003a00db
:1079d0006011b8008000eb0004007800c2020200d1
:1079e00000000000f01e02000000000001f0a100f5
:1079f00090b79f00a1b79f000902e80084007800bb
:107a000013002000d3b79f00c6fe37001fb09700b9
:107a1000afb097005c1e020000000000809fbe0017
:107a2000829fbe0063f92800831f7800e0072000d2
:107a300003ff37003fb097000000e0001a003a0053
:107a4000048454000801780084007800c0fc2f00f2
:107a50000f0040004404020000000000c1fc2f00a1
:107a60008f80400001044400004ceb006011b8001e
:107a70008000eb00c0fc2f000f004000c20202009b
:107a800000000000f01e0200000000000005be0023
:107a90000bf0a1000902e800840078001300200028
:107aa000b3b79f009ffe37000a00be005c1e0200b5
:107ab00000000000809fbe00829fbe00e0fc280006
:107ac000801f7800c0072000ddfe37004fb0970010
:107ad0000000e0000e003a006011b8008000eb00ea
:107ae00004007800c202020000000000f01e020044
:107af000000000000006be000df0a1000902e80031
:107b00008400780013002000c3b79f0085fe370073
:107b10000c00be005c1e020000000000809fbe0042
:107b2000829fbe0061002900811f7800d0072000dd
:107b3000c3fe370000cdb300004041008900e800db
:107b4000e94f500077fe36000280fb00801f78006e
:107b5000801f7800e0032900801f7800f0072000d4
:107b6000d9fe3700ffb097000100e0002900320085
:107b7000e0c2b300994f100069fe3a00e28f500056
:107b800013003a00a20020008000eb0004007800ff
:107b90009c01020000000000000178000000e000ed
:107ba000090035006110b9009a1e020000000000b3
:107bb0000005be000902e8008400780013002000e0
:107bc000f3b79f0057fe37000001ea00f5ff3700ca
:107bd0007fb09700e10f50000a003a006011b80032
:107be0008000eb0004007800c202020000000000e8
:107bf000f01e0200000000000006be000df0a10013
:107c0000e4fe370061072900811f7800000820008a
:107c1000e7fe3700f3092900831f780010082000d1
:107c2000e3fe3700500d2900801f78005007200028
:107c3000dffe3700f3112900831f78004007200082
:107c4000dbfe370050162900801f78003007200027
:107c5000d7fe37000a00e0000e003a00ffb09700a0
:107c60000100e000070032007fb09700e20f5000f3
:107c700016fe3200d11a2900811f780070072000fb
:107c8000cbfe370023232900831f780060072000e4
:107c9000c7fe3700d12729000800780064040200dd
:107ca000000000000000e000300032004128290000
:107cb00008007800640402000000000080047800de
:107cc00091282900080078006404020000000000e8
:107cd00080b79f008fb997000300e00014003200c6
:107ce0000900e00002003a000000e000100032004d
:107cf0000900e0000b0032001980fb00801f7800b3
:107d0000e3282900831f780090072000a68902003d
:107d100000000000f0ff2f00f1f72700e487570074
:107d200039fe37008fb097001180fb00f3ff37005a
:107d30000900e000020032000000e00003003a0009
:107d400011002000e1b79f00e0fd37001080fb002c
:107d5000801f78001980fb00801f7800502e2900ba
:107d6000801f7800a007200057fe370063332900ea
:107d7000831f7800800720008dfe3700811f780068
:107d8000f33b2900831f780020072000dfff370026
:107d90007fb097000000e800f0b79f00bcfd3700ff
:107da0000e07e800bafd37008fb997008301e8009d
:107db00083bf9f00b6fd37004f05b000889fbe000f
:107dc0008a9fbe008c9fbe008e1f78000004be00fc
:107dd000020678000305780084057800417b2100c5
:107de0009140780070c4b30080cf500095003200fd
:107df000417b2100914078006340500080cf5000cb
:107e0000900032000102200010002000c85402003f
:107e1000000000000000e0008a0032000a00e000dc
:107e2000cb0032000c00e000b90032000800e00096
:107e300095003a000900e0008a0032008a1f7800ad
:107e40008a1f78008c1f78001904e00083003a0034
:107e500010462900801f7800891f780025462900d8
:107e6000851f7800608a020000000000ec87570040
:107e700001c2b300b1c79f00c1c79f00c0c7b30014
:107e8000d0df9f00e1df9f000007eb006044b800f7
:107e9000f5fd2f00858647006f0064003200320038
:107ea0008a0f54003000320024002000e78f540075
:107eb00001003c000002eb006348b80000004200f3
:107ec00005fa2f008f82420005004000ec407c0044
:107ed0000181fb00c411de0015452900e3c17a00d1
:107ee000334898006f01610062c17a0042489800ef
:107ef00002c2b3005248980002c15000e0c5b3006e
:107f0000804f510015003e0081f67c000804e80017
:107f10008904e8008a0f5400dfff3a00f08f540014
:107f2000ddff3200708014006300b90004005000cf
:107f30000081e8006348b90003fa2f008f814100f7
:107f400000804100040040006b004000010220005e
:107f50008004020000000000cfff3700e0c2b30041
:107f600080f67c00e9ff37000800e00012003400d2
:107f7000a0c0b30080f67c0001fe2f000180470006
:107f8000090040000048eb0000fa2f000f004000fd
:107f90008e040200000000000001780001fa2f00aa
:107fa0008f80400010002000c24c02000000000042
:107fb0000e07e8008004eb008a0f54002100310016
:107fc0000b00e0000f003200110009000b87d80001
:107fd0008000fd000000e0000a003a000800e00018
:107fe00012003200f03f29008e0402000000000061
:107ff00000017800f13f290010002000c24c02006f
:1080000000000000881f7800881f7800434929007d
:10801000831f7800a0f92f000f00400060060200c7
:1080200000000000e68757009fff3700004029004e
:108030008e040200000000000001780001402900c9
:10804000edff37004f0778004f06be004f05be001a
:108050004f04be004f05b10000000600f0492900a2
:108060007cff37008a1f78008a1f78008c1f7800f9
:10807000234a2900831f7800608a02000000000064
:10808000e88757007aff37000808a300190032007c
:108090000900e0000f0032008a1f78008a1f780074
:1080a0001904e00009003a0010462900801f7800fa
:1080b000891f7800014d2900811f7800608a020025
:1080c00000000000ea87570069ff3700f0492900e7
:1080d000f6ff37008a1f78008a1f7800704e29004b
:1080e000801f7800608a020000000000e6875700c9
:1080f0005fff37000818a3005dff32008a1f780079
:108100008a1f780033502900831f7800f5ff37005d
:1081100061512900811f7800b0082000a689020063
:10812000000000000003eb00e5042000b40820007c
:108130005305200032532900e11a200080e728006f
:1081400040890200000000008f87e90037ff3700f8
:10815000b0532900801f7800608a020000000000f0
:108160008f87e900b7ff3700889fbe008a1f78001d
:1081700080047800010478000000e0006100320013
:108180000800e0004e0034000800e0004a00320021
:108190009940780000c2b30080cf50003d0032000b
:1081a000e9cf50003b0032001a002000d0c2b300db
:1081b00080cf500035003200b0c2b30080cf5000f5
:1081c0002f0032000800e00006003200194078005d
:1081d00001c2b300814f500020003200e94f50002f
:1081e0001e0032006033b8000804e900e10f4400cb
:1081f0001100320005cdb30019427800054042005d
:10820000e94f50000c003e006a31b8006a38b900ee
:10821000808141000480fb000003b100cf80de00bc
:1082200002034000838348008904e8000804e90051
:10823000e10f4400f0ff3a006151b9000230b8008c
:1082400003b2b900048240000791b90082004200e5
:108250004f0578004f04be00000006008904e800c6
:108260000804e900dfff320019407800814f500018
:10827000faff3200e94f5000f8ff3200d9ff370013
:108280008904e8000804e900ceff37000085eb0010
:10829000fbff37008904e8000804e900060032000b
:1082a0009940780080cf5000faff3200e9cf5000ab
:1082b000f8ff3200bcff370099407800baff370062
:1082c000881f780021552900811f78007008200040
:1082d000a689020000000000080378006505200060
:1082e000740820005305200012572900712b20002c
:1082f00080e728004089020000000000e487570062
:10830000a1ff370070572900801f78006008200007
:10831000a6890200000000000003eb00e504200035
:10832000640820005305200012572900312b20003b
:1083300080e7280040890200000000008f87e900e4
:108340008fff3700f6874700889fbe008a9fbe00d8
:108350008c9fbe008e1f7800d0b79f00e1b79f00b2
:1083600002067800f3b79f00840578000400e0005f
:10837000a50032000c00e00004003200eb0f4600c4
:1083800002003500eb0f5600100034008c1f7800ff
:1083900091592900811f780090082000a6890200c9
:1083a000000000000c037800250520009408200040
:1083b00053052000625b2900a138200080e72800d7
:1083c0004089020000000000e48757008c06780016
:1083d0000c00e0008a0035005fb09700efb0970016
:1083e000e00f5000e08f58007e0035008000eb0069
:1083f00081bf9f005fb49700efb497000c00e000ce
:10840000380035000d05e900090033000a00e000de
:1084100022003a000fb997000200e0001f0032006e
:10842000d0c2b300804d78000a05e900f7ff3b0099
:10843000e00f5400e08f5c000c003a007fb1970021
:108440000200e000020032000040eb0080f57e00f8
:108450000b0078004f0778004f06be004f05be00a6
:108460004f04be006f01b100000006008c1f7800b1
:108470004fb09700dfb09700809fbe00c15b29001e
:10848000811f7800a0082000a689020000000000db
:108490000000eb00e8875700eeff3700e00f5400c4
:1084a000e08f5c0003003a0000c3b30080757d00dc
:1084b000ddff3700a2002000030020000800be00fe
:1084c0009c040200000000000203be000002be0087
:1084d00001c3b3000140430080757d000404be0069
:1084e000d1ff37000007eb000fb997000285560057
:1084f000e00f150013003d00a20020000300200043
:108500000800be009c040200000000000203be0040
:108510000002be0001c3b30001404300e2fd2f0092
:108520000e01410000f17f000404be00e00f520084
:10853000e08f5a00030032000e07e8008a0f570050
:10854000edff3500e00f5400e08f5c00c7ff3a00fc
:108550000005eb000d00e0000f003400d3c2b300b3
:10856000e2fd2f000f0141000fba97008400410087
:1085700002c2b3000a00e0000d003a000fb89700f5
:108580000000e0000a003200834d78000a05e80090
:108590008d0f5500f7ff3500ffb097000100e00098
:1085a000abff32000040eb0080757d00a8ff370074
:1085b0000fba9700040055008e0f500004003c00d5
:1085c0000a0057006140780080757d00efff37009a
:1085d0007fb097000000e000efff3a0082757d0059
:1085e000eaff37001100200081bf9f005fb09700b5
:1085f000efb0970060041000e08418007fff3700a0
:108600008c06ea0074ff3700105f2900801f780095
:1086100080082000a6890200000000000003eb0093
:10862000e50420008408200053052000625b290037
:108630006138200080e72800408902000000000027
:108640008f87e9004bff3700e8874700889fbe000f
:108650008a9fbe008c9fbe008e1f780000077800a6
:10866000e1b79f00f2b79f0083bf9f000404be00e4
:108670000605be000000e000690032006fb0970000
:108680000000e000560032000801be001fb0970055
:10869000afb0970044290200000000000004be00b3
:1086a0007fb197008fb997000a00be0056290200db
:1086b0000000000052a32f00e3c02300242d02007d
:1086c0000000000048320200000000000001be006f
:1086d0000800be00242d0200000000009287210047
:1086e000a3282400242d0200000000000006be0084
:1086f0007fb197008fb997000a00be00442902009d
:108700000000000092872100a3282400242d0200ed
:10871000000000000004be000c01be000c00be0002
:10872000242d0200000000000005be000801be006c
:108730000800be00242d0200000000000001be0061
:108740000a00be005629020000000000302e020080
:1087500000000000008fbe000c01be000800be003b
:10876000461f02000000000012ee220053262400e3
:10877000242d0200000000000001be0000002000c7
:10878000412b240044290200000000000004be0028
:108790006011b800801f0200000000000000e0002f
:1087a00006003d0002002000433b24000800be00fc
:1087b00056290200000000000004be006fb09700c0
:1087c0000888be000000eb004f0778004f06be008f
:1087d0004f05be004f04be008f00b1000000060030
:1087e000e0602900801f7800e0082000a6890200d0
:1087f000000000000003eb00e5042000e408200076
:1088000053052000926329006116200080e72800ac
:1088100040890200000000008f87e9009aff3700be
:1088200070642900801f7800d0082000a68902000b
:10883000000000000003eb00e5042000d408200045
:1088400053052000926329002116200080e72800ac
:1088500040890200000000008f87e90087ff370091
:10886000e4874700889fbe008a9fbe008c9fbe00a1
:108870008e1f780000067800810578000205e90067
:108880000200e00007003a000000eb004f0778000c
:108890004f06be004f05be004f04be004f00b100a2
:1088a000000006009c4678001b84fb000d80fb0046
:1088b00080bf9f00ca04020000000000800478000e
:1088c0000807780008007800ca04020000000000d1
:1088d000808f54000a003a000000eb000d04e00015
:1088e000eaff32000c06e8008b05e8000a00780079
:1088f0000a05e9000000e000eaff3a00e2ff370065
:108900000fb89700ca0402000000000000047800bd
:108910000e007800ca0402000000000000005400ad
:10892000daff3700889fbe008a9fbe008c9fbe0082
:108930008e1f780080057800010578001b467800be
:108940001a84fb000c87fb000e007800ca040200aa
:108950000000000080047800880678000800780095
:10896000ca04020000000000808f54000b003a008f
:108970000000eb000c04e000030032008b05e8006f
:108980000a05e800edff37004f0778004f06be00ec
:108990004f05be004f04be00000006000e00780028
:1089a000ca04020000000000000478000d007800f6
:1089b000ca0402000000000000005400f2ff37006b
:1089c000889fbe008a9fbe00000478008105780061
:1089d00082047800030578000000e0000200320005
:1089e0001004e00006003a00004deb00800ceb00a4
:1089f0000000eb004f05be004f04be000000060063
:108a0000d804020000000000000444001804e00044
:108a1000f5ff32008b00780008007800fa040200ad
:108a20000000000000004400800c7800104d780029
:108a3000190078001004e000020032000048eb004a
:108a4000990ce80008007800eaff370081027800fe
:108a50008000eb0000027800104078000004e00085
:108a6000060032000080fb007f09b8008200400051
:108a7000544078000004e000faff3a0011000900b9
:108a80008580d8008000fd00000006001600fa0076
:108a9000889fbe008a9fbe008c1f7800a2480200fb
:108aa00000000000a0ea2d00801f780061872900e7
:108ab000811f7800608a020000000000e4875700f0
:108ac0001848e20006003200b191290080812000a0
:108ad00092440200000000000000e00026013a007d
:108ae00028922900881f7800608a02000000000098
:108af00080c4b300b4f7b70010c0b3001aefb700da
:108b00008f87e900ec0c2200c237ef00c437ef007a
:108b1000007d20000100200080b79f0091b79f00da
:108b2000e2bb8000f3bb8000c00320000014b8004b
:108b30000098b900808444000800be00841f020031
:108b400000000000b0b79f00c1b79f00d2b79f00e0
:108b5000e3b79f00e00f5400e08f5c00fc0035009d
:108b60001a4fe200f7003a00417b21009140780063
:108b700080c4b30080cf5000f20032000040eb0010
:108b8000c0e79f00417b21009140780070c4b30092
:108b900080cf5000b4003200417b2100914078002a
:108ba000d0c4b30080cf5000ab00320001042000dd
:108bb00020002000c8540200000000000000e00077
:108bc000840032003008e2004a003a004fe097008b
:108bd0000024a000c0e79f0002fe2f000f0141000b
:108be000fc80570030002000c44802000000000054
:108bf000000478000000e000340035000800e000c8
:108c00000f0032004fe097000028a3002b003a002d
:108c10000018a3000a003200417b21009140780037
:108c200070c4b30080cf50001c003200417b210093
:108c300091407800d0c4b30080cf500007003200cc
:108c400010be800021be800061004000e08048002e
:108c500010be880021be8800c1ff3700004eeb0027
:108c60008001eb0012002000e10c220002007800dd
:108c70001e4b02000000000030c0b3009c4f1000eb
:108c8000efff3a00200020007051020000000000b9
:108c900080c4b300b4f7b700e9ff3700885602007c
:108ca00000000000e10f5000e0ff3a000104200046
:108cb000f451020000000000dcff3700226c0200cb
:108cc000000000004fe09700d1ff37000003eb00e9
:108cd0008002eb0000027800d304200022962900d5
:108ce000f10e20007096290040890200000000006b
:108cf000c2ff3700765a020000000000f0b79f0064
:108d000081bf9f0092bf9f00a3bf9f0028bd80002e
:108d100039bd80000800be00841f02000000000072
:108d2000e00f5400e08f5c00240035000002be001c
:108d30000203be007fb097008fb897001fb997005d
:108d4000afb997008a1f0200000000003e20020019
:108d5000000000000005be00b2ac8000c3ac800083
:108d600002015000838158008041800001002000f2
:108d7000800f5100818f590094ff3900606f2100ee
:108d800050960200000000000000e00003003a00de
:108d9000baac8800cbac88008cff3700801f78000d
:108da000e8962900881f780090322000a6890200ea
:108db00000000000e4875700f5ff37006022b8008c
:108dc00006002000071f24008a2002000000000087
:108dd000d6ff370008102000881f780027bd21002b
:108de00006202000257d21005400200041002000a5
:108df000424080005340800020002000524e02007c
:108e0000000000008f87e9000000e0006dff3200e5
:108e100020002000801f780081992900811f7800a0
:108e200050042000a6890200000000002600200057
:108e3000d5042000540420008501780022962900e2
:108e4000b10c20007096290040890200000000004b
:108e5000e48757005bff37004fe097000014a00045
:108e6000c0e79f0051ff37000104200010002000e0
:108e7000c8540200000000000000e00004003200be
:108e80004fe097000014a000c0e79f0042ff3700aa
:108e90003fb29700cfb297005fb39700efb3970050
:108ea000e86e21003800be002801be008a200200c2
:108eb000000000000004be000205be00765a020059
:108ec000000000000002be000203be000800be0059
:108ed0000a01be0084210200000000000000e00042
:108ee0002dff3d00010420001000200086500200ec
:108ef000000000000000e000e1ff32001000200050
:108f0000801f7800119c2900811f780070192000b3
:108f1000a68902000000000016002000d5042000f1
:108f2000741920008501780022962900210b200069
:108f3000709629004089020000000000e487570075
:108f4000cfff3700245b02000000000004ff370061
:108f50006022b80006002000071f24008a200200bb
:108f600000000000b0b79f00c1b79f00d2b79f00bc
:108f7000e3b79f00fafe37001a6fef002c08e200fb
:108f80006800320040012000801f7800919f290076
:108f9000811f78002040800031408000809fbe000b
:108fa000d19f2900811f7800608a02000000000024
:108fb000ea87570020c0b300c0e79f0000e224000a
:108fc0000100200080b79f0091b79f0002fe2f0094
:108fd0000f014100fc80570010002000c44802002f
:108fe00000000000000478000000e00043003500ad
:108ff000e10f54000b003200d0c4b300b4f7b70047
:109000004040800051408000809fbe00c1a52900e3
:10901000811f7800608a020000000000e687570088
:10902000b8fe3700800c20000100200080b79f00b0
:1090300091b79f0003fe2f008f8141000801780047
:10904000e10c2200080078001e4b02000000000026
:10905000e10f50000f003200e8aa2900881f7800b5
:1090600000192000a6890200000000000003eb00a8
:1090700005192000d40420008401780022962900dc
:10908000810820007096290040890200000000003d
:109090009bfe3700a8b888002c08e2000f003200c1
:1090a000ec0c220031c0b3009ccf10000300320052
:1090b00070c4b300b4f7b70093fe370080c4b300a8
:1090c000b4f7b7001202200011ae290008007800a2
:1090d000c24c0200000000008bfe370080c4b300c9
:1090e000b4f7b7002202200031b029000800780050
:1090f000c24c02000000000082fe37000003eb00bb
:1091000080027800d404200084017800229629008f
:10911000b10620007096290040890200000000007e
:10912000b3ff370048012000881f780060b2290093
:10913000801f7800608a020000000000e48757006a
:109140009cff3700e0c4b300b4f7b7009a8902006f
:1091500000000000ea59020000000000e48b020059
:10916000000000006a880200000000003c56020077
:10917000000000008e57020000000000b6590200f7
:109180000000000000000500889fbe008a9fbe000e
:109190008c9fbe008e1f780080017800010478004b
:1091a000820478000000e900e70f500058003e00fc
:1091b000114178000204e0004d0032000047eb004e
:1091c0000006eb007bc5b3000900e000060032009a
:1091d0001900be00e9c55500e00f5000e08f5800af
:1091e00001003200e6c545001dc0b3000045eb009c
:1091f0000218a30031003a000228a30023003a001d
:109200000c00e0001e003a000a04e00011003a00e1
:1092100070c5b30080cf55001500320040c5b300c3
:1092200080cf55000b003a000d81fb001900be00f5
:10923000a05702000000000039011000a9811800a9
:109240004240a900030034008046eb00184178003a
:10925000e7ff37000e4c78000c0078004f077800cd
:109260004f06be004f05be004f04be0000000600c2
:10927000d4e2a8000140fe00d4e2a900f3ff3700c9
:10928000a459020000000000f2ff37000104200092
:1092900020002000be0507000000e00005003200ad
:1092a0007815e200d6ff32000e24a0000c06e8007c
:1092b000d3ff37000a45e800d1ff37000104200042
:1092c00010002000b20507000000e0000600320098
:1092d0003e15e200020032000e14a0000c06e80069
:1092e00018417800c4ff37000a45e800fcff37004a
:1092f00022b42900821f7800c0032000a689020042
:10930000000000000080eb008f87e900d3ff3700ea
:10931000831f780010b62900801f7800b00320005a
:10932000a6890200000000000080eb00e4875700df
:10933000caff3700e4874700889fbe008a9fbe00af
:109340008c9fbe008e1f7800000478008105780095
:1093500002057800030778000000e900e10f5000e3
:10936000a3003e000b00e00091003200e10f550029
:109370007e00360001042000080078008405070004
:109380000000e0006800320075c5b3000e00e00088
:10939000060032001e00be00e9c25200e00f50007d
:1093a000e08f580001003200e6c24200a003200016
:1093b0000040b800a34f210083044000e251210087
:1093c00002004000904678000a04e9000006eb0025
:1093d0000045eb0012c0b3004240a9002a0034004f
:1093e0005900900088007800800f5400010034007c
:1093f000800078000100e00035003400ee81440078
:10940000930078003145780081097800090a9000be
:109410004900900000004200808f50000100390098
:10942000840978008a5d78000c06e8000804e900e9
:1094300021042000914078008180fb00c508de00f7
:1094400001007800baf7b70000ceb3004260b70061
:10945000590090000000e900d0049800c508dd0024
:1094600042c0bf007f4060000140700042e0b70092
:109470008d4f5500140032000800e0001200340047
:109480000800e000d6ff3c0084d7bf000018a3000e
:109490000a003a000c0078008d4f550001003200a0
:1094a0000c00ea004f0778004f06be004f05be00d3
:1094b0004f04be004f00b10000000600a459020096
:1094c00000000000f3ff3700804deb00eeff370097
:1094d000e0c4b30080cf5200ebff3200694040008f
:1094e00080cf52000c0032000281fb001e00be0043
:1094f00085bf9f00a0570200000000003e01100041
:10950000ae8118008fba97004240a900deff3400f8
:109510000041eb00daff3700d4e2a8000140fe0072
:10952000d4e2a900d6ff3700881f7800c2b929000d
:10953000821f780000042000a689020000000000bd
:1095400008037800d504200004042000330520001f
:10955000f2bc2900d10e200090bd290040890200f4
:1095600000000000e487570087ff37008a1f78005b
:1095700020be2900801f7800f0032000a689020089
:10958000000000000a03780065052000f4032000b5
:1095900033052000f2bc2900810e200090bd290077
:1095a0004089020000000000e487570071ff370087
:1095b000e3c02900831f7800e0032000a689020091
:1095c000000000000003eb00e5042000e40320009d
:1095d00033052000f2bc2900410e200090bd290077
:1095e00040890200000000008f87e9005fff37001c
:1095f000881f780020002000801f7800d2c3290037
:10960000821f7800d0032000a6890200000000001d
:109610000803780025052000d4032000330520002e
:10962000f2bc2900010e200090bd290040890200f3
:1096300000000000e68757004aff3700e487470034
:10964000889fbe008a9fbe008c9fbe008e1f780040
:10965000000478000106780082047800030778008f
:109660000000e900e10f5000b3003e000c00e000f4
:10967000a10032000900e0008e0032000104200049
:1096800008007800c20407000000e0007800320003
:1096900071c5b30081f79f000e00e00008003200a2
:1096a0001e00be00e2c4b30082f79f00e00f50002e
:1096b000e08f58000200320043c5b30083f79f00db
:1096c000a00320000040b800a24f21000205400086
:1096d000890578008006eb0013c0b30093f79f0064
:1096e0000900e000300034005a0090000b047800bc
:1096f000808f550001003400000478000800e0006d
:10970000440034000a089000ca00900001004000a4
:10971000fa00900081045000890f54002f0034009b
:10972000090178000c007800180502000000000014
:1097300009004600090154008a089000180502003b
:10974000000000000a0890000800400009005000d6
:1097500070059800080646008886460088855500f2
:1097600021042000914078008180fb00c508de00c4
:1097700001007800baf7b70000ceb3004260b7002e
:109780005a0090000800500050059800c508dd0000
:1097900042c0bf007f4060000140700042e0b7005f
:1097a0000b00e000d0ff3c0084d7bf000018a300ee
:1097b00007003a000d0078004f0778004f06be0002
:1097c0004f05be004f04be004f00b1000000060070
:1097d000a459020000000000f6ff370008017800dd
:1097e0000c0078001805020000000000fa0090004c
:1097f00088804000710598000a0990004a00900096
:1098000000004100808f5000d2ff3900720598009f
:10981000d0ff3700e0c4b3008ff0970080cf500036
:10982000e1ff32006940400080cf50000c00320060
:109830009ff197000381fb001e00be00a0570200ad
:10984000000000003e011000ae8118004240a90057
:10985000d5ff34008041eb0093f79f00d0ff370025
:10986000d4e2a8000140fe00d4e2a900ccff3700fa
:10987000881f7800c0c72900801f7800400420009e
:10988000a68902000000000008037800d50420002b
:109890004404200033052000f2ca290031162000bc
:1098a00090bd29004089020000000000e4875700b5
:1098b00077ff3700801feb0093cb2900831f7800d0
:1098c00030042000a6890200000000000003eb0025
:1098d000650520003404200033052000f2ca290069
:1098e000e115200090bd2900408902000000000021
:1098f000e487570061ff370052ce2900821f7800ad
:1099000020042000a6890200000000000003eb00f4
:10991000e50420002404200033052000f2ca2900b9
:10992000a115200090bd2900408902000000000020
:109930008f87e9004fff3700881f78002000200044
:10994000801f780041d12900811f78001004200079
:10995000a689020000000000080378002505200009
:109960001404200033052000f2ca290061152000ec
:1099700090bd29004089020000000000e6875700e2
:109980003aff3700889fbe008a9fbe008c9fbe00b2
:109990008e1f78000006be00820578003408e200c1
:1099a0000b003200417b21009140780040c4b3009d
:1099b00080cf50000600320001022000100020007d
:1099c000f303070018c0b3000000e00001003a00f4
:1099d0000044eb000c00e900e10f50000b003600e2
:1099e0000804e000a5003a000c03780025052000db
:1099f000140420003305200032d52900411d200029
:109a000090bd290040890200000000000d00e00028
:109a1000870032000b00e0000b003a000804e00071
:109a20007b003a000003eb006505200034042000b1
:109a30003305200032d52900011e200090bd2900e9
:109a40004089020000000000010220000c007800a4
:109a5000cf0307000000e0000b003a000804e0001c
:109a600063003a000c0378006505200044042000e0
:109a70003305200032d52900711e200090bd290039
:109a80004089020000000000a00320000060b80030
:109a9000c2502100020540000007eb000b00e0006f
:109aa00036003200ca0090005a009000008050003a
:109ab0004240a9004a0034000b047800808f550012
:109ac00001003600000478000a0890000100400000
:109ad000ea01900083045000890f540031003400e3
:109ae000090178008d007800030078001805020055
:109af000000000000a089000090154008980460017
:109b000018050200000000000a089000080040004c
:109b10000900500060059800888646008885550039
:109b20000807470021042000914078008180fb0055
:109b3000c508de0001007800baf7b70000ceb30018
:109b40004260b7005a00900008004000500598009d
:109b5000c508dd0042c0bf007f40600001407000ca
:109b600042e0b700e10f56000c003200e20f560051
:109b7000080032000b00e000caff3a000e00780037
:109b80004f0778004f06be004f05be004f04be00d1
:109b9000000006008720a800f6ff37008540a800d7
:109ba000f4ff3700080178008d007800030078008a
:109bb0001805020000000000ea00900088804000c4
:109bc000610598000a0990004a00900000004100d9
:109bd000808f5000d0ff390062059800ceff37001b
:109be000d4e2a8000140fe00d4e2a900e1ff370062
:109bf0008c1f7800e0d52900801f780040042000e9
:109c0000a689020000000000e487570095ff370096
:109c1000801feb0022d92900821f78003004200029
:109c2000a689020000000000e48757007dff37008e
:109c30000804e0000a003a000003eb00e5042000fd
:109c4000240420003305200032d52900a11d200066
:109c500090bd290040890200000000006dff370020
:109c6000e0db2900801f780020042000a689020084
:109c7000000000008f87e900efff37008c1f78009d
:109c800020002000801f7800e2de2900821f78007b
:109c900010042000a689020000000000e68757009b
:109ca00051ff3700e6874700889fbe008a9fbe00ad
:109cb0008c9fbe008e1f7800800478000205be00d5
:109cc000f1b79f00040778000506780086bf9f0063
:109cd000870678000000e900e10f5000f8003e0020
:109ce0000a01be00e206b1000380b10020192c0079
:109cf00011002000800f5100818f5900df003e00cd
:109d0000ffb097000100e900e60f5000ca003e00d6
:109d10000e00e900e60f5000b6003e000c00e00027
:109d2000a40032000fb997000200e000900032005a
:109d30000d00e0007e0032003fb197000200e0001d
:109d40006a003200a00320000048b800624e2100e3
:109d500002044000180890000006b2005f003a00bc
:109d6000080078001c0009000018eb000a01be0082
:109d70000900780017030700e1ff2f000000e00052
:109d80002c003a002c1498001c1498000c14980015
:109d90003d1c98002d1c98001d1c98008fb8970042
:109da000610c98003fb1970072149800a0c0b300f6
:109db000007c9800e18f54002e003200e28f5400a6
:109dc00023003a001622ef008f00a9008f20a9007f
:109dd0008700a9008720a90067416700a0c0bf00d5
:109de00081cfb3000140600002407000a0e0b700e6
:109df000efe8970067c160004411dd00a0c0bf001c
:109e0000f1c8b3000140600002407000a0e0b7005c
:109e100000002800b010880000402800c010880012
:109e20008f00a8008f20a80010062000100c9800ba
:109e30008000eb00010078004f0778004f06be005d
:109e40004f05be004f04be006f00b10000000600c9
:109e5000891f7800e2e22900821f780000042000b8
:109e6000a6890200000000008080eb00e487570014
:109e7000f0ff37000c22ef008d20a9008d40a900d3
:109e80008520a9008540a900674167004411dd00d5
:109e900098c0bf00f1c8b3000140600002407000ec
:109ea00098e0b7006fe897006741600099c0bf0075
:109eb00081cfb300014060000240700099e0b7001c
:109ec0000000280060108800004028007010880002
:109ed0008d20a8008d40a800d3ff3700891f78008f
:109ee00030e62900801f7800dcff3700801feb0080
:109ef000e0e82900801f780020042000a6890200e5
:109f0000000000000003eb00650520002404200091
:109f100033052000d2eb2900e124200090bd290068
:109f20004089020000000000e487570085ff3700e9
:109f300071ec2900811f780020042000a68902000e
:109f4000000000000003eb00e504200024042000d2
:109f500033052000d2eb2900a124200090bd290068
:109f600040890200000000008f87e90072ff37007f
:109f7000801feb0030ef2900801f780020042000b4
:109f8000a6890200000000000003eb006505200028
:109f90002404200033052000d2eb29006124200096
:109fa00090bd29004089020000000000e4875700ae
:109fb0005fff370021f22900811f78002004200074
:109fc000a6890200000000000003eb00e504200069
:109fd0002404200033052000d2eb29002124200096
:109fe00090bd290040890200000000008f87e90031
:109ff0004cff37008e1f7800e0f42900801f7800a6
:10a0000020042000a6890200000000000e03780052
:10a01000250520002404200033052000d2eb290070
:10a02000e123200090bd29004089020000000000cb
:10a03000e487570039ff3700811f7800b2f9290003
:10a04000821f780020042000a68902000000000082
:10a050005fb397002505200024042000330520006d
:10a06000d2eb2900a123200090bd290040890200e5
:10a0700000000000e487570025ff37008a9fbe00dc
:10a0800092fe2900821f780020042000a689020089
:10a09000000000000a0378002505200024042000a9
:10a0a00033052000d2eb29006123200090bd290058
:10a0b0004089020000000000e687570010ff3700cb
:10a0c000891f780020002000801f780081022a006c
:10a0d000811f780010042000a68902000000000003
:10a0e0000903780025052000140420003305200012
:10a0f000d2eb29002123200090bd290040890200d5
:10a1000000000000e6875700f5fe3700889fbe007c
:10a1100080047800010478000000e900e10f50009d
:10a120005c003e0000022000800f5400130032004b
:10a1300000042000800f540010003200881f7800b7
:10a1400070062a00801f780020042000a6890200e3
:10a1500000000000080378002505200024042000ea
:10a1600033052000120a2a00712e200090bd29001c
:10a170004089020000000000e4875700a00320008f
:10a180000048b800824f2100020040001008a300e0
:10a190003d003200880078000102b2001000640027
:10a1a000880f50002a003200e18f54001d00320059
:10a1b000e28f540012003a000100e0000c0032006f
:10a1c0008720a9001942a80019e2a8008f20a80042
:10a1d000a00320000048b800824f21000200400088
:10a1e000100874000000eb004f04be0000000600e1
:10a1f0008700a9001822a9008f00a800f4ff3700eb
:10a20000891f7800000b2a00801f780000042000be
:10a21000a6890200000000000080eb00e4875700e0
:10a22000f1ff37000100e000050032008540a90081
:10a230000f42a8000fe2a8008d40a800e4ff3700fd
:10a240008520a9000e22a9008d20a800e0ff37007c
:10a25000a00e2a000100e00001003a00300f2a00a1
:10a26000801f7800891f7800b20f2a00821f7800b3
:10a2700000042000a6890200000000000080eb001e
:10a28000e6875700d8ff3700891f780030132a006f
:10a29000ddff3700891f780020002000801f780034
:10a2a000e2162a00821f780010042000a68902000e
:10a2b0000000000009037800250520001404200098
:10a2c00033052000120a2a00312e200090bd2900fb
:10a2d0004089020000000000e687570091ff370028
:10a2e000881f7800000478000000e900e10f5000aa
:10a2f0002a003e00e10f54001d003200e20f54001e
:10a3000012003a001622ef008f00a9008f20a9004a
:10a310008700a9008720a90080cfb300a060b60005
:10a32000f0c8b300a060b6001822ef00a003200020
:10a330000040b800824f2100020040000008eb00fe
:10a340000000eb004f04780000000600881f780032
:10a35000201b2a00801f780000042000a68902002c
:10a36000000000000080eb00e4875700f5ff370095
:10a370000c22ef008d20a9008d40a9008520a900a6
:10a380008540a900f0c8b3009860b60080cfb30044
:10a390009960b6000e22ef00e4ff3700881f7800b6
:10a3a00020002000801f7800821e2a00821f780073
:10a3b00010042000a68902000000000008037800b5
:10a3c00025052000140420003305200082222a00e5
:10a3d0008135200090bd2900408902000000000066
:10a3e000e6875700c3ff3700889fbe0080047800cf
:10a3f000010478000000e900e10f50003f003e003a
:10a4000000022000800f54001300320000042000de
:10a41000800f540010003200881f780030232a007b
:10a42000801f780020042000a689020000000000a0
:10a4300008037800250520002404200033052000af
:10a44000e2262a00d139200090bd2900408902006f
:10a4500000000000e4875700e18f54001d00320027
:10a46000e28f540012003a000858a3000d00320099
:10a470008f20a9008720a9001942a90019e2a9008c
:10a48000a00320000048b800824f210002004000d5
:10a490000881ea00100861000000eb004f04be00d4
:10a4a000000006008f00a9008700a900f4ff370014
:10a4b000891f7800e2272a00821f7800000420000c
:10a4c000a6890200000000000080eb00e48757002e
:10a4d000f2ff37000858a300050032008d40a900a4
:10a4e0008540a9000f42a9000fe2a900e4ff370050
:10a4f0008d20a9008520a900e1ff3700891f780081
:10a5000020002000801f7800922b2a00821f7800f4
:10a5100010042000a6890200000000000903780052
:10a52000250520001404200033052000e2262a001f
:10a530009139200090bd29004089020000000000f0
:10a54000e6875700aeff3700809fbe00829fbe00a7
:10a55000849fbe00861f78008041eb00d4c2bf00fc
:10a560000080fb004700de008082fb00d4e2a900ef
:10a570008540a90030aa800041aa80006100400007
:10a58000e080480030aa880041aa88005015e20007
:10a590001b003200d6002000b2aa800074aa8000fe
:10a5a0000f22ab0014003a00a1aa800011407800ed
:10a5b000ea4f50001c0032008041eb000080fb009d
:10a5c000801088008100e800a1aa880004004100f2
:10a5d000808f500001003900a2aa88005035ed009c
:10a5e00050aa800061aa800061004000e08048001d
:10a5f00050aa880061aa88005015e200e8ff3a00de
:10a60000c728dd00d4c2bf000074a1000140700063
:10a61000d4e2b7004f0378004f02be004f01be00e6
:10a620004f00be00004006000304e000e2ff3a00d5
:10a6300013c0b30086108800e9ff3700809fbe007a
:10a64000829fbe00d4c2bf000080fb004700de0036
:10a650008081fb00d4e2a900d4c2a8008520a90013
:10a66000a0a98000b1a9800061004000e0804800fe
:10a67000a0a98800b1a988000e22ab000700320013
:10a6800000a9800011a9800061004000e08048001e
:10a6900000a9880011a988003235a8000e02ab007d
:10a6a0000c0032000e42ab00170032003255a800f9
:10a6b00020a9800031a9800061004000e0804800ae
:10a6c00020a9880031a98800901080000e02ab00fc
:10a6d000f4ff3a000e22ab00020032000e22a90065
:10a6e0003235a900d4c2a900c718dd00d4c2bf000a
:10a6f0000074a10001407000d4e2b7004f01be0019
:10a700004f00be00004006003255a900f1a98000ac
:10a71000e0a98000808f5000130031003295a9001d
:10a7200001aa8000901080008058780001aa88005b
:10a7300022aa8000e0a9800000004100808f500024
:10a740000100390002aa8800c0a98000d1a98000b8
:10a7500061004000e0804800c0a98800d1a98800bd
:10a760003e35ec00d9ff370040a9800051a9800098
:10a7700061004000e080480040a9880051a988009d
:10a780003295a800d3ff3700809fbe00829fbe0095
:10a79000841f7800d4c2bf000080fb004700de00a9
:10a7a0000082fb00d4e2a9008720a90000ac800051
:10a7b00011ac800061004000e080480000ac8800df
:10a7c00011ac88008a15e2001500320043ac80000d
:10a7d00082ac80001922ab000f003a0070ac800000
:10a7e000b080fb00d110880070ac8800830041006d
:10a7f000810f50000100390072ac880020ac80004d
:10a8000031ac800061004000e080480020ac88004e
:10a8100031ac88008a35ed008a15e200edff3a0080
:10a82000c720dd00d4c2bf000074a1000140700049
:10a83000d4e2b7004f0278004f01be004f00be00c7
:10a8400000400600809fbe00829fbe00d482a80008
:10a85000d4c2bf000080fb004700de008081fb0007
:10a86000d4e2a9008700a90070ab800081ab800012
:10a8700061004000e080480070ab880081ab880038
:10a880001822ab0007003200d0aa8000e1aa8000a5
:10a8900061004000e0804800d0aa8800e1aa88005a
:10a8a0006c35a8001802ab000c0032001842ab0057
:10a8b000170032006c55a800f0aa800001ab8000a0
:10a8c00061004000e0804800f0aa880001ab8800e9
:10a8d000e01080001802ab00f4ff3a001822ab0031
:10a8e000020032001822a9006c35a900c718dd004b
:10a8f000d4c2bf000074a10001407000d4e2b700d0
:10a90000d482a9004f01be004f00be0000400600e7
:10a910006c55a900c1ab8000b0ab8000808f5000a7
:10a92000130031006c95a900d1ab8000e0108000cd
:10a9300080587800d1ab8800f2ab8000b0ab8000cb
:10a9400000004100808f500001003900d2ab880028
:10a9500090ab8000a1ab800061004000e080480027
:10a9600090ab8800a1ab88007835ec00d9ff3700a8
:10a9700010ab800021ab800061004000e080480007
:10a9800010ab880021ab88006c95a800d3ff37007e
:10a990000001be000000e900e10f50000a003e0087
:10a9a000a00320000010b800824f210002004000e8
:10a9b000030178000200a0001000610011002000d7
:10a9c000820f5000010032008000eb00010078008f
:10a9d00000000600889fbe008a9fbe008c9fbe00bc
:10a9e000000678000205be000000e900e10f5000fb
:10a9f00058003e000a01be00e206b1000380b1002b
:10aa000020192c0011002000800f5100818f590067
:10aa10003f003e0022bd800033bd80006a10b800b8
:10aa20006a19b900828040007051b800705ab900ac
:10aa3000848141006a280200000000000004be007a
:10aa4000a2002000030020008e2102000000000070
:10aa50001dc0b300e40f5000e08f580001003e001d
:10aa60008046eb00a2002000030020000800be008a
:10aa70006a280200000000000d81fb000001410077
:10aa80008201e900a00320000060b800244f2100eb
:10aa9000040140000a89be00624f2100020040000c
:10aaa00003087800e10f560014003200e20f560050
:10aab00009003a00b01080001622ef00f310880061
:10aac000b01088000000eb004f06be004f05be002e
:10aad0004f04be00000006008c1f7800e42f2a00ff
:10aae000841f780000042000a689020000000000f6
:10aaf0000080eb00e4875700f3ff37006010800010
:10ab00000c22ef00a310880060108800edff3700d2
:10ab10008a9fbe0074332a00841f7800200420001e
:10ab2000a6890200000000000a0378002505200025
:10ab30002404200033052000a2372a0001562000fb
:10ab400090bd29004089020000000000e687570000
:10ab5000b0ff37008c1f780020002000801f780095
:10ab600082382a00821f780010042000a689020083
:10ab7000000000000c0378002505200014042000cc
:10ab800033052000a2372a00c155200090bd2900be
:10ab90004089020000000000e687570095ff37005b
:10aba000889fbe0000047800814478000000e9001e
:10abb000e10f50001d003e00010420000800780055
:10abc00073ff07000000e00007003200a003200030
:10abd0000040b800e251210002004000094878001e
:10abe0004f04be0000000600881f7800b03c2a0019
:10abf000801f780040042000a689020000000000a9
:10ac000008037800d5042000440420003305200008
:10ac100072402a00213e200090bd29004089020098
:10ac200000000000e4875700e8ff3700881f780025
:10ac300020002000801f7800a2412a00821f780097
:10ac400010042000a689020000000000080378001c
:10ac500025052000140420003305200072402a003e
:10ac6000d13d200090bd2900408902000000000075
:10ac7000e6875700d0ff37002c08e20021003200a1
:10ac80002240800033408000c0122000801f7800e6
:10ac900027cd210006202000259d210064002000f2
:10aca0003100200010002000fefb07008f87e90024
:10acb0000000e00001003a00000006001000200043
:10acc000801f780020462a00801f78005004200052
:10acd000a68902000000000016002000d504200014
:10ace000540420003305200002492a00b1542000fa
:10acf00090bd29004089020000000000e487570051
:10ad0000edff37000240800013408000deff370077
:10ad10000c00fa00889fbe008a1f7800d4a2a80009
:10ad20008025200001002000f0b79f0081bf9f0018
:10ad3000a1b880000810200001005400e10f50006d
:10ad40006d0034000005eb0001015400e30c22000b
:10ad500083804000f2815700100020009a490200d1
:10ad6000000000000000e00010003c000c00350076
:10ad7000a4492a00841f780000322000a68902001e
:10ad8000000000008f87e900d4a2a9000a00780023
:10ad90004f0578004f04be000080fa000000060056
:10ada0001437b5000085eb00f7ff37001437b40007
:10adb0001a002000765a02000000000090bf9f0099
:10adc000a1bf9f00b2bf9f00c3bf9f00e46e2100e0
:10add000009abe000292be00e8bb8000f9bb800072
:10ade0000800be00841f020000000000e00f5400b5
:10adf000e08f5c003a0035000002be000203be0096
:10ae00001fb89700afb897003fb99700cfb9970028
:10ae10008a1f0200000000009421020000000000d0
:10ae2000b0b88800c1b88800a0b88000b20c220079
:10ae3000820040001437ef008001eb000100780031
:10ae4000e40c2200848f50000600390042c2b30097
:10ae5000904f1100200032000000e900840f5000e4
:10ae6000fbff31000300e00013003200838050003c
:10ae70008100e800626f2100030078009c910200cd
:10ae800000000000000478000000e000beff320077
:10ae9000e30f400006003200544b2a00841f780064
:10aea000f0322000a6890200000000008f87e90030
:10aeb0000885e900b4ff3700e34d2a00831f7800be
:10aec000e0322000a6890200000000001437ef00e5
:10aed000eaff2f00abff370080017800e1ff370069
:10aee0006022b80006002000071f24008a2002000c
:10aef00000000000c0ff370040512a00801f78008a
:10af000040332000a6890200000000008000eb0012
:10af10001437ef008f87e9008aff370080408000f8
:10af200091408000b0b78800c1b78800a040800081
:10af3000b1408000d0b78800e1b78800000006006b
:10af40000800fa00889fbe008a1f78000004be0037
:10af5000020578008457e2004e0032000a00e0004b
:10af600032003a0011c1bf000078a3000300320094
:10af7000d4e2a8000140fe00d4e2a900765a020003
:10af800000000000a87821003802be002803be009f
:10af9000ec210200000000006022b800060024003e
:10afa000f7082400f02102000000000090bf9f007d
:10afb000a1bf9f00b2bf9f00c3bf9f00e8bb80003e
:10afc000f9bb80000800be00841f020000000000e2
:10afd000e00f5400e08f5c000e0035000002be0060
:10afe0000203be001fb89700afb897003fb99700a3
:10aff000cfb997008a1f02000000000094210200d0
:10b00000000000004f0578004f04be000080fa00e9
:10b01000000006006022b80006002000071f240080
:10b020008a20020000000000ecff37000800be008c
:10b03000280007000000e00006003a00765a0200ef
:10b0400000000000a8782100009cbe000294be0011
:10b05000caff3700e4532a00841f780060192000db
:10b06000a6890200000000000003eb00d5042000c8
:10b07000641920003304200082552a00a104200016
:10b08000d0552a0040890200000000008f87e900a7
:10b09000eaff370050562a00801f78005019200020
:10b0a000a6890200000000000003eb00d504200088
:10b0b000541920003304200082552a00e1032000a7
:10b0c000d0552a0040890200000000008f87e90067
:10b0d000a2ff3700889fbe000004be008457e20034
:10b0e00039003200e00f5400e08f5c00260034008d
:10b0f00011c1bf000078a30003003a0084d7bf004d
:10b100000018a3000f003200c0582a00801f7800ea
:10b11000a0192000a6890200000000000003eb0037
:10b12000d5042000a419200033042000825b2a00eb
:10b1300061092000d0552a0040890200000000006b
:10b140008f87e9000821ef000621ef0004bc800092
:10b1500015bc80000821b80009a0b900008041009a
:10b1600005c2b900840140006208880073088800a5
:10b1700011e1a80030c0b30084f7b7000000eb0075
:10b180004f04be0000000600205c2a00801f7800eb
:10b1900050192000a6890200000000000003eb0007
:10b1a000650520009419200033042000825b2a00ea
:10b1b00001092000d0552a0040890200000000004b
:10b1c0008f87e900caff3700b05e2a00801f780031
:10b1d00090192000a6890200000000000003eb0087
:10b1e000d50420009419200033042000825b2a003b
:10b1f000b1082000d0552a0040890200000000005c
:10b200008f87e900b7ff3700809fbe00829fbe0096
:10b2100011e1a900d4c2bf000080fb004700de009e
:10b22000d4e2a90084e0a90032bc800043bc8000c5
:10b2300061014100e081490032bc880043bc8800c4
:10b2400051c0b3008000fd0084f7b7008000fd000e
:10b250004700dd00412d2000914078000174a100dd
:10b2600080c0700001007800d4e2b7004f01be003a
:10b270004f00be0000400600889fbe000004be00d4
:10b280008457e200200032000800be0091ff070052
:10b290000000e0000c003a0011c1bf000078a300dc
:10b2a00006003200d4e2a8000140fe00d4e2a9006a
:10b2b00011c1bf000078a300faff3a000000eb00c4
:10b2c0004f04be000000060070612a00801f780055
:10b2d00080192000a6890200000000000003eb0096
:10b2e000d50420008419200033042000f2632a00d2
:10b2f00061072000d0552a004089020000000000ac
:10b300008f87e900e4ff370050642a00801f78002f
:10b3100070192000a6890200000000000003eb0065
:10b32000d50420007419200033042000f2632a00a1
:10b33000c1062000d0552a0040890200000000000c
:10b340008f87e900d0ff370011e1a9000821ef0045
:10b350000621ef000e21ef007008800060088800d1
:10b3600050c0b30084f7b700000005001221ef00c1
:10b3700090088000800888000821ef000621ef0077
:10b380000e21ef00700880006008880080cfb300b5
:10b390009760b60097c0bf00f1c8b30001406000dd
:10b3a0000054a00097e0b7008cc0a9008ce0a80072
:10b3b00084c0a90084e0a9001061a80011a1a9001f
:10b3c000f0ccb3001061b60050c0b30084f7b700f2
:10b3d0000000060000002000211c200020bd880085
:10b3e00031bd8800e0bb8800f1bb88003033270006
:10b3f0000100200040bd880051bd880000bc8800cd
:10b4000011bc8800300a200060bd8800ae37ef0014
:10b41000000037002021ef0000098000f0088800bc
:10b420001621ef001421ef001c21ef00e00880003e
:10b43000d0088800f0c8b3009e60b6009fc0bf006f
:10b4400081cfb300014060000014a0009fe0b7006e
:10b450008ea0a9008ec0a80086a0a90086c0a90061
:10b460001e61a8001fa1a900f0ccb3001e61b600a8
:10b470000080eb00d0088800e00888001fe1a800e9
:10b4800030c0b300b2f7b7000000060086c0a900c4
:10b49000b037ec0000400600b257e200090032006d
:10b4a000a008800001002000b208800003002000f6
:10b4b000c011dd00020020000200700083807000d7
:10b4c000000006000003eb00d50420003413200028
:10b4d00033042000e2662a00d109200050672a00c8
:10b4e0004089020000000000edff37000800fa006c
:10b4f000889fbe008a1f7800b257e20048003200e1
:10b5000042c0bf000080fb004505de000a00780055
:10b51000baf7b70000ceb3004260b700a8088000b9
:10b5200009002000b008800001002000c000dd00fc
:10b530000000200000047400818474000800be0034
:10b54000841f02000000000090bf9f00a1bf9f0069
:10b55000b2bf9f00c3bf9f00e00f5400e08f5c00ac
:10b560002500350088bd80006140b900841f0200bd
:10b57000000000000800e000190035006022b8005b
:10b5800006002000071f2400f02102000000000038
:10b590000002be000203be001fb89700afb89700bc
:10b5a0003fb99700cfb997008a2002000000000041
:10b5b000c552dd0024042000144278007f4262005e
:10b5c000054272000002fd0042e0b7000002fd00eb
:10b5d0004f0578004f04be000080fa00000006000e
:10b5e0006022b80006002000070f24008a20020015
:10b5f00000000000e1ff37006022b80006002000d4
:10b60000071f24008a2002000000000090bf9f0056
:10b61000a1bf9f00b2bf9f00c3bf9f00d1ff3700f3
:10b620000003eb00d5042000341320003304200075
:10b63000d2672a00310b200050672a00408902009f
:10b6400000000000aeff37003c00fa00889fbe00fb
:10b650008a9fbe008c9fbe002c08e2007608320054
:10b660002040800031408000809fbe0080d82b00a9
:10b67000801f7800608a020000000000e687570003
:10b680001848e2000600320071d92b0080812000aa
:10b6900092440200000000000000e00064083a004c
:10b6a000e1d92b00811f7800608a020000000000b1
:10b6b00010c0b3001aefb7008f87e90082002000a6
:10b6c000e1dd2b0010002000c24c02000000000051
:10b6d0000e007800180009000018eb008001eb0054
:10b6e000220320008e007800100020009a490200fa
:10b6f00000000000a0c0b3002077980012002000d6
:10b70000210320008e80400002007800c24c02001d
:10b71000000000000e0478001e4078000004e000e5
:10b7200005003200e84f50002408320058407800ed
:10b730000004e000fbff3a000e047800f9c3b300f8
:10b74000184078000004e0000a0032000080fb008e
:10b7500088010200000000000000e00015083a0027
:10b7600018407800894f5000020032000804e800b9
:10b77000f3ff3700ed4f5000c1ff32000004e0003e
:10b78000bfff32000045eb000000eb00501f9800a7
:10b79000201f9800330320008e81410042032000c7
:10b7a0000e014100a13a2b0008007800e04402009d
:10b7b00000000000000478000000e000b0ff32004c
:10b7c0002e189000080050008004e900de18900058
:10b7d000311f98008000eb00680ab80082c02b007f
:10b7e0000202420009017800880078001400780005
:10b7f00030440200000000000000e000eb073a00c7
:10b800000a45e8003e1990006810b80083c02b007c
:10b8100083014000531f98000201e800321f980086
:10b8200082007800f0022000800f5100eaff36000d
:10b830000a04e000d7073200e14f5500cf073c0073
:10b840000040eb00007f98002e1c9000de18900056
:10b85000314090000081fb0003002000c103200064
:10b86000810f5100e08f5900b6073e0002600100d1
:10b8700094003700b3073700c000370006013700d7
:10b8800043013700af0737007c01370081013700e3
:10b89000ac073700af013700fe0137003e0237002a
:10b8a000a7023700dd0237000c0337004c033700d6
:10b8b00075033700ac033700e30337001804370083
:10b8c0004f04370084043700bf043700e604370014
:10b8d000e8043700ea043700f0043700f8043700c2
:10b8e0009807370097073700960737009507370006
:10b8f0002a053700930737005e05370094053700a7
:10b90000c705370044063700750637009406370030
:10b91000cf06370001073700130737001100370043
:10b92000210737002407370027073700340737007f
:10b93000650137004a0737004c0737008107370099
:10b94000800737007f0737007e0737007d07370005
:10b950007c0737007b0737007a0737007907370005
:10b960007d073700330320008e8141004203200011
:10b970000e014100a13a2b0008007800e0440200cb
:10b980000000000072982b000000e000420032002e
:10b990000001eb00410320008e80400026050200dc
:10b9a000000000000005be002e18900090407800b6
:10b9b00060c6b30080cf50002600320060c4b300e0
:10b9c00080cf5000230032006a4088007b4088000e
:10b9d0008a9fbe0070de2b00801f7800c1df2b0025
:10b9e000811f7800608a020000000000e88757008d
:10b9f000f4072000f30f200042002000c180200047
:10ba0000c0002f00a4ab0200000000009475ef00fe
:10ba10000e7890000004e00019ff3200de1890005c
:10ba2000b1009000811f78005e1990002201900003
:10ba3000821f7800de199000931f7800a0e02b0091
:10ba4000801f7800608a020000000000e88757002d
:10ba50000bff37000a00be009a1e02000000000023
:10ba600052b82e0013052400202b02000000000015
:10ba7000da22020000000000604088007140880067
:10ba80008a9fbe0072de2b00821f780063e22b00cb
:10ba9000831f7800d3ff3700821f7800de199000e3
:10baa000931f780020e32b00801f7800608a02003b
:10bab0000000000011c0b300017f9800e687570026
:10bac000d2ff370040c4b300b4f7b7003a8f02008a
:10bad0000000000080c4b300b4f7b700214280002a
:10bae00040be8000808f500011003200801f78001f
:10baf000811f7800e2e52b00821f7800d00e200025
:10bb0000a68902000000000046be800065052000f6
:10bb1000d40e200023052000c2ea2b00e11f2000e4
:10bb200090eb2b004089020000000000e6875700e0
:10bb3000f4072000f30f200082382000018020004d
:10bb400000002f00a4ab020000000000e48b020004
:10bb500000000000f4072000f30f200082342000d2
:10bb6000c1f1200080382f00a4ab020000000000cb
:10bb70008e57020000000000a4ff370033032000ae
:10bb80008e814100420320000e014100a13a2b00aa
:10bb900008007800e0440200000000000000e0001f
:10bba00021003200a20020008000eb009c01020076
:10bbb000000000000005be000001be00e206b1006a
:10bbc0000380b10020192c0011002000800f5100cb
:10bbd000818f59000b0036008a9fbe00de1990004d
:10bbe000931f780000ec2b00801f7800608a020011
:10bbf0000000000011c0b300017f9800e8875700e3
:10bc000082ff37002a4088003b408800f40720006c
:10bc1000f30f2000420020004180200040002f0050
:10bc2000a4ab0200000000004240800053408000ae
:10bc3000829fbe002040800031408000809fbe0077
:10bc400061ee2b00811f7800608a02000000000076
:10bc5000224080003340800010002000ea5402009f
:10bc600000000000007d200001002000fc9b02007d
:10bc70000000000070c4b300b4f7b700ea875700b3
:10bc80000000eb004f06be004f05be004f04be0093
:10bc90000080fa0000000600330320008e8141007e
:10bca000420320000e014100a13a2b000800780059
:10bcb000e0440200000000000000e0002500320027
:10bcc000a20020008000eb009c01020000000000a8
:10bcd0000005be000001be00e206b1000380b10015
:10bce00020192c0011002000800f5100818f590075
:10bcf0000a0036008a9fbe005e199000921f7800ed
:10bd000003ec2b00831f7800608a02000000000013
:10bd100010c0b300007f9800b8ff37004a40880089
:10bd20005b408800f4072000f30f20004200200051
:10bd30008180200080002f00a4ab020000000000e2
:10bd4000424080005340800020002000ea5402005e
:10bd5000000000004240800053408000829fbe00ef
:10bd600063f32b00831f7800608a0200000000004c
:10bd7000d0c4b300b4f7b700007d2000010020005c
:10bd8000fc9b020000000000e6875700bcff370064
:10bd9000330320008e814100420320000e01410048
:10bda000a13a2b0008007800e044020000000000e7
:10bdb0000000e00020003200a20020008000eb0024
:10bdc0009c010200000000000005be000001be0052
:10bdd000e206b1000380b10020192c001100200000
:10bde000800f5100818f59000a0036008a9fbe00e3
:10bdf0005e189000901f780001ec2b00811f7800e6
:10be0000608a02000000000012c0b300027f9800a8
:10be10007aff37000a4088001b408800f4072000a2
:10be2000f30f2000420020000180200000002f00be
:10be3000a4ab020000000000004080001140800020
:10be4000809fbe00c1f62b00811f7800608a02002f
:10be500000000000803e200001002000fc9b02004a
:10be6000000000000240800013408000100020000d
:10be7000ea5402000000000010ff3700404080003c
:10be800051408000809fbe0061f32b00811f78002d
:10be9000b5ff3700f2012000b1f82b0010002000a0
:10bea000c24c020000000000007d200001002000c4
:10beb000fc9b0200000000001000200070510200f6
:10bec000000000000000fe000800780072a80200d8
:10bed000000000000000e0000300320011c0b300c9
:10bee000017f9800c9fe3700f4072000f30f2000ff
:10bef00022002000c18b2000c00b2f00a4ab020049
:10bf000000000000f4072000f30f200022002000b2
:10bf1000e18b2000e00b2f00a4ab0200000000002a
:10bf2000f4072000f30f2000020c2000018c2000f9
:10bf3000000c2f00a4ab020000000000f40720005a
:10bf4000f30f2000822020000198200000182f000d
:10bf5000acfe3700330320008e81410042032000f5
:10bf60000e014100a13a2b0008007800e0440200d5
:10bf70000000000000047800b3fa2b000000e0008d
:10bf80003a0032008e04020000000000301f9800ca
:10bf9000e60f50002e003c000001e900321f98001f
:10bfa000820478001f003b00880078008081200018
:10bfb000b805020000000000f4072000f30f200085
:10bfc000820020008181200080012f00a4ab0200ac
:10bfd000000000002008f80083812000831f780003
:10bfe00050fb2b00801f780090b8200060060200f4
:10bff0000000000090b820008e0402000000000045
:10c0000093ebb70081812000811f7800b2fb2b00e9
:10c01000821f7800608a020000000000ea87570053
:10c020007afe370068c07c000080fb00c205020079
:10c030000000000000f47c003e1890000001e900c0
:10c04000321f980082047800f6ff3b00d6ff3700cd
:10c05000881f780063002000831f78005e1890001e
:10c06000901f7800c1fd2b0064ff3700831f78000c
:10c070005e189000901f780021e32b00811f78004c
:10c08000608a02000000000012c0b300027f980026
:10c090008afe3700330320008e81410042032000d6
:10c0a0000e014100a13a2b0008007800e044020094
:10c0b000000000000004780003502b000000e000a6
:10c0c000eaff32001080fb00d005020000000000f3
:10c0d0000000e00005003a00881f7800de1990009b
:10c0e000931f780030012c006ffe37000001eb0039
:10c0f0008000eb0008007800260502000000000028
:10c10000ef0f5000e08f58000a003600881f7800bb
:10c110005e199000921f780033012c00831f780075
:10c12000608a02000000000010c0b300007f980089
:10c1300062fe37006f00600000418800f4072000b5
:10c14000f30f2000220020000182200000022f00b7
:10c15000a4ab0200000000002008f800818120004c
:10c16000811f780052fb2b00821f780090b82000be
:10c17000600602000000000090b820008e0402005b
:10c180000000000093ebb7002008f80063042c00c7
:10c19000831f78009fff3700330320008e8141000a
:10c1a000420320000e014100a13a2b000800780054
:10c1b000e044020000000000000478000000e000fd
:10c1c0005d003200dc390200000000000006be0005
:10c1d000f2ff2f00f3f72700801f0200000000008d
:10c1e0000000e0000c003a00881f7800c0942b008b
:10c1f000801f7800de189000911f780022062c0026
:10c20000821f7800608a02000000000013c0b300a3
:10c21000037f980079fe37002e189000330320002a
:10c220008e814100420320000e014100a13a2b0003
:10c23000e044020000000000000478000000e0007c
:10c2400032003200dc390200000000000005be00b0
:10c25000f2ff2f00f3f72700801f0200000000000c
:10c260000000e00003003a00881f7800b0962b0021
:10c27000dfff37008c4088009d408800aa4088007e
:10c28000bb408800f4072000f30f2000420020008c
:10c290000181200000012f00a4ab0200000000007b
:10c2a000f4072000f30f200042002000418120000d
:10c2b00040012f00a4ab0200000000008e570200d6
:10c2c00000000000a0408000b14080005c1e020021
:10c2d00000000000809fbe00829fbe008040800062
:10c2e000914080005c1e020000000000809fbe00a4
:10c2f000829fbe0050082c00801f7800608a0200d8
:10c3000000000000f2875700c0fd3700b0962b00f8
:10c31000801f7800de189000911f780022e32b0028
:10c32000821f7800608a02000000000013c0b30082
:10c33000037f9800e1fd370090902b00f4ff370059
:10c34000330320008e814100420320000e01410092
:10c35000a13a2b0008007800e04402000000000031
:10c36000000478000000e00026003200dc39020002
:10c37000000000000006be00f2ff2f00f3f72700c8
:10c38000801f0200000000000000e00007003a00eb
:10c39000881f7800c1942b00811f78005e199000df
:10c3a000921f780023062c0056fe37008c40880030
:10c3b0009d408800f4072000f30f20004200200079
:10c3c0000181200000012f00a4ab0200000000004a
:10c3d0008e570200000000008040800091408000e5
:10c3e0005c1e020000000000809fbe00829fbe0015
:10c3f000d10a2c00811f7800608a02000000000032
:10c4000006ff3700c1942b00811f78005e19900051
:10c41000921f780023e32b0040ff370033032000f6
:10c420008e814100420320000e014100a13a2b0001
:10c4300008007800e04402000000000000047800da
:10c44000b3962b000000e00008ff3200dc39020048
:10c45000000000000005be00f2ff2f00f3f72700e8
:10c46000801f0200000000000000e00007003a000a
:10c47000881f7800b3962b00831f78005e18900009
:10c48000901f780021062c005cfe3700aa4088002f
:10c49000bb408800f4072000f30f2000420020007a
:10c4a0004181200040012f00a4ab020000000000e9
:10c4b0008e57020000000000a0408000b1408000c4
:10c4c0005c1e020000000000809fbe00829fbe0034
:10c4d000930c2c00831f7800c7ff37003303200024
:10c4e0008e814100420320000e014100a13a2b0041
:10c4f00008007800e0440200000000000000e000b6
:10c5000035003200a20020008000eb009c010200f8
:10c51000000000006105b90061005500e0805d0089
:10c52000e50f5000e08f58001f003e0022418000c0
:10c530006110b800800f5500818f5d000b00340042
:10c54000821f78008a9fbe00de199000931f78003a
:10c55000500e2c00801f7800608a0200000000004e
:10c5600011c0b300017f9800acfe37001a4188006b
:10c57000f4072000f30f2000220020002182200079
:10c5800020022f00a4ab0200000000002208f800e7
:10c5900062112c00821f7800608a020000000000f7
:10c5a000e487570019fd37008a9fbe006300200012
:10c5b000831f78005e189000901f7800e1122c0015
:10c5c000811f7800608a02000000000012c0b300e2
:10c5d000027f980091fe3700f3152c00a3fe370070
:10c5e000330320008e814100420320000e014100f0
:10c5f000a13a2b0008007800e0440200000000008f
:10c600000000e000f4ff3200a20020008000eb00f8
:10c610009c010200000000006105b90061005500a6
:10c62000e0805d00e50f5000e08f5800deff3e0027
:10c63000124180006110b800800f5500818f5d00ad
:10c6400006003d00821f78008a9fbe00de19900020
:10c65000931f780010162c00beff37002a41880077
:10c66000f4072000f30f2000220020004182200068
:10c6700040022f00a4ab0200000000002408f800d4
:10c6800002192c00c3ff3700330320008e814100c4
:10c69000420320000e014100a13a2b00080078005f
:10c6a000e0440200000000000000e0002c00320026
:10c6b0009040780090c7b30080cf50002300320034
:10c6c00090c5b30080cf50002000320010c3b300eb
:10c6d00080cf50001d00320040c7b30080cf500013
:10c6e0001a00320040c5b30080cf5000170032005e
:10c6f0007140400080cf50001400320050c4b3009d
:10c7000080cf5000110032003628ef0032002000a8
:10c71000a11a2c0010002000c24c020000000000f2
:10c7200052012000e11a2c0010002000c24c02002f
:10c7300000000000f4072000f30f2000220020007a
:10c740006183200060032f00aefc37001200200040
:10c75000b241880022002000411c2c00edff370070
:10c7600092402b00ccfc3700330320008e81410027
:10c77000420320000e014100a13a2b00080078007e
:10c78000e0440200000000000000e0002c00320045
:10c790009040780090c7b30080cf50002300320053
:10c7a00090c5b30080cf50002000320010c3b3000a
:10c7b00080cf50001d00320040c7b30080cf500032
:10c7c0001a00320040c5b30080cf5000170032007d
:10c7d0007140400080cf50001400320050c4b300bc
:10c7e00080cf5000110032003828ef0032002000c6
:10c7f000a11a2c0010002000c24c02000000000012
:10c80000b2012000711c2c0010002000c24c02005c
:10c8100000000000f4072000f30f20002200200099
:10c820008183200080032f0076fc37001300200056
:10c83000c341880022002000411c2c00edff37007e
:10c8400093402b0009fe3700330320008e81410006
:10c85000420320000e014100a13a2b00080078009d
:10c86000e0440200000000000000e000bcff3200d5
:10c870009040780090c7b30080cf50002300320072
:10c8800090c5b30080cf50002000320010c3b30029
:10c8900080cf50001d00320040c7b30080cf500051
:10c8a0001a00320040c5b30080cf5000170032009c
:10c8b0007140400080cf50001400320050c4b300db
:10c8c00080cf5000110032003a28ef0032002000e3
:10c8d000a11a2c0010002000c24c02000000000031
:10c8e000a2012000311e2c0010002000c24c0200ca
:10c8f00000000000f4072000f30f200022002000b9
:10c90000a1832000a0032f003efc3700120020006e
:10c91000d241880022002000411c2c00edff37008e
:10c92000330320008e814100420320000e014100ac
:10c93000a13a2b0008007800e0440200000000004b
:10c940000000e0002c0032009040780090c7b30057
:10c9500080cf50002300320090c5b30080cf50003c
:10c960002000320010c3b30080cf50001d00320001
:10c9700040c7b30080cf50001a00320040c5b3005a
:10c9800080cf5000170032007140400080cf50002f
:10c990001400320050c4b30080cf500011003200a8
:10c9a0002628ef0032002000a11a2c0010002000e1
:10c9b000c24c02000000000022012000e11f2c00f8
:10c9c00010002000c24c020000000000f40720000c
:10c9d000f30f2000220020006182200060022f005f
:10c9e00008fc3700100020003041880022002000a1
:10c9f000411c2c00eeff370090402b0044fe370016
:10ca0000330320008e814100420320000e014100cb
:10ca1000a13a2b0008007800e0440200000000006a
:10ca20000000e00086ff32009040780090c7b3001d
:10ca300080cf50002300320090c5b30080cf50005b
:10ca40002000320010c3b30080cf50001d00320020
:10ca500040c7b30080cf50001a00320040c5b30079
:10ca600080cf5000170032007140400080cf50004e
:10ca70001400320050c4b30080cf500011003200c7
:10ca80002a28ef0032002000a11a2c0010002000fc
:10ca9000c24c0200000000009201200011212c0075
:10caa00010002000c24c020000000000f40720002b
:10cab000f30f200022002000a1822000a0022f00fe
:10cac000d0fb3700130020005341880022002000d3
:10cad000411c2c00edff3700330320008e81410004
:10cae000420320000e014100a13a2b00080078000b
:10caf000e0440200000000000000e00018ff3200e7
:10cb00009040780090c7b30080cf500029003200d9
:10cb100090c5b30080cf50002600320010c3b30090
:10cb200080cf50002300320040c7b30080cf5000b8
:10cb30002000320040c5b30080cf50001d003200fd
:10cb40007140400080cf50001a00320050c4b30042
:10cb500080cf50001700320000c7b30080cf5000d4
:10cb60001400320000c5b30080cf50001100320025
:10cb70003c28ef0032002000a11a2c0010002000f9
:10cb8000c24c02000000000082032000b1222c00f1
:10cb900010002000c24c020000000000f40720003a
:10cba000f30f200022002000c1832000c0032f00cb
:10cbb00094fb370012002000e24188002200200090
:10cbc000411c2c00edff370080c02b00501f980047
:10cbd00041262c00811f780002272c00821f78003c
:10cbe00053272c00831f7800d0272c00801f78004b
:10cbf000608a0200000000000001eb00321f980074
:10cc0000e8875700f8022000de18900021409000cd
:10cc10000004e00008003a00de199000e8814100bd
:10cc2000531f98000201e800321f9800880f51003e
:10cc3000f5ff360075fb370031019000821f780048
:10cc4000a1019000831f7800911f7800e1282c003b
:10cc5000811f7800608a020000000000e88757000a
:10cc60003e199000ecff3700c08d0200000000006c
:10cc700066fb37005a8502000000000063fb3700a6
:10cc80004428ef00c2052000112a2c0010002000cb
:10cc9000c24c020000000000f6ff370040682a0086
:10cca0008e040200000000000001780041682a00a4
:10ccb00010002000c24c02000000000053fb3700af
:10ccc000330320008e814100420320000e01410009
:10ccd000a13a2b0008007800e044020000000000a8
:10cce000000478000000e000d5fe320002022000bf
:10ccf000e12f2c0010002000c24c020000000000b8
:10cd00009840780090c7b30080cf50001e003200da
:10cd100090c5b30080cf50001b00320010c3b30099
:10cd200080cf50001800320040c7b30080cf5000c1
:10cd30001500320040c5b30080cf50001200320011
:10cd40007140400080cf50000f00320050c4b3004b
:10cd500080cf50000c0032002c28ef001201200080
:10cd6000f1312c0010002000c24c02000000000035
:10cd7000f4072000f30f200022002000c1822000d1
:10cd8000c0022f001ffb3700130020006341880002
:10cd90004200200011332c00f2ff37003303200043
:10cda0008e814100420320000e014100a13a2b0078
:10cdb00008007800e0440200000000000000e000ed
:10cdc00067fe32009040780090c7b30080cf5000db
:10cdd0002300320090c5b30080cf50002000320005
:10cde00010c3b30080cf50001d00320040c7b30015
:10cdf00080cf50001a00320040c5b30080cf5000f1
:10ce0000170032007140400080cf50001400320003
:10ce100050c4b30080cf5000110032003428ef001e
:10ce200032002000a11a2c0010002000c24c020089
:10ce300000000000b201200061332c00100020002f
:10ce4000c24c020000000000f4072000f30f200095
:10ce5000220020004183200040032f00e9fa370020
:10ce600012002000a241880022002000411c2c005a
:10ce7000edff3700330320008e8141004203200084
:10ce80000e014100a13a2b0008007800e0440200a6
:10ce9000000000000000e0002b0032000001eb0069
:10cea0008000eb0026050200000000000005be0027
:10ceb000401f2000800f5500e08f5d000c00360001
:10cec0008a9fbe00411f2000811f78005e199000dc
:10ced000921f780023352c00831f7800608a02009f
:10cee0000000000010c0b300007f98004bfc37002a
:10cef0007a418800f4072000f30f20002200200070
:10cf0000e1822000e0022f00a4ab0200000000003c
:10cf1000704180000000e00008003200801f7800af
:10cf200091382c00811f780032392c00821f780044
:10cf3000608a020000000000e0fa370002022000d0
:10cf4000613b2c005aff3700c0562b00f0fc370025
:10cf5000330320008e814100420320000e01410076
:10cf6000a13a2b0008007800e04402000000000015
:10cf7000c1562b000000e00023fd32000001eb0051
:10cf80008000eb002605020000000000e10f4000d9
:10cf9000e08f58000e003600809fbe00f2ff2f0089
:10cfa00003002000829fbe00de199000931f7800ce
:10cfb000703d2c00801f7800608a02000000000095
:10cfc00011c0b300017f9800ec8757008ffa37003b
:10cfd000f0418800f4072000f30f20002200200019
:10cfe000e1832000e0032f00a4ab0200000000005a
:10cff000f04180000000e00006003200801f780051
:10d00000f2402c00821f780033392c00831f7800f7
:10d01000c7ff3700b2012000f1412c0024ff370088
:10d02000330320008e814100420320000e014100a5
:10d03000a13a2b0008007800e04402000000000044
:10d0400000047800b1432c000000e000eefc320048
:10d05000608420001f0009000018eb00620020001f
:10d0600051442c0008007800304402000000000009
:10d070000000e0005a0032000001eb00321f98006f
:10d08000080078008e04020000000000e84f500005
:10d0900043003e008004eb000085fb00e00f15001c
:10d0a00008003d0068c07c000080fb00c205020053
:10d0b0000000000000f47c008904e8008a8f54001e
:10d0c000f8ff35003e1890006800b8006284200028
:10d0d000020040000a017800880078004404020041
:10d0e000000000002e189000330320008e814100c4
:10d0f000420320000e014100a13a2b00e04402004f
:10d1000000000000000478006e7590003e1890004a
:10d110000001e800321f9800e70f510002003c00b8
:10d120000800e000d6ff3a00e14f45000f00320052
:10d130000a40e80088ebb700f4072000f30f200056
:10d14000020420006184200060042f00a4ab0200d0
:10d150000000000088cbbf000080fb00801f78002b
:10d16000c1442c00811f78000bfd3700de199000b0
:10d17000931f780030472c00801f7800608a0200df
:10d1800000000000f30f20000204200061042f00c3
:10d1900060842000d6ac02000000000000fd3700d3
:10d1a00082002000821f7800881f78003e189000bf
:10d1b000801fe800de199000931f7800e0492c00e2
:10d1c000801f7800608a02000000000000c5eb00ac
:10d1d00011c0b300017f9800ea875700d2ff3700e3
:10d1e000886bef00f4072000f30f200002042000fa
:10d1f0006184200060042f00a4ab02000000000046
:10d20000614d2c00811f7800608a02000000000040
:10d210008f87e900fdf93700330320008e8141003c
:10d22000420320000e014100a13a2b0008007800c3
:10d23000e0440200000000000000e0002600320090
:10d240000001eb008000eb0026050200000000005a
:10d250000005be00e00f5000e08f580005003200ce
:10d260006a005000e0805800eb0f4000e08f58004b
:10d2700011003e008a418800f4072000f30f2000cf
:10d28000220020000183200000032f00a4ab020035
:10d2900000000000804180000000e0000300320038
:10d2a000801f7800324f2c0056ff3700720120009b
:10d2b000a14f2c007efe37008a9fbe00809feb00ae
:10d2c000a2002000821f7800de199000931f7800d2
:10d2d00020512c0037ff3700c2562b00eef93700e3
:10d2e000330320008e814100420320000e014100e3
:10d2f000d1542c0008007800e04402000000000037
:10d30000000478000000e000130032006088200074
:10d31000150009000018eb00b20220008800780018
:10d32000608820004404020000000000f407200090
:10d33000f30f2000c20220006188200060082f0047
:10d34000a4ab02000000000060882000801f78006d
:10d3500001552c0083ff370030572c00ecfb3700c1
:10d3600022582c000800e000cbf9320098407800e9
:10d37000f0c2b30080cf50000f003200c0c5b30030
:10d3800080cf50000c00320000cdb30000c0400040
:10d39000e94f500008003600f0c9b30000c040005b
:10d3a000e94f500004003600f0cbb30000c040004d
:10d3b000f94f500020003e0018419000f0cdb3001e
:10d3c00000404100d1c5b300814f50000600360037
:10d3d000e2582c00821f7800de199000931f78001d
:10d3e000005b2c00b0f937001880fb004800dd001e
:10d3f0008280fb000100700090418800f40720004b
:10d40000f30f2000220020002183200020032f00a2
:10d41000a4ab020000000000ae1890001140900084
:10d420000080fb00801f78001180fb00801f7800c7
:10d43000425d2c00bdfe3700135f2c00831f780077
:10d440005e189000901f7800015b2c000bfb3700ea
:10d45000330320008e814100420320000e01410071
:10d46000a13a2b0008007800e04402000000000010
:10d470000004780023622c000000e000fbfa320078
:10d480008e04020000000000301f9800e90f5000d9
:10d490001f003c000001e900321f98008204780060
:10d4a00010003b0088007800208b2000b8050200a7
:10d4b00000000000f4072000f30f2000a20020006d
:10d4c000218b2000200b2f00a4ab020000000000e5
:10d4d000238b2000831f780040632c00801f78007e
:10d4e0002dfc370068c07c000080fb00c2050200f4
:10d4f0000000000000f47c003e1890000001e900ec
:10d50000321f980082047800f6ff3b00e5ff3700e9
:10d51000881f780093002000cffa37000042800077
:10d520000080ea000042880051652c0001003a00aa
:10d5300081652c00811f7800c2652c00821f780055
:10d54000608a020000000000f4072000f30f2000b2
:10d55000220020000184200000042f00a4ab020060
:10d56000000000000efc370028a8ee00f4072000a1
:10d57000f30f2000220020008182200080022f0073
:10d58000a4ab0200000000002808e2000400320002
:10d5900000672c00801f780040672c00cfff370009
:10d5a000b0682c00fbff3700c0022000ae9b0200d9
:10d5b0000000000015f93700a1ea2d00811f780056
:10d5c000e2682c00f3fb3700080178005e18900039
:10d5d00090007800e0022000eaa1020000000000b4
:10d5e0000000e0003dfa3a00f4072000f30f2000ad
:10d5f00022002000c18b2000c00b2f0046fa37000c
:10d6000008017800de19900093007800f0022000f5
:10d61000eaa10200000000000000e0000300320068
:10d6200010c0b300007f9800f8f83700f40720001e
:10d63000f30f200022002000e18b2000e00b2f00e0
:10d64000a4ab020000000000f4072000f30f20004c
:10d65000020c2000018c2000000c2f00e9f837009c
:10d660001ca9020000000000e8f837003303200086
:10d670008e814100420320000e014100a13a2b009f
:10d6800008007800e0440200000000000004780078
:10d69000d3692c000000e00074fa3200904078005a
:10d6a00040c6b30080cf50001f00320040c4b3001a
:10d6b00080cf50001c00320000c7b30080cf500064
:10d6c0000900320000c5b30080cf500006003200d0
:10d6d000881f7800de199000931f7800906a2c0054
:10d6e000801f780012fe3700800020001042880062
:10d6f00000072000301f9800e2012000216d2c005f
:10d7000010002000c24c020000000000f4072000be
:10d71000f30f200022002000610320008e804000d3
:10d7200020042f00b7f83700400020001042880086
:10d7300042062000321f9800e2012000116f2c00e9
:10d74000efff37000080fb00801f780003712c0082
:10d75000831f780090fb3700b5d7bf0000c0ea00f8
:10d76000b5f7b70041732c0001003a0071732c002b
:10d77000811f7800b1732c007afe37008e1f78006d
:10d7800082742c00821f780023752c00831f780080
:10d79000b8f737008e1f780030762c00801f780095
:10d7a00021752c00811f7800b2f737003e199000d8
:10d7b00019f8370018407800eef737008e0f540044
:10d7c0000f0032000804e900281f98008800780044
:10d7d000184078000004e000d5f73200a141900025
:10d7e000834878002e1890008000e800211f9800e0
:10d7f0001104e000f9ff3a0018407800ccf7370038
:10d800008e0078002e1f98001e04e000faff320000
:10d8100011419000824878002e1890008000e800a6
:10d82000211f98001104e000f9ff3a00f2ff3700d1
:10d830001a6fef00a1f73700004080001140800010
:10d8400089f737008a01fa00889fbe0082162000ff
:10d85000e1df210020002000a40307000000e00019
:10d860005701340000be8800765a02000000000014
:10d870003e20020000000000e0bd8800f1bd8800ed
:10d8800001be800022e72f000f014100e0df2100f0
:10d890004f020700e17c2c00e30f5000d2003a0059
:10d8a000b557e20041013a004f809600f00f50005a
:10d8b00004003600af489500a0c3b30080cf5000ed
:10d8c000040132004008e200fb00320081812000a8
:10d8d00082e72f0002804700dc0502000000000004
:10d8e0000000e00006003a007ff894000000d1003c
:10d8f0006f00600001418000810f5000ec00320099
:10d9000020e72f000f0040009c9f02000000000055
:10d91000000478000000e000de003500b557e200aa
:10d92000060032000800e00004003400d17d2c0025
:10d9300020e72f000f0040003705070020e72f00e9
:10d940000f0040003e9c0200000000000000e000cc
:10d95000c4003a00765a020000000000a0bf9f00f9
:10d96000b1bf9f00c2bf9f00d3bf9f0028bd8000f2
:10d9700039bd80000800be00841f020000000000c6
:10d98000e00f5400e08f5c00b00035000002be00e4
:10d990000203be002fb89700bfb897004fb9970099
:10d9a000dfb997008a1f0200000000003e2002003d
:10d9b00000000000903f9e00a13f9e003e08e20054
:10d9c00096003a002e08e2000700320020e72f0000
:10d9d0000f004000bc8a020000000000d17e2c0035
:10d9e000e10f50008000320020e72f000f004000c0
:10d9f000d4790200000000000000e00002003200c4
:10da00003c08e20083003200ee80570020e72f0040
:10da10000f004000e48102000000000000047800d4
:10da2000e40f50006300320016003c00e20f50008b
:10da300008003e00f17f2c0020e72f000f0040007f
:10da4000590407000000eb004f04be000080fa00fc
:10da500000000600881f780010822c00801f7800cc
:10da6000608a020000000000e1852c00e0e62f0043
:10da70000f004000e80407000080eb00e487570037
:10da8000f1ff3700e80f5000f2ff3a002808e200eb
:10da90003c003a001fb89700e10f4000330032000d
:10daa000801fe8007c00b80062f32000e01f7900ce
:10dab00010882c00801f7800608a0200000000009f
:10dac000e6875700a1892c0020e72f000f004000b7
:10dad000350407008216200061f6210020e72f00a0
:10dae0000f004000c7000700800478000000e0003d
:10daf0001a0032000001780061f6210020002000a9
:10db0000b1020700890f50000e003a00b557e2003d
:10db100007003a003e08e200caff32008fb89700c3
:10db2000310090000000a000b0009800c5ff370051
:10db3000b1892c0020e72f000f004000b604070039
:10db4000f4ff3700801f7800728a2c00821f780053
:10db5000608a020000000000c7ff3700801feb0052
:10db6000d18b2c00811f7800f9ff3700628e2c00ca
:10db7000821f7800608a0200000000008f87e900a1
:10db8000d0ff370020e72f000f004000ab05070053
:10db90000000e000bfff3200c18f2c00811f780021
:10dba000a0042000a6890200000000008f87e90081
:10dbb000b8ff37001fb89700e10f40000f00320098
:10dbc000801fe8007c00b80062f32000e01f7900ad
:10dbd00070912c00801f7800608a02000000000015
:10dbe000e6875700a1892c0020e72f000f00400096
:10dbf000ed0307000080eb0093ff370000932c003b
:10dc0000801f7800608a0200000000008f87e90012
:10dc1000f4ff370061942c00f3ff3700f0805700c9
:10dc200020e72f000f004000449b0200000000008e
:10dc3000e10f500063ff3a009201200061962c0032
:10dc4000c24c020000000000e6ff37006022b8006e
:10dc500006002000071f24008a20020000000000a8
:10dc60004aff37000000d000a1342e00e09f78006a
:10dc700002982c00821f7800608a020000000000d9
:10dc8000a1892c00e0e62f000f004000c60307002a
:10dc900079ff3700801f780070992c00801f780072
:10dca000608a020000000000e48757001bff370075
:10dcb000519b2c00ccff3700719c2c00811f7800f9
:10dcc000608a0200000000000080eb008f87e900fe
:10dcd0005dff37004f509500814f5000f9fe3a002c
:10dce00032b92000124178000281fb00b0e82f0019
:10dcf0008080470090b8200000060200000000006d
:10dd00000000e000effe3a0082e72f00828047002b
:10dd1000208b2000dc050200000000000000e00075
:10dd2000e8fe3a0050e92f0000844700720020000e
:10dd3000819d2c00080078002606020000000000eb
:10dd40000000e0001500320072002000019e2c004f
:10dd50000800780026060200000000000000e00035
:10dd6000d8fe3a0040a8ef0032012000819e2c002e
:10dd700010002000c24c020000000000f407200048
:10dd8000f30f2000220020000184200000042f0057
:10dd9000a4ab020000000000cafe37004028ef00dc
:10dda00042012000c19f2c00f1ff370011a12c007f
:10ddb00020e72f000f00400017040700bafe3700cd
:10ddc0000000e00007003a00a0a12c00801f7800ae
:10ddd00000052000a6890200000000008f87e900ee
:10dde00084ff3700801f780001a32c00811f78007a
:10ddf00060042000a689020000000000e4875700ac
:10de00007cff37006801fa00889fbe008a9fbe0031
:10de10008004780081057800020578000000e000a9
:10de2000db0032000b00e000c900320010032000cc
:10de3000800f5500b500360004e92f000f024200a4
:10de40000004eb008002eb008000eb0002c4b30092
:10de500001804400604890000004e00001003a00a6
:10de6000150020000500e000a6003200024a7800fc
:10de70008100e8000402e8000804e800e58f500093
:10de8000f3ff340059509000005a78000804e8006d
:10de90008002eb008000eb0002c4b300018044006c
:10dea000604090000004e00001003a0015002000ee
:10deb0000500e00091003200024a78008100e8008d
:10dec0000402e8000804e800e58f5000f3ff340086
:10ded00059489000004a7800a9d892000104e00057
:10dee00002003a001404a000a9d892000402e8003d
:10def0000804e8008003eb000104e0002000320089
:10df00008002eb008000eb006839b80006c4b30063
:10df10000280400009004000205892000004e00008
:10df200001003a00150020000500e00071003200f9
:10df3000064a78008100e8000402e8000804e800ce
:10df4000e58f5000f2ff3400028044001060920020
:10df5000004a7800a9d892000180fb000000e90087
:10df6000808f5300600032008703e8000402e8005d
:10df70000804e8000180fb00808f5300e0ff3500bb
:10df800030c0b300005a780000cfb300005a7800c8
:10df90000884e80039099000020044006400400051
:10dfa0008a0f50004a003e00f880440004007800c8
:10dfb0001805020000000000390890000004440029
:10dfc0000b02780000ccb300005a7800005aeb0036
:10dfd0000001eb008000eb00e00f140010003d009a
:10dfe00080427800b3cdb300c6cdb300d7cdb30027
:10dff00009e92f008184440069c07f00854f5000eb
:10e0000026003200834f500012003200004a780090
:10e010008100e8000402e800888f5000f4ff35001a
:10e0200000ccb300005a78000200440063044000b2
:10e03000640040008a0f500001003e00004aeb00df
:10e04000080078004f05be004f04be000080fa00b3
:10e0500000000600005a78000201e80002004400b7
:10e06000640040008a0f500002003e00074a78001a
:10e07000e7ff3700801f78008a1f780069a42c0012
:10e08000891f780040052000a689020000000000da
:10e090000080eb00e6875700eaff3700035a78005c
:10e0a0000201e80002004400640040008a0f5000b2
:10e0b00002003e00064a7800d5ff3700801f780036
:10e0c0008a1f780060a42c00801f7800edff3700c5
:10e0d000801f78008a1f780069a42c00891f7800af
:10e0e00030052000e8ff37001404a000a9d89200f2
:10e0f0009dff3700004ad0008eff3700004ad00055
:10e100006eff3700004ad00059ff37008a1f7800a1
:10e1100040a92c00801f7800f0042000a68902008e
:10e12000000000000a03780065052000f4042000c8
:10e130004305200042ac2c00b125200040ad2c004e
:10e140004089020000000000e48757003aff3700d2
:10e15000a0ad2c00801f7800e0042000a6890200fa
:10e16000000000000003eb00e50420000502780039
:10e170004305200042ac2c007125200040ad2c004e
:10e1800040890200000000008f87e90027ff370068
:10e19000b0b02c00801f7800d0042000a6890200b7
:10e1a000000000000003eb00e5042000d404200080
:10e1b0004305200042ac2c003125200040ad2c004e
:10e1c00040890200000000008f87e90015ff37003a
:10e1d000889fbe008a9fbe008c9fbe008e1f780065
:10e1e0000004780001077800020578000000e000d4
:10e1f000e50032000a00e000d30032000e00e0002b
:10e20000c0003200220020006e0645008c04780019
:10e210000a007800be0009000018eb000884e8003e
:10e220008005eb008006eb000e00e0001d003200d0
:10e23000e30f5100970032004a003c00e10f51000b
:10e2400038003200e20f51002d003a008b05e80043
:10e25000e68f550020003400804ceb001840780019
:10e26000704698008005eb00660645008c04780037
:10e270007c4090000000d1006f00600010003a0068
:10e28000120020008d06e8000804e8008e8f56007a
:10e2900004003100e70f510002003200e80f510086
:10e2a000e3ff3a004af892000080fb004f07780035
:10e2b0004f06be004f05be004f04be000000060022
:10e2c000c0b32c00801f7800608a020000000000ac
:10e2d0008f87e900eaff37009840780000c4b30058
:10e2e00080cf5000040032000180fb000000d1000c
:10e2f000805c7800e3ff3700805ceb00e1ff3700d3
:10e30000821f7800b0b52c00801f7800d005200057
:10e31000a68902000000000010002000e4875700da
:10e32000e2ff37008b05e800e68f5500eaff340076
:10e33000804ceb0018407800704698008005eb0098
:10e340001880fb00420020000008a300cdff3a0027
:10e35000ac1120000a0646008c0478003200200030
:10e36000c8ff3700e50f510044003200e40f5100b0
:10e370002d003400e60f5100e1ff3a00984178008b
:10e3800000ccb30080cf5100240032000e00e90021
:10e39000808f560016003200ba089000f00f20005f
:10e3a000808f500006003e00835c78003a089000a1
:10e3b0000000e800300d98008b05e800b1ff370041
:10e3c000811fe80010b92c00801f78006006200033
:10e3d000a689020000000000804ceb0080c0b30062
:10e3e00040fd9a0082002000e4875700a5ff370017
:10e3f00080bd2c00801f780050062000a6890200f6
:10e4000000000000804ceb0080c0b30040fd9a008b
:10e41000820020008f87e9009aff3700804ceb00d4
:10e420007200200097ff37001840780020fd9a0006
:10e43000720020001880fb00e10060000d00320037
:10e440000018a30009003200c00ab20004003a001c
:10e4500030c0b30040fd9a005200200089ff370011
:10e4600020c0b30040fd9a0086ff370010c0b30003
:10e47000fcff370041fd9a0082ff3700184078000a
:10e4800030fd9a00f80445008005eb006200200092
:10e490007cff37008b05e800e68f55008eff3400c7
:10e4a000804ceb0018407800704698008005eb0027
:10e4b0002ad892000040e80020dd9a00e74f500083
:10e4c00008003e001880fb000008a3000200320094
:10e4d000420020006bff3700680646008c0478007d
:10e4e00068ff370080002000801f7800a0c12c004a
:10e4f000801f780090052000a6890200000000001f
:10e50000b6ff3700801feb0050c62c00801f78003c
:10e5100080052000a6890200000000000003eb0037
:10e52000650520008405200043052000d2c82c008a
:10e530006133200040ad2c00408902000000000043
:10e54000e48757002fff3700c0c92c00801f7800d8
:10e5500070052000a6890200000000000003eb0007
:10e56000e50420007405200043052000d2c82c00db
:10e570002133200040ad2c00408902000000000043
:10e580008f87e9001dff370090cc2c00801f78009a
:10e5900060052000a6890200000000000003eb00d7
:10e5a000e50420006405200043052000d2c82c00ab
:10e5b000e132200040ad2c00408902000000000044
:10e5c0008f87e9000bff3700889fbe008a1f780005
:10e5d0008004780001057800020478000000e9005a
:10e5e000e10f50002e003e000a00e0001c00320047
:10e5f0000800e00009003200080178008a00780075
:10e6000009007800c24c02000000000008007800f9
:10e610004f0578004f04be0000000600801feb008d
:10e6200050cf2c00801f780000062000a689020031
:10e63000000000000003eb00650520000406200038
:10e640004305200092d12c005141200040ad2c0008
:10e650004089020000000000e4875700e6ff370011
:10e6600040d22c00801f7800f0052000a68902000f
:10e67000000000000003eb00e5042000f40520008a
:10e680004305200092d12c001141200040ad2c0008
:10e6900040890200000000008f87e900d4ff3700a6
:10e6a000891f780020002000801f7800b0d42c0043
:10e6b000801f7800e0052000a6890200000000000d
:10e6c0000003eb0025052000e405200043052000a1
:10e6d00092d12c00d140200040ad2c004089020096
:10e6e00000000000e6875700bfff3700e4874700bf
:10e6f000889fbe008a9fbe008c9fbe008e1f780040
:10e700008005780081067800020578000000e900a5
:10e71000e10f50007d003e000d00e0006b00320074
:10e720000a00e000580032006044b8001ec0b30088
:10e730000cccb3008a8f54004e0031008001eb00f6
:10e7400012002000f08057000b0078001e4b0200e2
:10e7500000000000e10f500041003a00e10f5400ba
:10e76000280032000800e00022003200e20f5400ce
:10e7700017003a008ff09700d0cdb30080cf500043
:10e7800010003200c0cdb30080cf50000a0032002c
:10e79000180020000e04e000e6ff3a0009007800af
:10e7a0004f0778004f06be004f05be004f04be0065
:10e7b0004f00b100000006008cf67c008904e800e0
:10e7c000f3ff370000c0e90080f67c00fbff370054
:10e7d000881f7800c1d72c00811f780070062000a8
:10e7e000a6890200000000000080eb00e4875700cb
:10e7f000ebff37008ff097008ccf5000e5ff3a0019
:10e80000edff37008ff097008ccf500008003200ea
:10e81000b0cdb30080cf50000300320081f67c0001
:10e820008904e800dbff370028002000d9ff37000b
:10e83000e18f5400d7ff36008cf67c008904e80095
:10e840000047eb008a8f5400d2ff39008a1f7800fe
:10e85000b0db2c00801f780060062000e0ff37004e
:10e86000801f780041df2c00811f780050062000b7
:10e87000dbff37008a1f7800b0db2c00801f780098
:10e8800040062000d6ff3700801feb0071e22c000d
:10e89000811f780030062000a689020000000000d9
:10e8a0000003eb006505200034062000430520002e
:10e8b000b2e42c001144200040ad2c00408902003d
:10e8c00000000000e487570097ff370050e52c0058
:10e8d000801f780020062000a689020000000000aa
:10e8e0000003eb00e504200024062000430520007f
:10e8f000b2e42c00d143200040ad2c00408902003e
:10e90000000000008f87e90085ff37008b1f78002b
:10e9100020002000801f7800b1e72c00811f7800c4
:10e9200010062000a6890200000000000003eb0092
:10e93000250520001406200043052000b2e42c0029
:10e940009143200040ad2c004089020000000000ef
:10e95000e687570070ff37000200fa00889fbe006c
:10e960008a9fbe00800478000105780002047800c8
:10e97000417b21009140780070c4b30080cf5000eb
:10e9800041003200417b21009140780063405000fb
:10e9900080cf50003c003200010220001000200017
:10e9a000c8540200000000000000e0003600320001
:10e9b0000900e0006c0032000a00e000590032005b
:10e9c000a0c0b300e0f79f0012002000ea805700cb
:10e9d00002007800c24c0200000000000800e000c5
:10e9e000020032001804e00045003a000004eb0089
:10e9f0000a00e0001d003200bb0d200069417c00d0
:10ea00008280fb008b8f50003a0032002d003c00ca
:10ea1000000c2000808f5000270032000204e0002c
:10ea20001d0035000280fb000000d000e1272d0012
:10ea3000608078008e040200000000000001780071
:10ea400069407c000080fb000000d000e1272d0021
:10ea5000e080780010002000c24c0200000000009e
:10ea60000804e8008a0f5400e4ff3900ea805700e8
:10ea7000a0c0b30080687800120020000200780077
:10ea8000c24c0200000000004f05be004f04be0053
:10ea90000080fa00000006000280fb00801f780062
:10eaa000b0ea2c00801f7800608a0200000000009d
:10eab000e4875700eaff37004200200021eb2c00da
:10eac000e4ff3700c00d2000808f500006003200a8
:10ead0000000e800808f5000d0ff3a004200200084
:10eae00071eb2c00dbff370042002000c1eb2c0053
:10eaf000d8ff37004200200011ec2c00d5ff370072
:10eb0000080078008e040200000000000001780078
:10eb10008800780010002000c24c020000000000b5
:10eb2000b2ff3700801feb0061ec2c00811f7800e2
:10eb300090062000a6890200000000000003eb0000
:10eb400065052000940620004305200072ee2c008d
:10eb5000814c200040ad2c004089020000000000e4
:10eb6000e487570096ff370020ef2c00801f7800c5
:10eb700080062000a6890200000000000003eb00d0
:10eb8000e5042000840620004305200072ee2c00de
:10eb9000414c200040ad2c004089020000000000e4
:10eba0008f87e90084ff37000800fa00889fbe00c5
:10ebb0008a9fbe008c1f78008004780001057800d1
:10ebc0000000e00084003200595090000080fb00fb
:10ebd0000000d1000080fb00010020006f006000f9
:10ebe0008000eb007282570013002000e2ff2f002c
:10ebf000a2410200000000006e84570059489000b6
:10ec00000080fb000000d1000080fb00010020001c
:10ec10006f0060008000eb00080278001300200005
:10ec2000e2ff2f00a241020000000000d950900036
:10ec30000100d1006f006000728157000000e00009
:10ec400001003a00a2892c00821f78000100d10047
:10ec50006f00600021f12c0001003a00a1892c0016
:10ec6000811f7800ee9f4400d94890000100d10038
:10ec70006f0060000801780001003a00a2892c00b2
:10ec8000821f78000100d1006f00600021f12c008c
:10ec900001003a00a1892c00811f7800e69f440002
:10eca0008a0078000a00e00049003200811f7800e5
:10ecb00041f12c00811f7800608a020000000000f2
:10ecc0000006eb00f087570029d892000004e0000e
:10ecd000320032006865b8000a844400186092006f
:10ece0000080fb000000d1000080fb00010020003c
:10ecf0006f0060008000eb0072825700130020005c
:10ed0000e2ff2f00a2410200000000001860920004
:10ed100041f22c000078a30001003a00a1892c00e8
:10ed2000811f78000a804400106092000000d1002a
:10ed30006f006000f48057000000e00001003a001e
:10ed4000a1892c00811f78000a8044001060920085
:10ed50000000d1006f00600021f12c0001003a009a
:10ed6000a1892c00811f78000a804400a111200095
:10ed7000811f400060f22c00801f7800608a020032
:10ed800000000000ea8757000c06e80029d892002e
:10ed90000080fb00800f5600ceff3500f89f440036
:10eda000b90c9000891f780001f32c00811f7800b6
:10edb000608a020000000000e68757004f067800d6
:10edc0004f05be004f04be000080fa0000000600a0
:10edd000a1892c00b5ff370020f42c00801f78009b
:10ede000a0062000a6890200000000000003eb003e
:10edf000e5042000a40620004305200092f62c0024
:10ee0000d14f200040ad2c004089020000000000de
:10ee10008f87e9006cff3700889fbe000004be00aa
:10ee20000000e0000b0032000800be0019000700df
:10ee3000b809900078014400a4002000b1f72c002c
:10ee400010002000dc3e0200000000004f04be0065
:10ee50000000060000f82c00801f7800a0062000ab
:10ee6000a6890200000000000003eb00e50420007a
:10ee7000a40620004305200002fa2c0021532000a4
:10ee800040ad2c0040890200000000008f87e9009f
:10ee9000e5ff37000800fa00889fbe008a9fbe0089
:10eea0008c1f780080047800010578000000e000e5
:10eeb000d2003200595090000080fb000000d100c9
:10eec0000080fb00010020006f0060008000eb006c
:10eed0007282570013002000e2ff2f00a2410200bf
:10eee000000000006e845700594890000080fb002d
:10eef0000000d1000080fb00010020006f006000d6
:10ef00008000eb000802780013002000e2ff2f00d1
:10ef1000a241020000000000594990000280fb005d
:10ef2000c500de00e39f6000c700de00811f78009f
:10ef3000801f78000000d1006f006000880078001a
:10ef400001003a00b1fa2c00811f78000200d100c4
:10ef50006f00600021f12c0001003a00e1fa2c0062
:10ef6000811f7800e69f440061002000811f780027
:10ef7000595190000280fb00c500de00e39f600055
:10ef8000c700de00811f7800801f78000000d100dc
:10ef90006f006000a1fd2f008f8040000000e000a6
:10efa00001003a00b1fa2c00811f78000200d10064
:10efb0006f00600021f12c0001003a00e1fa2c0002
:10efc000811f7800ee9f440060002000801f7800c1
:10efd0008a0078000a00e00086003200811f780075
:10efe00001fb2c00811f7800608a020000000000f5
:10eff0000006eb000f02b10029d892000004e000e7
:10f00000380032006865b8000a8444001860920035
:10f010000080fb000000d1000080fb000100200008
:10f020006f0060008000eb00728257001300200028
:10f03000e2ff2f00a24102000000000018609200d1
:10f040004500de00e31f6000186092004700de000c
:10f05000e11f6000186092000080fb00801f7800b4
:10f06000186092000000d1006f006000f880570027
:10f070000000e00001003a00b1fa2c00811f780086
:10f080000a804400106092000000d1006f00600010
:10f0900021f12c0001003a00e1fa2c00811f7800d8
:10f0a0000a804400a1112000811f40006000200060
:10f0b000801f78000c04e800881f7800f1002d0004
:10f0c000811f7800608a020000000000f28757006c
:10f0d0000806780029d892000080fb00800f5400b9
:10f0e000c8ff3500595090000080fb004701de004a
:10f0f000594890000080fb004700de00c1032d004e
:10f10000804f51000400320081042d000204e00011
:10f1100001003a0081052d00811f780039f8920026
:10f120000080fb00801f780029f892000080fb001f
:10f13000801f780090062d00801f7800608a0200f2
:10f140000000000059f892000084fb00e887570097
:10f150000818a3002200320069f092000080fb0032
:10f16000801f780059f092000080fb00801f78001b
:10f1700049f092000080fb00801f780039f0920077
:10f180000080fb00801f78000930910099309100c9
:10f190005c1e020000000000809fbe00829fbe0037
:10f1a00069289100f92891005c1e0200000000000f
:10f1b000809fbe00829fbe0030092d000828a3005a
:10f1c00001003a00a0892c00801f7800b1092d00b1
:10f1d000811f7800608a020000000000fc87570051
:10f1e0004f0678004f05be004f04be000080fa00b5
:10f1f00000000600a1892c0078ff3700b00d2d001b
:10f20000801f7800a0062000a689020000000000f0
:10f210000003eb00e5042000a406200043052000c5
:10f22000f20f2d007154200040ad2c0040890200e7
:10f23000000000008f87e9001eff3700889fbe0096
:10f24000800478000000e00039003200a27c210038
:10f2500012417800e14f41002e00320029d892007f
:10f26000e74f500021003e008081fb006818b80085
:10f2700000804400a8112000000444000200fb00ac
:10f28000808f51000b0034006800540008017800a2
:10f2900080007800070009003159780000047800e8
:10f2a0008301e900cad7bf000000fb00808f510036
:10f2b000f5ff3c008181200008007800b8050200bd
:10f2c000000000002048d40001ceb30001407000cf
:10f2d0007044980029d892000040e800a0dc9a0011
:10f2e0000000eb004f04be0000000600800020007c
:10f2f000801f7800e0372d00801f7800a0202000bc
:10f30000a689020000000000e0ff2f00e4875700fc
:10f31000f4ff3700b03a2d00801f7800608a0200a9
:10f32000000000000080eb008f87e900edff370050
:10f33000503d2d00801f7800a0062000a689020005
:10f34000000000000003eb00e5042000a4062000fc
:10f3500043052000223f2d00a15e200040ad2c007f
:10f3600040890200000000008f87e900b7ff3700e6
:10f37000800178000001eb006410b800e47a2c00f2
:10f38000840040001180fb00808f51000400320097
:10f390000201e800e70f5100f7ff3600000005000a
:10f3a00011009000000006003000fa00889fbe00a7
:10f3b0008a9fbe008c1f7800800578000000e00066
:10f3c0009a0132005b5090000000d1006f00600095
:10f3d000120032008004eb006e8545000904d00065
:10f3e00042582d0002044400180078008e040200e8
:10f3f00000000000000178008a0078001800780002
:10f4000000060200000000000000e000830132005e
:10f410008904e800f98f5400f0ff3600ca15200077
:10f420000b054500f88445003b0c9000d0c7b300a5
:10f43000994f1000690132005bf892000004a000af
:10f44000d0fd9a00194078000080fb0001002000e8
:10f450007c005000e0805800f2052000820f500030
:10f46000e08f58006b003e0000600100140137007f
:10f47000130137006700370066003700650037006a
:10f480006e00370063003700620037005700370016
:10f49000600037005f003700090137005d0037006a
:10f4a0005c0037005b0037005a0037005900370016
:10f4b0005800370057003700a600370055003700c6
:10f4c0005400370053003700520037005100370016
:10f4d000500037004f0037004e0037004d00370016
:10f4e0004c0037004b0037004a0037004900370016
:10f4f00052003700470037004600370095003700bc
:10f500004400370043003700420037004100370015
:10f51000400037003f0037003e0037003d00370015
:10f520003c0037003b0037003a0037003900370015
:10f530003800370037003700360037003500370015
:10f540003400370033003700320037003100370015
:10f55000300037002f0037002e0037002d00370015
:10f560002c0037002b0037002a0037002900370015
:10f57000280037002700370026003700d00037006a
:10f580002400370023003700220037002100370015
:10f59000200037001f0037001e0037001d00370015
:10f5a0001c0037001b0037001a0037001900370015
:10f5b0001800370017003700160037001500370015
:10f5c0001400370013003700120037001100370015
:10f5d000100037000f0037000e0037000d00370015
:10f5e0000c0037000b0037000a0037000a017800d2
:10f5f00088007800090078009c910200000000005b
:10f600000000e00003003a005bf892000014a00044
:10f61000d0fd9a005bf89200620060000000cf000d
:10f620000000e9004f00de004f0678004f05be00e5
:10f630004f04be000080fa00000006005980fb0065
:10f64000d0050200000000000000e00027003200aa
:10f65000820020008900780060fc2f000f0040002d
:10f6600044040200000000000046eb00eccf9f00c5
:10f670008000eb0060fc2f000f004000fb00070043
:10f68000008dbe00f2ff2f00f3f72700801f02005d
:10f69000000000000000e000deff3200e9844400ca
:10f6a000e0fd2f0000844700920020000800be000b
:10f6b0004404020000000000fce79f00110020004d
:10f6c00008007800e900070020059800310598003f
:10f6d000f2ff2f00f3f72700801f02000000000058
:10f6e0000000e000cbff3200c7ff37008000eb00d6
:10f6f0000900780018020700008dbe00f2ff2f00fd
:10f70000f3f72700801f0200000000000000e00067
:10f71000c0ff3200e9844400110020000900780095
:10f720000d0207002005980031059800f2ff2f0018
:10f73000f3f72700801f0200000000000000e00037
:10f74000b4ff32005bf892000034a000d0fd9a00b4
:10f75000adff37008904e80069449000f0c2b300af
:10f76000804f540036003200a0c7b300804f5400d1
:10f770003300320080c6b300804f5400a5ff3a002a
:10f780002100200009007800b440020000000000c1
:10f79000005d9800f74f50009eff3e008984e8000e
:10f7a0002100200009007800b440020000000000a1
:10f7b000105d9800b8c3b300804f540095ff390026
:10f7c0008984e8002100200009007800b44002008c
:10f7d00000000000205d9800804f54008dff39002c
:10f7e000e3844400820020008900780060fc2f0040
:10f7f0000f00400044040200000000000046eb003f
:10f80000eccf9f008000eb0060fc2f000f00400059
:10f8100096000700008dbe00f2ff2f00f3f72700cf
:10f82000801f0200000000000000e00079ff3200ad
:10f83000e9844400e2fd2f00028447009aff37006c
:10f840002100200009007800b44002000000000000
:10f85000705598000040e900fe4f50006dff3e00db
:10f860008984e8002100200009007800b4400200eb
:10f8700000000000005d9800f74f500065ff3e005b
:10f880008984e8002100200009007800b4400200cb
:10f8900000000000105d9800b2c3b300804f51001b
:10f8a0005cff3900a0c7b300804f5400ccff3a0082
:10f8b0005bf892000044a000d0fd9a00c8ff37001a
:10f8c0005bf892000024a000d0fd9a006b489000e5
:10f8d000070207006a00b900000478007b48900026
:10f8e00003020700000444006140b9009a1e0200b0
:10f8f00000000000008dbe000b509000fc010700ce
:10f900006a00b900000478001b509000f80107005d
:10f91000000444006140b9009a1e0200000000008b
:10f920009288280083c82300242d020000000000d4
:10f930000001be001a00be005629020000000000af
:10f94000008dbe002b509000e90107006a00b9004d
:10f95000000478003b509000e501070000044400db
:10f960006140b9009a1e020000000000e2332c0042
:10f97000e3922300242d0200000000000001be00dd
:10f980001a00be005629020000000000008dbe00d3
:10f990001b509000ef0107000000e00003003a0058
:10f9a0001a00be0001f0a200008dbe003b50900086
:10f9b000e8010700000478002b509000e5010700e3
:10f9c000800078000900e80008417800ed01070098
:10f9d00020059800310598000bff37005bf8920076
:10f9e0000074a000d0fd9a00a10320000900780057
:10f9f0004406020000000000000178001000200012
:10fa00000200e00008ff32000280540000004400c1
:10fa10000004e9008204e80087fe37005bf89200ea
:10fa20000064a000d0fd9a007cfe3700805b2d00b2
:10fa3000801f780040002000a6890200000000001e
:10fa40000003eb00e5042000440020001304200024
:10fa5000425e2d0061032000205f2d0040890200de
:10fa6000000000008f87e90056fe3700889fbe0027
:10fa70008a9fbe008c9fbe008e1f78008005780094
:10fa8000010478000000e000020032001004e000f1
:10fa90000f003a00905f2d00801f780010012000b9
:10faa000a6890200000000000003eb00e50420002e
:10fab000140120001304200012622d00e118200020
:10fac000205f2d0040890200000000008f87e900c0
:10fad0000800e00063003a00210020000b007800dd
:10fae000b440020000000000000778000001780028
:10faf0000000e00059003500f4ff2f00f5f7270063
:10fb0000a0052000800f510049003c008b85e800d3
:10fb1000210020000b007800b4400200000000002b
:10fb200000047800000178000000e0004900350082
:10fb3000f4ff2f00f5f72700b0032000800f5100dd
:10fb40003b003c00e3854500210020000b007800cd
:10fb5000b440020000000000000578006140b900d8
:10fb60009a1e0200000000000004be006150b900af
:10fb70009a1e020000000000a2702d0033c2230074
:10fb8000242d0200000000000001be000800be009d
:10fb900056290200000000000006be0001f0a1008e
:10fba0000200200003272400581e0200000000006d
:10fbb0000000e00024003d006170b9009a1e0200c0
:10fbc000000000000004be009288280083c82300c3
:10fbd0000c00be00242d0200000000000001be0049
:10fbe0000800be0056290200000000000004be000c
:10fbf00001f0a10002002000432b2400581e020047
:10fc0000000000000000e0000f003c00ab4090004e
:10fc1000e0c4b30080cf50000400320009f0a2001d
:10fc20006540400080cf500007003a000802be0047
:10fc30000400be004f0778004f06be004f05be000f
:10fc40004f04be0000000600f4ff2f00f5f7270068
:10fc5000f7ff37000001ea00b5ff37000001ea00b6
:10fc6000a5ff3700310020000b007800b4400200ef
:10fc70000000000000077800000178000000e000ac
:10fc80004e003500f4ff2f00f5f72700400b200051
:10fc9000800f5100e6ff3c00e38545002100200075
:10fca0000b007800b440020000000000000478005f
:10fcb000000178000000e0003e003500f4ff2f0056
:10fcc000f5f72700b0032000800f5100d8ff3c005b
:10fcd000e3854500210020000b007800b4400200bd
:10fce00000000000000578006140b9009a1e020083
:10fcf000000000000004be006150b9009a1e02001e
:10fd000000000000a2702d0033c22300242d020049
:10fd1000000000000001be000800be0056290200dd
:10fd2000000000000006be0001f0a100020020005b
:10fd300003272400581e0200000000000000e0001d
:10fd4000c1ff3d006170b9009a1e02000000000072
:10fd50000004be009288280083c823000c00be0067
:10fd6000242d0200000000000001be000800be00bb
:10fd700056290200000000000004be0001f0a100ae
:10fd80000200200043332400581e0200000000003f
:10fd90000000e000acff3c00ab40900050c4b3005a
:10fda00080cf5000a1ff320009f0a2007240400055
:10fdb0009cff37000001ea00c0ff37000001ea00a5
:10fdc000b0ff3700889fbe008a9fbe008c1f78005e
:10fdd0000005be000204be00040678000200e00038
:10fde0004d003200e48f54003a0036000c00e00071
:10fdf00030003a000a01be0000002000412b240020
:10fe0000442902000000000002fc2f00938b240014
:10fe1000242d020000000000da2202000000000091
:10fe200032fa2700b30020009c040200000000000a
:10fe30000203be000002be0010c2b300004c42002c
:10fe400092052200030020000600be009c04020070
:10fe5000000000000203be000002be0011c2b30099
:10fe60000140420010449800b20520000300200029
:10fe70000600be009c040200000000000203be0059
:10fe80000002be0011c2b3000140420020449800ad
:10fe900001404300304498000040eb00404498008b
:10fea000080078004f0678004f05be004f04be00e2
:10feb0000000060002002000433324000a00be00b8
:10fec000562902000000000002fc2f00938324004a
:10fed000cfff3700891f7800e1622d00811f780075
:10fee00010012000a689020000000000090378002c
:10fef000e50420001401200013042000f2652d0009
:10ff0000b1212000205f2d00408902000000000088
:10ff1000e4875700b5ff3700c0662d00801f7800ca
:10ff200010012000a6890200000000000003eb0081
:10ff3000e50420001401200013042000f2652d00c8
:10ff400071212000205f2d00408902000000000088
:10ff50008f87e900a3ff3700889fbe000004be0022
:10ff60000000e00003003200104078000004e000d0
:10ff700010003a0030692d00801f78001001200029
:10ff8000a6890200000000000003eb00e504200049
:10ff90001401200013042000b26b2d000125200065
:10ffa000205f2d0040890200000000008f87e900db
:10ffb000184078000080fb00b40520000480b900e0
:10ffc00052442f00020040006101b9001840900027
:10ffd0000080fb00010020000200400083804800f8
:10ffe0000401b8000488b9008081410056442f0004
:10fff000f7ff2f000201430083814b00284090004f
:020000040001f9
:100000000080fb00010020000200400083804800c7
:100010000401b800048ab900848141000201430050
:1000200083814b00384090000080fb0001002000dd
:1000300002014000838148001202b1000380b10038
:100040000900e0001a003a000200be009a1e0200f9
:100050000000000082c4220003632300242d02005c
:10006000000000000001be0000002000412b240021
:1000700044290200000000000004be0001f0a100bd
:1000800002002000432b2400581e02000000000044
:100090000000e00003003c000800be004f04be006a
:1000a00000000600f0ff2f00f1f72700fbff3700ec
:1000b0000200be009a1e02000000000082c422005e
:1000c000036b2300242d020000000000020020002a
:1000d00043332c0056290200000000000004be003b
:1000e00001f0a1000200200043332400e6ff3700a6
:1000f0000041780000cdb30000404100e94f5000be
:1001000005003e000280fb0002fd2f00820040003f
:100110000100780000000600f0cbb3000040410071
:10012000e94f500003003e000280fb00f2fb2f006d
:10013000f6ff370000cbb300004041008000eb0029
:10014000e94f5000f2ff3e000280fb0002fb2f004f
:10015000eeff37008040780000cdb30000c04000c3
:10016000e94f50000400360042062000c0c4b3002e
:1001700080cf500001003a000001eb00020078003f
:1001800000000600889fbe008a9fbe008c9fbe00b4
:100190000004780081447800824678000000e00086
:1001a0005200320098c04400fcc5500002c3b300a6
:1001b00002c04000e94f500046003e0000cbb300b3
:1001c00080c54500184090007c455000b0c3b30086
:1001d000804f55000200360040ccb300004545007a
:1001e000284090007c4650000b00fb00cf80de00d2
:1001f0009a1e0200000000000004be000b04e00094
:100200002e0035000a00fb00cf80de009a1e02009f
:10021000000000000a04e000230035009288280056
:1002200083c82300242d0200000000000001be004e
:100230000800be0056290200000000000004be00b5
:100240000c00fb00cf80de009a1e020000000000c0
:100250000c04e0000f003500e2332c00e392230091
:10026000242d0200000000000001be000800be00b6
:1002700056290200000000000d04e00001003200d9
:1002800001f0a2004f06be004f05be004f04be00a5
:100290000000060002002000033824005629020056
:1002a00000000000ecff37000200200003382400ab
:1002b0005629020000000000d8ff3700020020008d
:1002c0000338240056290200000000000004be008c
:1002d000ccff370062c2b30002c04000e94f5000bb
:1002e000b8ff3e0080457800b6ff3700806c2d00d7
:1002f000801f7800c0012000a689020000000000d5
:100300000003eb00e5042000c401200013042000da
:10031000226f2d0061292000205f2d0040890200fe
:10032000000000008f87e9009eff370002002000d8
:1003300003e82300242d0200000000001c2302001b
:10034000000000001002b00000000600004278002b
:10035000f6022000a23f2d008001eb0045512d0048
:10036000850f510009003100924f520010003200f9
:1003700012409000804f520006003200630141009d
:100380008301e800850f5100f7ff3900060078006f
:10039000000006002240900080cf5000f7ff3a0096
:1003a00010022000030040000003ea00f7ff3700be
:1003b0002240900080cf5000edff3a00160220004e
:1003c00003034300f1ff3700f2874700889fbe0018
:1003d0008a9fbe008c9fbe008e1f7800800678002a
:1003e000010778000000e000ae0132000100e000eb
:1003f000a4013200c215200002014000d2b79f00c4
:10040000c9f12000e0ff2f00800878000006eb0013
:1004100028428000e00f14001900310009599000b3
:100420008280fb0070032000808f50007801320032
:100430005b003c000080e900808f50003e003200ed
:100440000000e800808f5000150032000280fb00a1
:10045000801f7800647a2d00841f780050032000ec
:10046000a689020000000000e487570028428000af
:100470000c06e800fc844400880f5600e7ff3900b2
:10048000008feb00104280004f0778004f06be003f
:100490004f05be004f04be002f01b1000000060052
:1004a000195890000080fb000058a3000c003a008f
:1004b0000048a3000e003200090078008e040200fc
:1004c0000000000000017800e68046000900780086
:1004d00030440200000000000000e000e3ff3a00aa
:1004e0000c0f7800195890006f006000e6ff37008d
:1004f000620020008280460009007800304402003b
:10050000000000000000e000d8ff3a0019589000f9
:100510000068a300f2ff3200e94090008180fb00f8
:100520005d4890000000d1006f006000808f500097
:10053000ceff3a00eaff3700195890000080fb0018
:100540000058a300e6ff3a000048a300060032006e
:10055000090078008e04020000000000000178000d
:10056000ee804600d9ff370062002000ee80460092
:100570000900780030440200000000000000e000a4
:10058000baff3a00195890000068a300d4ff320067
:10059000e94090008180fb005d509000e1ff370052
:1005a00090032000808f5000f5003200910035004c
:1005b0000000e800808f5000410032000000e80099
:1005c000808f5000a1ff3a005df892000068a30000
:1005d000a7ff3a0049489000add89200814f5000e3
:1005e000a3ff3e000004e000310032000080fb0069
:1005f0000000e900e0b79f00ab1120008d854500a9
:1006000000057800efb09700810f500098ff3d0083
:10061000195890000080fb000058a300b0ff3a007a
:100620000048a3000d003200620020008b0078001b
:100630000900780030440200000000000000e000e3
:10064000a7ff32000a05e800e88545006fb1970072
:10065000820f550085ff3d00edff37000b0078004d
:100660008e04020000000000000178008b0078007a
:100670000900780030440200000000000000e000a3
:10068000f0ff3a00195890000068a30094ff320070
:10069000e94090008180fb007b4090000000d10089
:1006a0006f006000808f5000e6ff3a008cff37003b
:1006b0000000eb008180fb00e1b79f00ceff370018
:1006c0005df892000018a30069ff32002c08e200d8
:1006d00043003200b2b78000c3b78000d0b78000bb
:1006e000e1b78000dfb2970025029000b5029000cc
:1006f000849fbe003fb297001403be000002be00fc
:10070000e1fd2f008f8040007e80570024430200cf
:1007100000000000e48757000000e00029003a00d4
:100720001fb59700afb597001901be000a00be00c3
:10073000581e0200000000000000e0004bff3500e2
:1007400039019000c90190000a00be00801f02001c
:10075000000000000000e00044ff3c003fb09700b4
:10076000cfb09700f0b79f0081bf9f006901900054
:10077000f9019000581e0200000000000000e00097
:100780003aff3500190d9000a90d90006011b800d6
:100790000a00be0052230200000000000000e0003a
:1007a0004fff32000a01be007fb097008fb897005c
:1007b000801f0200000000000000e0002bff3c0052
:1007c00047ff3700c57d2d00851f780030032000ce
:1007d000a6890200000000008f87e90023ff370090
:1007e0008240800093408000a0408000b1408000a3
:1007f000bcff37005df892000018a3001cff320018
:10080000194078008080fb00e48f500050003200d7
:1008100023003c00e28f50001800320011003c0021
:10082000e18f5000060032000080fb00801f78003e
:10083000f07f2d00801f78002003200008ff370084
:100840005fb197001200be0039019000c90190000d
:10085000581e0200000000000000e00004ff340009
:100860001fff3700dfb2970025009000b500900011
:1008700069019000f9019000f5ff37005fb2970021
:100880001400be0039019000c9019000581e0200fa
:10089000000000000000e000f5fe3400f1ff37002a
:1008a000e68f500021003200e58f50001a0034001e
:1008b000e78f500014003200e88f5000daff3a0052
:1008c0005fb297001400be0039019000c90190008a
:1008d000581e0200000000000000e000e4fe3400aa
:1008e000dfb2970025009000b500900069019000ec
:1008f000f9019000801f0200000000000000e000ed
:10090000dbfe3d00f6fe37005fb19700220090004d
:10091000b2009000f5ff37005fb297001400be00f0
:1009200039019000c9019000f2ff3700dfb2970053
:100930001500be0039019000c9019000801f02001f
:10094000000000000000e000c9fe3d00eeff37009f
:100950005fb197001200be0039019000c9019000fc
:10096000801f0200000000000000e000c0fe3d000b
:100970005fb2970024009000b4009000bcff3700e5
:100980005df892000018a300b9fe3200dfb09700b6
:100990001105be001901be000a00be00801f020042
:1009a000000000000000e000b1fe3c006901900082
:1009b000f90190000a00be00581e0200000000006d
:1009c0000000e000aafe35005fb19700220590000c
:1009d000b205900039019000c90190000a00be00e4
:1009e000581e0200000000000000e000a0fe3500dc
:1009f00019099000a90990000a00be00801f02009a
:100a0000000000000000e00099fe3c00b4fe37004a
:100a10005df892000018a30095fe32006902900074
:100a2000f902900039019000c9019000dfb09700f1
:100a300021009000b1009000809fbe003fb0970061
:100a40001003be00e1fd2f008f8040007e80570024
:100a50002443020000000000e48757000000e0008b
:100a600004003a001901be003fb09700cfb09700d4
:100a70004fff3700c17d2d00811f7800100320003b
:100a800053ff3700b1832d00811f7800e002200062
:100a9000a689020000000000100020008f87e900f6
:100aa00079fe370070862d00801f7800d00220006c
:100ab000f7ff37005000fa00889fbe008a9fbe00f3
:100ac0008c1f780080342000801f7800c101200036
:100ad000811f7800e0012000801f78004408f800a2
:100ae00011892d00811f7800608a0200000000003b
:100af000ea8757004408e20013003a0010428000e1
:100b0000618d2d00e40f500004003200b18d2d00e6
:100b1000e80f500001003200018e2d00811f780087
:100b2000208e2d00801f7800608a020000000000e7
:100b3000e48757004f0678004f05be004f04be0003
:100b40000080fa000000060081912d00811f7800ce
:100b500000922d00801f780051922d00811f780097
:100b6000c0922d00801f7800608a02000000000003
:100b700091942d00811f7800628d2d00114280001c
:100b800040062000808f500001003200b28d2d0001
:100b9000821f780020952d00801f7800608a020057
:100ba000000000000004eb00c9f12000ee875700b0
:100bb0004408e200dfff3200740547008b0220008a
:100bc0008e854500cc0320000e0646000e007800fe
:100bd000090009000018eb000a007800090009006c
:100be0000018eb000b007800090009000018eb006a
:100bf0000c007800090009000018eb00095990006a
:100c00008280fb0070032000808f5000fa003200c9
:100c10004f003c000080e900808f5000240032002b
:100c20000000e800808f5000210032008c1f780007
:100c30008b1f78008a1f78008e1f78000280fb00cf
:100c40000f010700801f7800195890000080fb00fa
:100c500080007800010fb200811f78006f006000f3
:100c6000b18d2d00e80f500004003200618d2d0081
:100c7000e40f500001003200018e2d00811f78002a
:100c80000804e800881f780050962d00801f780027
:100c9000608a020000000000f2875700fc844400d4
:100ca00020428000800f5400c8ff3900a1ff3700a8
:100cb000195890000080fb000058a3000300320088
:100cc000a0c2b300004f7800d8ff37000048a3004f
:100cd0001a003a000068a3000e003200694090003c
:100ce0000080fb00801f7800891f780061002000d1
:100cf000811f780080982d00801f78000e007800fa
:100d00006006020000000000e887570009599000c3
:100d1000c6ff3700891f780061002000811f78001e
:100d200010992d00801f78000e00780060060200e8
:100d300000000000e6875700f4ff3700891f7800a5
:100d400061002000811f780070992d00f5ff3700a9
:100d500090032000808f50007e0032005c00350040
:100d60000000e800808f50002c0032000000e800f6
:100d7000808f5000adff3a00494890000004e00029
:100d80002300320001c3b300014f40001958900006
:100d90000080fb000058a30003003200a0c2b30093
:100da000004d7800a1ff37000048a30013003a006f
:100db0000068a3000a003200694090000080fb0038
:100dc000801f7800891f780060002000801f780055
:100dd00081982d00811f78000a007800c8ff370035
:100de000891f780060002000801f780011992d0075
:100df000811f78000a007800ccff3700891f780037
:100e000060002000801f780071992d00f8ff3700e6
:100e1000a0c2b300004f7800dcff37001900be000d
:100e20005c1e020000000000809fbe00829fbe008a
:100e3000e0992d00801f78000e0078006006020007
:100e40000000000039009000c90090005c1e020004
:100e500000000000809fbe00829fbe00c19a2d004e
:100e6000811f78000a007800600602000000000080
:100e700069009000f90090005c1e02000000000074
:100e8000809fbe00829fbe00a09b2d00801f780027
:100e90000b007800600602000000000019089000b6
:100ea000a90890005c1e020000000000809fbe00a8
:100eb000829fbe00619c2d00811f78000c0078008d
:100ec00060060200000000008f02b1008fff3700b3
:100ed0001980fb000000d00041792d00e09f7800d0
:100ee000209d2d00801f78000e0078006006020013
:100ef0000000000039009000c90090005c1e020054
:100f000000000000809fbe00829fbe00c19d2d009a
:100f1000811f78000a0078006006020000000000cf
:100f200069009000f90090005c1e020000000000c3
:100f3000809fbe00829fbe00b09e2d00801f780063
:100f40000b0078006006020000000000f8875700e0
:100f50006eff37001900be005c1e0200000000009a
:100f6000809fbe00829fbe00919f2d00811f780050
:100f70000e007800600602000000000039009000ba
:100f8000c90090005c1e020000000000809fbe00af
:100f9000829fbe0090a02d00801f78000a0078007c
:100fa000600602000000000069009000f900900057
:100fb0005c1e020000000000809fbe00829fbe00f9
:100fc00091a12d00811f78000b00780060060200bf
:100fd0000000000019089000a90890005c1e0200a3
:100fe00000000000809fbe00829fbe0090a22d00e6
:100ff000801f7800b1ff37001900be005c1e0200a0
:1010000000000000809fbe00829fbe0081a32d00d3
:10101000811f78000e0078006006020000000000ca
:1010200039009000c90090005c1e02000000000022
:10103000809fbe00829fbe00c09d2d00801f780053
:101040000a007800600602000000000069009000bd
:10105000f90090005c1e020000000000809fbe00ae
:10106000829fbe00b19e2d00811f78000b0078008a
:101070006006020000000000fe87570023ff3700d3
:10108000800178000082eb000001eb006410b800e2
:10109000c5742d0005004000908f51000b003200f8
:1010a0000201e800eb0f5100f8ff3600607c2100e0
:1010b000e10f4200040032006420b800a2742d0049
:1010c00060007900000006000000060002027800bf
:1010d000f6ff3700f30f20008234200081382f0004
:1010e000c0f12000d6ac0400000000000400fa00ab
:1010f000889fbe008a9fbe0081057800a200200064
:10110000110009000280d800e1f79f0011000900da
:101110000280d800d1f79f00110009000280d8009a
:10112000c1f79f00d4a2a800a00f2000010020005a
:10113000fc9b020000000000d4a2a900a00f200028
:1011400001002000fc9b020000000000d4a2a800c7
:10115000a00f200001002000fc9b02000000000006
:10116000d4a2a900a00f200001002000fc9b0200d7
:1011700000000000d4a2a800a00f20000100200061
:10118000fc9b020000000000d4a2a900a00f2000d8
:1011900001002000fc9b020000000000d4a2a80077
:1011a000a00f200001002000fc9b020000000000b6
:1011b000d4a2a900c05d200001002000fc9b020019
:1011c000000000000005eb006c8057008004450023
:1011d000194078000004e000220032000004eb0017
:1011e0000e003200d4a2a800401f20000100200001
:1011f000fc9b020000000000d4a2a900401f2000b8
:1012000001002000fc9b0200000000000804e80030
:101210001980fb00800f5400f2ff3500c05d2000f4
:1012200001002000fc9b0200000000000a05e8000d
:10123000e20f5500e4ff34000b00e000050032002f
:10124000c05d200001002000fc9b020000000000a7
:10125000b4ff37004f05be004f04be000080fa0007
:1012600000000600d4a2a800007d2000010020009c
:10127000fc9b020000000000d4a2a900e7ff370099
:10128000889fbe008a9fbe008c9fbe008e1f780084
:101290000007780081067800020678008305780050
:1012a0008404780005057800060478000102200017
:1012b00010002000c8540200000000000000e00000
:1012c000130032003408e20011003200417b21009b
:1012d0009140780040c4b30080cf50000c00320031
:1012e000881f78008a1f7800891f78008b1f78007c
:1012f0008c1f78008d1f78008e1f780040a42d0071
:10130000801f7800608a020000000000f08757000c
:10131000b14180000900780074ff07000000fe0062
:101320004f0778004f06be004f05be004f04be00b9
:1013300000000600d422ef00f0f02f009016880085
:10134000d4a2a900d4e2a900000006000000fa001f
:10135000881f7800000478003408e2000b00320097
:10136000417b21009140780040c4b30080cf500001
:10137000060032000102200010002000c8540200c4
:10138000000000000000e0000b003a00301f2000c9
:10139000800f5400030036004f0478000080fa00ec
:1013a000000006008000eb0008007800768802004c
:1013b00000000000f8ff37003fb897000000e00091
:1013c00030003200823e2000110009000284d80063
:1013d000301f2000808f500024003600423f210043
:1013e00080a72d0005000900305978005800200022
:1013f000423f2100020244006108b8008001eb0076
:1014000032002000a24102000000000063044400fa
:10141000413f210001004400a1c3b30001587800fe
:10142000fac05000015878000048eb000884e8003a
:10143000c112200088805000423f21000200440079
:10144000ea8157003fb99700a4060200000000009f
:101450000004440008017800413f210010002000f2
:10146000c24c020000000000cbff3700423f2100c9
:10147000e0a72d0006000900305978006800200020
:10148000dbff370051a82d00811f7800c01220001b
:10149000aeff070008037800e5042000c412200016
:1014a0000305200002aa2d009104200060aa2d004f
:1014b00040890200000000008f87e900c1ff37006b
:1014c0000000fa003408e2001a003200417b2100db
:1014d0009140780040c4b30080cf50001500320026
:1014e0000102200010002000c8540200000000008b
:1014f0000000e0000f0032004fb897000000e0004d
:101500000e003200c0122000e88157004fb997004a
:1015100080007800403f2100a40602000000000087
:1015200000017800413f210010002000c24c020061
:10153000000000000080fa0000000600e0aa2d0074
:10154000801f7800d012200080ff07000003eb000e
:10155000e5042000d412200003052000a2ac2d00d9
:101560002108200060aa2d00408902000000000030
:101570008f87e900e3ff37000400fa00881f780036
:10158000000478000000e0006f0032000081eb00f2
:101590006602440063002000c810dd003480fb00b8
:1015a000808070004810de000000d00062672900d3
:1015b00002004000108168008301e900e18f4100d2
:1015c000f5ff3a006e02440063002000c810dd0001
:1015d0003480fb00808070004810de000000d000e6
:1015e0006567290005004000108168008301e9005b
:1015f000e18f4100f5ff3a00820178007802440053
:10160000380990000201e900e10f41000b003200af
:10161000c818dd003480fb00808070004818de00b0
:101620000000d0006367290003004000908168003b
:101630000201e900e10f4100f5ff3a00584890002f
:101640000000d1006f406000a0ff9f000040eb0051
:10165000b0ff9f00c0ff9f0003027800e6815700a3
:1016600022002000c820dd003380fb008080700055
:101670004820de000000d00064672900040040001c
:10168000108268000201e900e10f4100f5ff3a0015
:101690008201780045b920008000eb00520920004b
:1016a00025009000800f5200250032008100e800e4
:1016b000e6824200828f5000f9ff3600e18f410040
:1016c0000f0032001501be00704180000000410093
:1016d000e08049001801be0014002000820f500075
:1016e000838f580002003e00828abe000002eb0099
:1016f000040078004f0478000080fa000000060023
:10170000c37880006618b80085b920000501400044
:101710000409780042b92000020040001802be000f
:101720000488be008301e800c378880050092000c7
:10173000808f5100edff3400182fef00ebff3700d2
:1017400081017800ddff370020ad2d00801f78007b
:1017500050192000a6890200000000000003eb00e1
:10176000e5042000541920004304200092af2d000e
:101770008103200040b02d004089020000000000dd
:101780008f87e90081ff37000002be000201e900f7
:10179000e10f41000a003200c820dd003580fb0067
:1017a000808070004820de000000d000608079005a
:1017b000008268000201e900e10f4100f6ff3a00f3
:1017c0000400780000000600f30f20004200200013
:1017d00001002f0000802000d6ac020000000000b5
:1017e000f30f20004200200041002f004080200025
:1017f000d6ac020000000000f30f200042002000e1
:1018000081002f0080802000d6ac02000000000084
:10181000f30f200042002000c1002f00c0802000f4
:10182000d6ac020000000000f30f200042002000b0
:1018300001012f0000812000d6ac02000000000052
:10184000f30f20004200200041012f0040812000c2
:10185000d6ac020000000000f30f20008200200040
:1018600081012f0080812000d6ac02000000000022
:10187000f30f20002200200001022f000082200030
:10188000d6ac0200000000002008f8008081200093
:10189000801f7800c3b02d00831f780090b820000f
:1018a000600602000000000090b820008e040200d4
:1018b0000000000093ebb700f30f2000220020008f
:1018c00021022f0020822000d6ac02000000000080
:1018d000f30f20002200200041022f004082200050
:1018e000d6ac020000000000f30f20002200200010
:1018f00061022f0060822000d6ac020000000000d0
:10190000f30f20002200200081022f00808220009f
:10191000d6ac020000000000f30f200022002000df
:10192000c10b2f00c08b2000d6ac020000000000cd
:10193000f30f200022002000e10b2f00e08b20009d
:10194000d6ac020000000000f30f2000020c2000c3
:10195000010c2f00008c2000d6ac0200000000001b
:10196000f30f20008220200001182f000098200093
:10197000d6ac020000000000f30f2000220020007f
:10198000c1032f00c0832000d6ac0200000000007d
:10199000f30f200022002000a1022f00a0822000cf
:1019a000d6ac020000000000f30f2000220020004f
:1019b000c1022f00c0822000d6ac0200000000004f
:1019c000f30f200022002000e1022f00e08220001f
:1019d000d6ac020000000000f30f2000220020001f
:1019e00001032f0000832000d6ac0200000000009d
:1019f000f30f20002200200021032f00208320006d
:101a0000d6ac020000000000f30f2000a20020006e
:101a1000210b2f00208b2000d6ac0200000000001c
:101a2000f30f20002200200001042f00008420007a
:101a3000d6ac020000000000f30f200022002000be
:101a400041032f0040832000d6ac020000000000bc
:101a5000f30f20002200200061032f00608320008c
:101a6000d6ac020000000000f30f2000220020008e
:101a700081032f0080832000d6ac0200000000000c
:101a8000f30f200022002000a1032f00a0832000dc
:101a9000d6ac020000000000f30f2000220020005e
:101aa000e1032f00e0832000d6ac0200000000001c
:101ab000f30f20002200200021042f0020842000aa
:101ac000d6ac020000000000e687570011428000fb
:101ad00000052000808f50002700320006003600ed
:101ae00040062000808f5000030032006c00400050
:101af000808f5000200032004000200010428800fb
:101b0000f30f20002200200041042f004084200019
:101b1000d6ac020000000000f30f200002042000f9
:101b200061042f0060842000d6ac02000000000099
:101b30000001eb006810b80063842000030040003f
:101b40001004e000030032000201e800e70f51003a
:101b5000f8ff34000200780088ebb7009475ef00be
:101b6000f30f2000c202200061082f0060882000cf
:101b7000d6ac04000000000080002000dfff37002a
:101b8000881f7800417b21009140780070c4b30029
:101b900080cf5000a1003200417b210091407800ad
:101ba0006340500080cf50009c00320001022000b2
:101bb00010002000c8540200000000000000e000f7
:101bc000960032009041800080007800f107b2005a
:101bd000811f78004800de00801f78003008f80080
:101be0003e08f8002e08f8002408f8002208f80043
:101bf0004040800051408000809fbe002040800017
:101c000031408000809fbe00004080001140800075
:101c1000809fbe006040800071408000809fbe00b9
:101c2000a0408000b14080005c1e02000000000067
:101c3000809fbe00829fbe00804080009140800057
:101c40005c1e020000000000809fbe00829fbe005c
:101c50004008e2008500320020b12d00801f78008e
:101c60002008f80081812000811f78006200200098
:101c7000821f780080382000801f7800a1ea2d00a4
:101c8000811f780052b12d00821f7800608a020007
:101c900000000000cf03b1002608e200710032000e
:101ca00000c12d00801f78002a08e2006b0032007e
:101cb00000c12d00801f7800218b2000811f78003b
:101cc00062882000821f780030c12d00801f7800bc
:101cd000608a02000000000088cbbf0091c52d0083
:101ce00001003a00a1c52d00811f78000080fb0093
:101cf000801f780011c62d00811f7800608a0200c5
:101d0000000000000004eb00f087570088cbbf0004
:101d10000080fb00e00f100015003d000000e9000e
:101d200091c52d00800f54000100320041c72d00e5
:101d3000811f78006840b80062842000821f400044
:101d400080002000801f780061c72d00811f78006f
:101d5000608a020000000000e88757000804e800dd
:101d600088cbbf000080fb00800f5400ebff3500e4
:101d700010428000d1c72d00e40f50000400320053
:101d800021c82d00e80f50000100320071c82d005d
:101d9000811f78004408f8003808e2002d00320066
:101da00090c82d00801f78003608e200270032001e
:101db00090c82d00801f78003c08e200210032000e
:101dc00090c82d00801f78003a08e2001b00320006
:101dd00090c82d00801f78002c08e200150032000a
:101de00090c82d00801f78002808e2000f00320004
